:020000040800F2
:1078000000A00020AD700208D1910008D7910008B7
:10781000F1910008F7910008FD91000800000000B8
:1078200000000000000000000000000003920008BB
:1078300011920008000000001F9200082D9200081D
:10784000FD700208F5B60108FD700208FD7002081F
:10785000FD700208FD700208FD700208FD7002084C
:10786000FD700208FD700208FD700208FD7002083C
:107870003D92000851920008FD700208FD70020858
:107880006592000879920008DD910008FD700208F9
:107890008D920008FD700208FD700208A192000898
:1078A000FD700208C5920008FD700208FD70020814
:1078B000FD700208FD700208D9920008FD700208F0
:1078C000FD700208FD700208FD700208FD700208DC
:1078D000FD700208FD700208F9920008119300087B
:1078E000FD700208FD700208FD7002080000000033
:1078F0000000000000000000000000000000000088
:10790000000000000000000000000000FD70020800
:10791000FD700208FD700208FD7002080000000002
:10792000FD700208FD700208FD700208FD7002087B
:10793000FD700208000000000000000000000000D0
:10794000FD700208FD700208000000000000000049
:107950000000000000000000000000000000000027
:107960000000000000000000FD700208FD70020829
:10797000FD70020800000000000000000000000090
:0879800000000000FD70020888
:1079900010B5054C237833B9044B13B10448AFF349
:1079A00000800123237010BDD005002000000000DE
:1079B000BC9B020808B5034B1BB103490348AFF356
:1079C000008008BD00000000D4050020BC9B020818
:1079D00010F8012B11F8013B012A28BF9A42F7D079
:1079E000D01A7047034613F8012B002AFBD1181A4E
:1079F0000138704700000000000000000000000097
:107A000001F0FF01102A2BDB10F0070F08D010F84F
:107A1000013B013A8B422DD010F0070F42B3F6D153
:107A2000F0B441EA012141EA014122F007047FF06C
:107A300000070023F0E80256083C85EA010586EAC3
:107A4000010685FA47F5A3FA87F586FA47F6A5FAFF
:107A500087F68EB9EED1F0BC01F0FF0102F007020B
:107A600032B110F8013B013A83EA010313B1F8D1B6
:107A70000020704701387047002D06BF3546033897
:107A8000073815F0010F07D1013015F4807F02BFD0
:107A9000013015F4C03F0130F0BC0138704700BF21
:107AA00070B54FF0FF0C4CF4E06C1CEA11541DBF94
:107AB0001CEA135594EA0C0F95EA0C0F00F0DEF85F
:107AC0002C4481EA030621EA4C5123EA4C5350EA44
:107AD000013518BF52EA033541F4801143F4801395
:107AE00038D0A0FB02CE4FF00005E1FB02E506F026
:107AF0000042E0FB03E54FF00006E1FB03569CF07B
:107B0000000F18BF4EF0010EA4F1FF04B6F5007F80
:107B100064F5407404D25FEA4E0E6D4146EB0606F2
:107B200042EAC62141EA55514FEAC52040EA5E507B
:107B30004FEACE2EB4F1FD0C88BFBCF5E06F1ED825
:107B4000BEF1004F08BF5FEA500E50F1000041EB5C
:107B5000045170BD06F0004646EA010140EA020009
:107B600081EA0301B4EB5C04C2BFD4EB0C0541EA2B
:107B7000045170BD41F480114FF0000E013C00F340
:107B8000AB8014F1360FDEBF002001F0004170BD64
:107B9000C4F10004203C35DA0C341BDC04F114047D
:107BA000C4F1200500FA05F320FA04F001FA05F209
:107BB00040EA020001F0004221F0004110EBD370D6
:107BC00021FA04F642EB06015EEA430E08BF20EA02
:107BD000D37070BDC4F10C04C4F1200500FA04F3A5
:107BE00020FA05F001FA04F240EA020001F0004137
:107BF00010EBD37041F100015EEA430E08BF20EAAA
:107C0000D37070BDC4F1200500FA05F24EEA020EF1
:107C100020FA04F301FA05F243EA020321FA04F020
:107C200001F0004121FA04F220EA020000EBD370D7
:107C30005EEA430E08BF20EAD37070BD94F0000FD7
:107C40000FD101F00046400041EB010111F4801F0B
:107C500008BF013CF7D041EA060195F0000F18BFBC
:107C6000704703F00046520043EB030313F4801FF8
:107C700008BF013DF7D043EA0603704794EA0C0FB2
:107C80000CEA135518BF95EA0C0F0CD050EA4106C8
:107C900018BF52EA4306D1D181EA030101F0004145
:107CA0004FF0000070BD50EA410606BF104619466D
:107CB00052EA430619D094EA0C0F02D150EA013679
:107CC00013D195EA0C0F05D152EA03361CBF1046BA
:107CD00019460AD181EA030101F0004141F0FE4159
:107CE00041F470014FF0000070BD41F0FE4141F4DD
:107CF000780170BD81F0004102E000BF83F00043D5
:107D000030B54FEA41044FEA430594EA050F08BF36
:107D100090EA020F1FBF54EA000C55EA020C7FEAFA
:107D2000645C7FEA655C00F0E2804FEA5454D4EB77
:107D30005555B8BF6D420CDD2C4480EA020281EA41
:107D4000030382EA000083EA010180EA020281EA79
:107D50000303362D88BF30BD11F0004F4FEA0131CB
:107D60004FF4801C4CEA113102D0404261EB4101DA
:107D700013F0004F4FEA03334CEA133302D0524260
:107D800063EB430394EA050F00F0A780A4F101041C
:107D9000D5F1200E0DDB02FA0EFC22FA05F2801856
:107DA00041F1000103FA0EF2801843FA05F359413C
:107DB0000EE0A5F120050EF1200E012A03FA0EFCBB
:107DC00028BF4CF0020C43FA05F3C01851EBE371E5
:107DD00001F0004507D54FF0000EDCF1000C7EEB02
:107DE00000006EEB0101B1F5801F1BD3B1F5001F40
:107DF0000CD349085FEA30004FEA3C0C04F101045F
:107E00004FEA445212F5800F80F09A80BCF1004F87
:107E100008BF5FEA500C50F1000041EB045141EA09
:107E2000050130BD5FEA4C0C404141EB0101013CD2
:107E300028BFB1F5801FE9D291F0000F04BF0146C1
:107E40000020B1FA81F308BF2033A3F10B03B3F193
:107E500020020CDA0C3208DD02F1140CC2F10C0223
:107E600001FA0CF021FA02F10CE002F11402D8BF81
:107E7000C2F1200C01FA02F120FA0CFCDCBF41EA4D
:107E80000C019040E41AA2BF01EB0451294330BD1C
:107E90006FEA04041F3C1CDA0C340EDC04F11404F9
:107EA000C4F1200220FA04F001FA02F340EA0300D0
:107EB00021FA04F345EA030130BDC4F10C04C4F116
:107EC000200220FA02F001FA04F340EA03002946F6
:107ED00030BD21FA04F0294630BD94F0000F83F440
:107EE000801306BF81F480110134013D4EE77FEA23
:107EF000645C18BF7FEA655C29D094EA050F08BF6F
:107F000090EA020F05D054EA000C04BF194610464F
:107F100030BD91EA030F1EBF0021002030BD5FEA93
:107F2000545C05D14000494128BF41F0004130BDBB
:107F300014F580043CBF01F5801130BD01F000450F
:107F400045F0FE4141F470014FF0000030BD7FEA82
:107F5000645C1ABF194610467FEA655C1CBF0B467D
:107F6000024650EA013406BF52EA033591EA030F94
:107F700041F4002130BD00BF90F0000F04BF00218C
:107F8000704730B54FF4806404F132044FF00005BF
:107F90004FF0000150E700BF90F0000F04BF002138
:107FA000704730B54FF4806404F1320410F000459E
:107FB00048BF40424FF000013EE700BF42004FEA99
:107FC000E2014FEA31014FEA02701FBF12F07F4316
:107FD00093F07F4F81F06051704732F07F4208BFCD
:107FE000704793F07F4F04BF41F40021704730B5D4
:107FF0004FF4607401F0004521F000411CE700BF20
:1080000050EA010208BF704730B54FF000050AE0A2
:1080100050EA010208BF704730B511F0004502D5A3
:10802000404261EB41014FF4806404F132045FEAA5
:10803000915C3FF4D8AE4FF003025FEADC0C18BF4E
:1080400003325FEADC0C18BF033202EBDC02C2F140
:10805000200300FA03FC20FA02F001FA03FE40EAD2
:108060000E0021FA02F11444BDE600BF4FF0FF3CC0
:1080700006E000BF4FF0010C02E000BF4FF0010C22
:108080004DF804CD4FEA410C7FEA6C5C4FEA430C9B
:1080900018BF7FEA6C5C1BD001B050EA410C0CBFEA
:1080A00052EA430C91EA030F02BF90EA020F00204C
:1080B000704710F1000F91EA030F58BF994208BFB3
:1080C00090422CBFD8176FEAE37040F00100704770
:1080D0004FEA410C7FEA6C5C02D150EA013C07D1C7
:1080E0004FEA430C7FEA6C5CD6D152EA033CD3D012
:1080F0005DF8040B704700BF8446104662468C460C
:108100001946634600E000BF01B5FFF7B7FF00283E
:1081100048BF10F1000F01BD4DF808EDFFF7F4FF67
:108120000CBF012000205DF808FB00BF4DF808EDF2
:10813000FFF7EAFF34BF012000205DF808FB00BF15
:108140004DF808EDFFF7E0FF94BF012000205DF837
:1081500008FB00BF4DF808EDFFF7CEFF94BF0120EC
:1081600000205DF808FB00BF4DF808EDFFF7C4FFE5
:1081700034BF012000205DF808FB00BF4FEA410238
:1081800012F5001215D211D56FF47873B3EB625269
:1081900012D94FEAC12343F0004343EA505311F090
:1081A000004F23FA02F018BF404270474FF0000022
:1081B000704750EA013005D111F0004008BF6FF060
:1081C000004070474FF00000704700BF4A0011D2D6
:1081D00012F5001211D20DD56FF47873B3EB625221
:1081E0000ED44FEAC12343F0004343EA505323FA2D
:1081F00002F070474FF00000704750EA013002D1A2
:108200004FF0FF3070474FF00000704780B582B0EC
:1082100000AF264B264A9A6005F0BEF800F04CF8F5
:1082200000F0CCF800F012FB00F08EFA00F042FEF5
:1082300000F070FE00F0AAF900F03EFB00F0A0FB99
:1082400000F004FC13F054F800237B6006F0D4FC2B
:10825000786012F003FF1CF09DFB12F01DFB14F080
:10826000A3FF15F0A7F816F07FFB17F0B5FC17F089
:108270002FFC19F01BFD1EF0FDFE1BF00FFE0EF093
:1082800027F90DF0CBFF0CF077FC12F08BF912F010
:10829000EFF80EF031FE0AF0BDFF064BB3F91430D3
:1082A0001BB2012BD5D112F09BFDD2E700ED00E00F
:1082B00000780008183A002080B59CB000AF07F1A4
:1082C00048032822002118461EF05CFF07F1340302
:1082D00000221A605A609A60DA601A613B463422C2
:1082E000002118461EF04EFF0123BB644FF480337B
:1082F000FB6400233B650123BB6502237B664FF4CF
:108300008033BB664FF4E013FB6607F14803184661
:1083100005F09CF80346002B01D000F03FF80F2336
:108320007B630223BB630023FB634FF480633B64E6
:1083300000237B6407F134030221184606F03AFA61
:108340000346002B01D000F029F886233B60002370
:10835000FB6000233B614FF480737B623B46184611
:1083600006F030FD0346002B01D000F017F800BFE7
:108370007037BD4680BD000080B582B000AF786028
:108380007B681B68044A934201D105F01BF800BFCB
:108390000837BD4680BD00BF002C014080B400AF4F
:1083A00072B600BFFEE780B483B000AF786039607A
:1083B00000BF0C37BD465DF8047B704780B58AB0BE
:1083C00000AF07F1140300221A605A609A60DA6065
:1083D0001A61594B5B69584A43F400235361564B69
:1083E0005B6903F400233B613B69534B5B69524A71
:1083F00043F480035361504B5B6903F48003FB60DB
:10840000FB684D4B5B694C4A43F4003353614A4B64
:108410005B6903F40033BB60BB68474B5B69464A4A
:1084200043F480235361444B5B6903F480237B60F6
:108430007B6801224FF4F8714FF0904007F0E8F9A3
:10844000002244F207013D4807F0E2F94FF460438F
:108450007B610323BB610023FB6107F11403194611
:10846000374806F067FF40F202637B610323BB617C
:108470000023FB6107F1140319464FF0904006F00A
:1084800059FF4FF4A8737B611123BB610023FB618B
:1084900000233B6207F1140319464FF0904006F0A9
:1084A00049FF20237B611123BB610023FB61002373
:1084B0003B6207F1140319464FF0904006F03AFF73
:1084C00007237B610123BB610023FB6100233B6227
:1084D00007F114031946194806F02CFF4FF48043A6
:1084E0007B610123BB610123FB6100233B6207F138
:1084F00014031946114806F01DFF4FF440537B61E9
:108500000323BB610023FB6107F1140319460B48E9
:1085100006F010FF4FF440437B610023BB61012351
:10852000FB6107F114031946044806F003FF00BF7E
:108530002837BD4680BD00BF00100240000400483F
:108540000008004880B588B000AF0346FB71FB7996
:10855000122B14D107F10C0300221A605A609A60A2
:10856000DA601A614FF47043FB6000233B61022321
:108570007B6107F10C031946034806F0DBFE00BFE0
:108580002037BD4680BD00BF0004004880B58AB0DA
:1085900000AF07F11C0300221A605A609A603B1D6D
:1085A00000221A605A609A60DA601A615A613D4B83
:1085B0004FF0A0421A603B4B00225A60394B002218
:1085C0009A60384B00221A61364B00225A76354B9E
:1085D000002283F82020334B0022DA62314B012243
:1085E0009A62304B0022DA602E4B0122DA612D4B69
:1085F000002283F830202B4B04225A61294B0022A1
:108600001A76284B00225A63274B4FF0A0421A607B
:10861000254B00221A61244B00225A76224B00225D
:1086200083F82020204B01229A621F4B0022DA603F
:108630001D4B0122DA611B4802F0BAFF0346002BF2
:1086400001D0FFF7ABFE184802F0B2FF0346002B43
:1086500001D0FFF7A3FE0023FB6107F11C031946BD
:10866000104804F0ABFB0346002B01D0FFF796FE49
:1086700001237B600123BB6000233B610323FB607C
:1086800000237B610023BB613B1D1946054803F0B5
:1086900059FF0346002B01D0FFF780FE00BF2837AB
:1086A000BD4680BD3C060020EC05002080B58AB0A8
:1086B00000AF786007F1140300221A605A609A60D4
:1086C000DA601A617B681B68B3F1A04F33D11C4B91
:1086D0005B691B4A43F080535361194B5B6903F09C
:1086E00080533B613B69164B5B69154A43F4003389
:1086F0005361134B5B6903F40033FB60FB68012398
:108700007B610323BB610023FB6107F1140319465E
:108710004FF0904006F00EFE00220021122007F0DC
:1087200005FD122007F02EFD0021064803F052FE41
:10873000044803F01BFB00BF2837BD4680BD00BFC7
:10874000001002403C06002080B500AF174B184ACD
:108750001A60164B06225A60144B00229A60134B83
:108760000022DA60114B4FF400321A610F4B4FF4C4
:1087700080125A610D4B00221A760C4B01225A7658
:108780000A4B00229A76094B0022DA76074B002228
:108790001A77064B01225A77044807F0C1FF0346B7
:1087A000002B01D0FFF7FAFD00BF80BD8C06002032
:1087B0000064004080B58AB000AF786007F1140310
:1087C00000221A605A609A60DA601A617B681B683E
:1087D0001C4A934231D11C4BDB691B4A43F00073A6
:1087E000D361194BDB6903F000733B613B69164BA6
:1087F0005B69154A43F400335361134B5B6903F41F
:108800000033FB60FB684FF4C0537B610223BB6104
:108810000023FB6103233B6209237B6207F11403FE
:1088200019464FF0904006F085FD002200211420EB
:1088300007F07CFC142007F0A5FC00BF2837BD46DC
:1088400080BD00BF006400400010024080B582B0CF
:1088500000AF184B5B69174A43F001035361154B96
:108860005B6903F001037B607B68002200210C2020
:1088700007F05CFC0C2007F085FC002200210D2095
:1088800007F054FC0D2007F07DFC00220021102091
:1088900007F04CFC102007F075FC0022002111208D
:1088A00007F044FC112007F06DFC00BF0837BD46FF
:1088B00080BD00BF0010024080B58AB000AF07F154
:1088C0001C0300221A605A609A603B4600221A601C
:1088D0005A609A60DA601A615A619A61274B4FF0C8
:1088E00080421A60254B48225A60244B00229A602D
:1088F000224B44F61F62DA60204B00221A611F4BA4
:1089000000229A611D4800F0B7FF0346002B01D0FA
:10891000FFF744FD0023FB6100237B6207F11C038A
:108920001946164802F0EEFC0346002B01D0FFF773
:1089300035FD60233B6000237B600023BB60002388
:108940003B613B46002219460C4801F0EFFA034612
:10895000002B01D0FFF722FD3B46042219460748B1
:1089600001F0E4FA0346002B01D0FFF717FD03489E
:1089700000F026F900BF2837BD4680BDB4060020B0
:1089800080B58AB000AF07F11C0300221A605A605C
:108990009A603B4600221A605A609A60DA601A6157
:1089A0005A619A61274B284A1A60264B48225A601E
:1089B000244B00229A60234B44F61F62DA60214B5D
:1089C00000221A611F4B00229A611E4800F054FFDA
:1089D0000346002B01D0FFF7E1FC0023FB610023DD
:1089E0007B6207F11C031946164802F08BFC034614
:1089F000002B01D0FFF7D2FC60233B6000237B609B
:108A00000023BB6000233B613B46002219460D4812
:108A100001F08CFA0346002B01D0FFF7BFFC3B4668
:108A200004221946074801F081FA0346002B01D0C1
:108A3000FFF7B4FC034800F0C3F800BF2837BD4679
:108A400080BD00BF000700200004004080B588B052
:108A500000AF07F1100300221A605A609A60DA60D2
:108A60003B1D00221A605A609A601D4B1D4A1A6015
:108A70001B4B47225A601A4B00229A60184B44F64F
:108A80001F62DA60164B00221A61154B00229A61B0
:108A9000134800F0DDFC0346002B01D0FFF77EFCFD
:108AA0004FF480533B6107F1100319460C4801F065
:108AB00051FC0346002B01D0FFF770FC00237B60C4
:108AC0000023FB603B1D1946054802F01BFC0346D2
:108AD000002B01D0FFF762FC00BF2037BD4680BDF0
:108AE0004C0700200008004080B584B000AF7860DB
:108AF0007B681B68164A93420CD1164BDB69154AFA
:108B000043F00203D361134BDB6903F00203FB6004
:108B1000FB6818E07B681B680F4A934213D10D4B2A
:108B2000DB690C4A43F00403D3610A4BDB6903F0B1
:108B30000403BB60BB68002200211E2007F0F6FA88
:108B40001E2007F01FFB00BF1037BD4680BD00BFD1
:108B500000040040001002400008004080B485B0CE
:108B600000AF78607B681B68B3F1804F0CD1124B6B
:108B7000DB69114A43F00103D3610F4BDB6903F05A
:108B80000103FB60FB6810E07B681B680B4A9342A3
:108B90000BD1094BDB69084A43F00203D361064B52
:108BA000DB6903F00203BB60BB6800BF1437BD463E
:108BB0005DF8047B704700BF0010024000040040D5
:108BC00080B58CB000AF786007F11C0300221A60FA
:108BD0005A609A60DA601A617B681B68B3F1804F53
:108BE0003AD13F4B5B693E4A43F4003353613C4BFF
:108BF0005B6903F40033BB61BB69394B5B69384A7D
:108C000043F480235361364B5B6903F480237B611B
:108C10007B694FF40043FB6102233B6200237B62CC
:108C20000023BB620123FB6207F11C0319464FF0CE
:108C3000904006F07FFB0823FB6102233B62002388
:108C40007B620023BB620123FB6207F11C03194610
:108C5000244806F06FFB3FE07B681B68224A934282
:108C60001CD11F4B5B691E4A43F4802353611C4B8C
:108C70005B6903F480233B613B693023FB61022382
:108C80003B6200237B620023BB620223FB6207F18D
:108C90001C031946134806F04DFB1DE07B681B685A
:108CA000124A934218D10E4B5B690D4A43F480235C
:108CB00053610B4B5B6903F48023FB60FB684FF44B
:108CC0005073FB6102233B620023BB6207F11C036C
:108CD0001946044806F02EFB00BF3037BD4680BD64
:108CE000001002400004004800040040000800405A
:108CF00080B500AF0021124800F0AEFE04211048FC
:108D000000F0AAFE00210F4800F0A6FE04210D4845
:108D100000F0A2FE0A4B1B684FF47A725A63084BAC
:108D20001B684FF47A729A63064B1B684FF47A7291
:108D30009A63044B1B684FF47A725A6300BF80BD7C
:108D4000B40600200007002080B590B000AF0346B5
:108D5000FB7107F1300300221A605A609A60DA60F2
:108D600007F1240300221A605A609A6007F1080391
:108D700000221A605A609A60DA601A615A619A6138
:108D8000FB79122B40F08D80484B494A1A60474BC3
:108D900047225A60454B00229A60444B44F61F62BA
:108DA000DA60424B00221A61404B00229A613F4830
:108DB00000F04EFB0346002B01D0FFF7EFFA4FF413
:108DC00080533B6307F130031946384801F0C2FA7B
:108DD0000346002B01D0FFF7E1FA344800F04CFDC8
:108DE0000346002B01D0FFF7D9FA00237B62002352
:108DF000FB6207F1240319462C4802F083FA03466C
:108E0000002B01D0FFF7CAFA6023BB600023FB6090
:108E100000233B610023BB6107F1080300221946D0
:108E2000224801F083F80346002B01D0FFF7B6FA81
:108E300007F10803082219461C4801F077F8034699
:108E4000002B01D0FFF7AAFA07F108030C221946FC
:108E5000164801F06BF80346002B01D0FFF79EFA8D
:108E60001248FFF7ADFE0021104800F0F5FD082183
:108E70000E4800F0F1FD0C210C4800F0EDFD0B4B0D
:108E80001B6840F2DC525A63084B1B684FF47A723D
:108E9000DA63064B1B684FF47A721A64172007F0E6
:108EA00089F900BF4037BD4680BD00BF4C07002098
:108EB0000008004080B500AF144B154A1A60134BF0
:108EC0004FF4E1325A60114B00229A600F4B00229E
:108ED000DA600E4B00221A610C4B0C225A610B4BCC
:108EE00000229A61094B0022DA61084B00221A62C3
:108EF000064B00225A62054808F07EFC0346002B10
:108F000001D0FFF74BFA00BF80BD00BF98070020DB
:108F10000044004080B500AF144B154A1A60134B53
:108F20004FF4E1325A60114B00229A600F4B00223D
:108F3000DA600E4B00221A610C4B0C225A610B4B6B
:108F400000229A61094B0022DA61084B00221A6262
:108F5000064B00225A62054808F04EFC0346002BDF
:108F600001D0FFF71BFA00BF80BD00BF2008002022
:108F70000048004080B58CB000AF786007F11C035A
:108F800000221A605A609A60DA601A617B681B6876
:108F9000834A93427DD1834BDB69824A43F4003399
:108FA000D361804BDB6903F40033BB61BB697D4B4C
:108FB0005B697C4A43F4003353617A4B5B6903F489
:108FC00000337B617B690C23FB6102233B6200233E
:108FD0007B620323BB620723FB6207F11C03194674
:108FE0004FF0904006F0A6F96F4B704A1A606E4B36
:108FF00010225A606C4B00229A606B4B8022DA6020
:10900000694B00221A61684B00225A61664B0022AC
:109010009A61654B0022DA61634806F069FC0346F9
:10902000002B01D0FFF7BAF97B685F4A1A675E4AE6
:109030007B6853625E4B5F4A1A605D4B00225A6048
:109040005B4B00229A605A4B8022DA60584B002218
:109050001A61574B00225A61554B00229A61544BBA
:109060000022DA61524806F043FC0346002B01D08F
:10907000FFF794F97B684E4A5A674D4A7B68536202
:1090800000220021262007F051F8262007F07AF868
:1090900081E07B681B68484A93427CD1414BDB6985
:1090A000404A43F48023D3613E4BDB6903F48023C1
:1090B0003B613B693B4B5B693A4A43F48023536114
:1090C000384B5B6903F48023FB60FB684FF440631B
:1090D000FB6102233B6200237B620323BB62072305
:1090E000FB6207F11C031946344806F023F9344BA0
:1090F000344A1A60324B00225A60314B00229A6087
:109100002F4B8022DA602E4B00221A612C4B00225A
:109110005A612B4B00229A61294B0022DA612848C0
:1091200006F0E6FB0346002B01D0FFF737F97B681A
:10913000234A5A67224A7B685362234B234A1A60A8
:10914000214B10225A60204B00229A601E4B802235
:10915000DA601D4B00221A611B4B00225A611A4B28
:1091600000229A61184B0022DA61174806F0C0FB12
:109170000346002B01D0FFF711F97B68124A1A67EA
:10918000114A7B68536200220021272006F0CEFF9F
:10919000272006F0F7FF00BF3037BD4680BD00BF77
:1091A0000044004000100240A80800208000024057
:1091B000EC0800206C000240004800400004004819
:1091C0003009002030000240740900201C000240D9
:1091D00080B400AFFEE780B400AFFEE780B500AF1B
:1091E000024802F0D1FE00BF80BD00BF3C06002057
:1091F00080B400AFFEE780B400AFFEE780B400AFFC
:10920000FEE780B400AF00BFBD465DF8047B704749
:1092100080B400AF00BFBD465DF8047B704780B4EA
:1092200000AF00BFBD465DF8047B704780B400AF5F
:1092300000BFBD465DF8047B7047000080B500AFFD
:10924000024806F051FD00BF80BD00BF7409002038
:1092500080B500AF024806F047FD00BF80BD00BFEB
:109260003009002080B500AF024806F03DFD00BF88
:1092700080BD00BFEC08002080B500AF024806F0BA
:1092800033FD00BF80BD00BFA808002080B500AF3F
:10929000024808F081F800BF80BD00BF8C060020A6
:1092A00080B500AF402006F00BFB802006F008FBE5
:1092B0004FF4807006F004FB4FF4007006F000FBE2
:1092C00000BF80BD80B500AF024800F02DFD00BF9B
:1092D00080BD00BFBC09002080B500AF044800F08D
:1092E00023FD044B1B680133024A136000BF80BD9D
:1092F0004C070020B809002080B500AF034808F0F3
:109300007DFC02480AF016F800BF80BD98070020D7
:1093100080B500AF034808F071FC02480AF00AF873
:1093200000BF80BD2008002080B483B000AF0F4B89
:109330009B690E4A43F0010393610C4B9B6903F058
:1093400001037B607B68094BDB69084A43F080536B
:10935000D361064BDB6903F080533B603B6800BF81
:109360000C37BD465DF8047B704700BF001002401B
:1093700080B58CB000AF78600023BB6200237B62B5
:109380002E4B9B692D4A43F4006393612B4B9B69E1
:1093900003F40063BB60BB6807F10C0207F1100324
:1093A0001146184605F0CCFC05F0A8FCB862BB6A73
:1093B000234AA2FB03239B0C013B7B62214B224AE5
:1093C0001A60204B40F2E732DA601E4A7B6A536033
:1093D0001C4B00221A611B4B00229A60194B002281
:1093E0009A61184800F034F8034687F82F3097F850
:1093F0002F30002B1BD1134800F0A8F9034687F843
:109400002F3097F82F30002B11D1192006F0BAFE1B
:109410007B680F2B08D800227968192006F086FE99
:109420000A4A7B68136002E0012387F82F3097F81F
:109430002F3018463037BD4680BD00BF00100240B7
:1094400083DE1B43BC090020002C014000000020EB
:1094500080B582B000AF78607B68002B01D101231A
:10946000D2E07B681B686A4A934227D07B681B68FE
:10947000B3F1804F22D07B681B68664A93421DD0AF
:109480007B681B68644A934218D07B681B68634AF8
:10949000934213D07B681B68614A93420ED07B686D
:1094A0001B68604A934209D07B681B685E4A9342FE
:1094B00004D04FF48D715D48FEF775FF7B689B68A3
:1094C000002B14D07B689B68102B10D07B689B68A6
:1094D000202B0CD07B689B68402B08D07B689B6856
:1094E000602B04D040F21B115048FEF75CFF7B68F4
:1094F0001B69002B0ED07B681B69B3F5807F09D0F8
:109500007B681B69B3F5007F04D04FF48E71474828
:10951000FEF749FF7B681B68B3F1804F0FD07B6873
:10952000DB68002B06D07B68DB68B3F5803F01D297
:10953000012300E0002303F00103DBB206E07B68B7
:10954000DB68002B14BF01230023DBB2002B04D106
:1095500040F21D113548FEF726FF7B689B69002B02
:1095600008D07B689B69802B04D04FF48F712F4803
:10957000FEF719FF7B6893F83D30DBB2002B06D174
:109580007B68002283F83C207868FFF7ADFA7B689F
:10959000022283F83D207B681A687B6804331946F1
:1095A000104601F0EBF97B68012283F848207B68C4
:1095B000012283F83E207B68012283F83F207B68EC
:1095C000012283F840207B68012283F841207B68D8
:1095D000012283F842207B68012283F843207B68C4
:1095E000012283F844207B68012283F845207B68B0
:1095F000012283F846207B68012283F847207B689C
:10960000012283F83D20002318460837BD4680BD5F
:10961000002C014000040040000800400010004001
:10962000004001400044014000480140D89B02082E
:1096300080B584B000AF78607B681B683A4A93427B
:1096400027D07B681B68B3F1804F22D07B681B68F2
:10965000364A93421DD07B681B68354A934218D026
:109660007B681B68334A934213D07B681B68324A7D
:1096700093420ED07B681B68304A934209D07B68C6
:109680001B682F4A934204D04FF4CE712D48FEF749
:109690008AFE7B6893F83D30DBB2012B01D00123B9
:1096A0003DE07B68022283F83D207B681B681E4AF0
:1096B000934213D07B681B68B3F1804F0ED07B6858
:1096C0001B681A4A934209D07B681B68184A934268
:1096D00004D07B681B68184A934215D17B681B68CD
:1096E0009A68194B1340FB60FB68062B15D0FB688A
:1096F000B3F5803F11D07B681B681A687B681B68D4
:1097000042F001021A6008E07B681B681A687B68F7
:109710001B6842F001021A6000E000BF00231846F7
:109720001037BD4680BD00BF002C01400004004042
:10973000000800400010004000400140004401408B
:1097400000480140D89B02080700010080B584B0A2
:1097500000AF78607B681B683E4A934227D07B68E5
:109760001B68B3F1804F22D07B681B683A4A934252
:109770001DD07B681B68394A934218D07B681B68F0
:10978000374A934213D07B681B68364A93420ED007
:109790007B681B68344A934209D07B681B68334A54
:1097A000934204D040F2D7113148FEF7FCFD7B68AC
:1097B00093F83D30DBB2012B01D0012345E07B68FB
:1097C000022283F83D207B681B68DA687B681B688F
:1097D00042F00102DA607B681B681E4A934213D094
:1097E0007B681B68B3F1804F0ED07B681B681A4AF8
:1097F000934209D07B681B68184A934204D07B6867
:109800001B68184A934215D17B681B689A68194BEC
:109810001340FB60FB68062B15D0FB68B3F5803F57
:1098200011D07B681B681A687B681B6842F00102D4
:109830001A6008E07B681B681A687B681B6842F046
:1098400001021A6000E000BF002318461037BD4631
:1098500080BD00BF002C0140000400400008004013
:109860000010004000400140004401400048014019
:10987000D89B02080700010080B582B000AF786075
:109880007B68002B01D10123D2E07B681B686A4A08
:10989000934227D07B681B68B3F1804F22D07B684E
:1098A0001B68664A93421DD07B681B68644A9342DA
:1098B00018D07B681B68634A934213D07B681B688F
:1098C000614A93420ED07B681B68604A934209D07C
:1098D0007B681B685E4A934204D040F239515D4870
:1098E000FEF761FD7B689B68002B14D07B689B684A
:1098F000102B10D07B689B68202B0CD07B689B685A
:10990000402B08D07B689B68602B04D040F23A5112
:109910005048FEF748FD7B681B69002B0ED07B6822
:109920001B69B3F5807F09D07B681B69B3F5007FA5
:1099300004D040F23B514748FEF735FD7B681B6879
:10994000B3F1804F0FD07B68DB68002B06D07B68BB
:10995000DB68B3F5803F01D2012300E0002303F070
:109960000103DBB206E07B68DB68002B14BF012338
:109970000023DBB2002B04D140F23C513548FEF706
:1099800012FD7B689B69002B08D07B689B69802B4C
:1099900004D040F23D512F48FEF705FD7B6893F857
:1099A0003D30DBB2002B06D17B68002283F83C20DF
:1099B0007868FFF7D3F87B68022283F83D207B6844
:1099C0001A687B6804331946104600F0D7FF7B689D
:1099D000012283F848207B68012283F83E207B68BF
:1099E000012283F83F207B68012283F840207B68B6
:1099F000012283F841207B68012283F842207B68A2
:109A0000012283F843207B68012283F844207B688D
:109A1000012283F845207B68012283F846207B6879
:109A2000012283F847207B68012283F83D20002330
:109A300018460837BD4680BD002C01400004004098
:109A40000008004000100040004001400044014078
:109A500000480140D89B020880B584B000AF786010
:109A600039607B681B687F4A934211D13B68002BA9
:109A700061D03B68042B5ED03B68082B5BD03B6811
:109A80000C2B58D03B68102B55D03B68142B52D070
:109A90007B681B68B3F1804F0BD13B68002B4AD029
:109AA0003B68042B47D03B68082B44D03B680C2B09
:109AB00041D07B681B686C4A93420BD13B68002BFA
:109AC00039D03B68042B36D03B68082B33D03B6839
:109AD0000C2B30D07B681B68644A93420BD13B68E7
:109AE000002B28D03B68042B25D03B68082B22D0C4
:109AF0003B680C2B1FD07B681B685D4A934205D1E5
:109B00003B68002B17D03B68042B14D07B681B6884
:109B1000584A934202D13B68002B0CD07B681B68EB
:109B2000554A934202D13B68002B04D040F2C35106
:109B30005248FEF738FC3B68002B09D17B6893F84C
:109B40003E30DBB2012B14BF01230023DBB23CE02B
:109B50003B68042B09D17B6893F83F30DBB2012BC3
:109B600014BF01230023DBB22FE03B68082B09D18F
:109B70007B6893F84030DBB2012B14BF0123002334
:109B8000DBB222E03B680C2B09D17B6893F84130B3
:109B9000DBB2012B14BF01230023DBB215E03B68CD
:109BA000102B09D17B6893F84230DBB2012B14BF34
:109BB00001230023DBB208E07B6893F84330DBB27B
:109BC000012B14BF01230023DBB2002B01D00123A2
:109BD0009BE03B68002B04D17B68022283F83E2087
:109BE00023E03B68042B04D17B68022283F83F20EA
:109BF0001BE03B68082B04D17B68022283F84020DD
:109C000013E03B680C2B04D17B68022283F84120CF
:109C10000BE03B68102B04D17B68022283F84220C2
:109C200003E07B68022283F843207B681B680122E3
:109C30003968184601F0FAFA7B681B68094A9342B2
:109C40000ED07B681B680A4A934209D07B681B6868
:109C5000084A934204D07B681B68074A93420FD19D
:109C600001230EE0002C01400004004000080040E9
:109C7000004001400044014000480140D89B0208D8
:109C80000023002B07D07B681B685A6C7B681B681D
:109C900042F400425A647B681B681E4A934213D008
:109CA0007B681B68B3F1804F0ED07B681B681A4A33
:109CB000934209D07B681B68184A934204D07B68A2
:109CC0001B68174A934215D17B681B689A68154B2D
:109CD0001340FB60FB68062B15D0FB68B3F5803F93
:109CE00011D07B681B681A687B681B6842F0010210
:109CF0001A6008E07B681B681A687B681B6842F082
:109D000001021A6000E000BF002318461037BD466C
:109D100080BD00BF002C014000040040000800404E
:109D2000004001400700010080B584B000AF7860BA
:109D30007B681B68DB68FB607B681B681B69BB601A
:109D4000BB6803F00203002B20D0FB6803F0020382
:109D5000002B1BD07B681B686FF002021A617B68C6
:109D600001221A777B681B689B6903F00303002BB1
:109D700003D0786800F0E4FD05E0786800F0D6FDD7
:109D8000786800F0E7FD7B6800221A77BB6803F073
:109D90000403002B20D0FB6803F00403002B1BD02E
:109DA0007B681B686FF004021A617B6802221A77D5
:109DB0007B681B689B6903F44073002B03D07868B1
:109DC00000F0BEFD05E0786800F0B0FD786800F0B6
:109DD000C1FD7B6800221A77BB6803F00803002BE3
:109DE00020D0FB6803F00803002B1BD07B681B68A6
:109DF0006FF008021A617B6804221A777B681B687F
:109E0000DB6903F00303002B03D0786800F098FDB2
:109E100005E0786800F08AFD786800F09BFD7B68BB
:109E200000221A77BB6803F01003002B20D0FB68D8
:109E300003F01003002B1BD07B681B686FF010022F
:109E40001A617B6808221A777B681B68DB6903F458
:109E50004073002B03D0786800F072FD05E078684D
:109E600000F064FD786800F075FD7B6800221A77C9
:109E7000BB6803F00103002B0CD0FB6803F0010367
:109E8000002B07D07B681B686FF001021A617868AD
:109E9000FEF772FABB6803F08003002B0CD0FB685E
:109EA00003F08003002B07D07B681B686FF08002F3
:109EB0001A61786801F054FBBB6803F48073002BCF
:109EC0000CD0FB6803F08003002B07D07B681B6875
:109ED0006FF480721A61786801F04CFBBB6803F084
:109EE0004003002B0CD0FB6803F04003002B07D08D
:109EF0007B681B686FF040021A61786800F034FDDF
:109F0000BB6803F02003002B0CD0FB6803F0200398
:109F1000002B07D07B681B686FF020021A617868FD
:109F200001F014FB00BF1037BD4680BD80B586B080
:109F300000AFF860B9607A600023FB757B68002B86
:109F400016D07B68042B13D07B68082B10D07B685D
:109F50000C2B0DD07B68102B0AD07B68142B07D0FC
:109F60007B683C2B04D041F2C2018148FEF71BFA0A
:109F7000BB681B68602B1CD0BB681B68702B18D09B
:109F8000BB681B687B4A934213D0BB681B687A4A44
:109F900093420ED0BB681B68784A934209D0BB68D5
:109FA0001B68774A934204D041F2C3017048FEF720
:109FB000FAF9BB689B68002B08D0BB689B68022B32
:109FC00004D041F2C4016A48FEF7EDF9BB681B6991
:109FD000002B08D0BB681B69042B04D041F2C501DB
:109FE0006348FEF7E0F9FB6893F83C30012B01D1A0
:109FF0000223A3E1FB68012283F83C207B68142B39
:10A0000000F2948101A252F823F000BF61A0000881
:10A010002DA300082DA300082DA30008F1A000081F
:10A020002DA300082DA300082DA300089DA1000862
:10A030002DA300082DA300082DA300080FA20008DF
:10A040002DA300082DA300082DA3000883A200085B
:10A050002DA300082DA300082DA30008D7A20008F7
:10A06000FB681B68474A934222D0FB681B68B3F128
:10A07000804F1DD0FB681B68434A934218D0FB6891
:10A080001B68424A934213D0FB681B68404A9342C4
:10A090000ED0FB681B683F4A934209D0FB681B68DF
:10A0A0003D4A934204D041F2CF013148FEF77BF99B
:10A0B000FB681B68B968184600F0EEFCFB681B687B
:10A0C0009A69FB681B6842F008029A61FB681B688A
:10A0D0009A69FB681B6822F004029A61FB681B689E
:10A0E0009969BB681A69FB681B680A439A6120E199
:10A0F000FB681B68234A934218D0FB681B68B3F1C6
:10A10000804F13D0FB681B681F4A93420ED0FB6838
:10A110001B681E4A934209D0FB681B681C4A934285
:10A1200004D04FF487511248FEF73DF9FB681B68D5
:10A13000B968184600F060FDFB681B689A69FB6807
:10A140001B6842F400629A61FB681B689A69FB68AD
:10A150001B6822F480629A61FB681B689969BB687E
:10A160001B691A02FB681B680A439A61E1E000BFA1
:10A17000D89B02084000010050000100600001006F
:10A1800070000100002C0140000400400008004065
:10A19000004001400044014000480140FB681B684A
:10A1A000684A934213D0FB681B68B3F1804F0ED00E
:10A1B000FB681B68644A934209D0FB681B68634ACA
:10A1C000934204D041F2F1016148FEF7ECF8FB68DC
:10A1D0001B68B968184600F0B7FDFB681B68DA69B0
:10A1E000FB681B6842F00802DA61FB681B68DA69E9
:10A1F000FB681B6822F00402DA61FB681B68D969FE
:10A20000BB681A69FB681B680A43DA6191E0FB6866
:10A210001B684C4A934213D0FB681B68B3F1804F14
:10A220000ED0FB681B68484A934209D0FB681B6844
:10A23000464A934204D041F202114548FEF7B3F872
:10A24000FB681B68B968184600F026FEFB681B68AF
:10A25000DA69FB681B6842F40062DA61FB681B681C
:10A26000DA69FB681B6822F48062DA61FB681B68AC
:10A27000D969BB681B691A02FB681B680A43DA616B
:10A2800057E0FB681B682F4A934204D041F2141137
:10A290002F48FEF788F8FB681B68B968184600F07D
:10A2A0006DFEFB681B685A6DFB681B6842F0080274
:10A2B0005A65FB681B685A6DFB681B6822F0040234
:10A2C0005A65FB681B68596DBB681A69FB681B6897
:10A2D0000A435A652DE0FB681B681A4A934204D072
:10A2E00041F227111A48FEF75EF8FB681B68B9684F
:10A2F000184600F0A1FEFB681B685A6DFB681B68DE
:10A3000042F400625A65FB681B685A6DFB681B6863
:10A3100022F480625A65FB681B68596DBB681B6933
:10A320001A02FB681B680A435A6502E00123FB75A9
:10A3300000BFFB68002283F83C20FB7D18461837DD
:10A34000BD4680BD002C01400004004000080040D4
:10A35000D89B020880B584B000AF786039600023D4
:10A36000FB737B6893F83C30012B01D10223CEE2D2
:10A370007B68012283F83C207B68022283F83D2021
:10A380003B681B68B3F5805F29D03B681B68702B66
:10A3900025D03B681B68B3F5005F20D03B681B6885
:10A3A000402B1CD03B681B68502B18D03B681B68A7
:10A3B000602B14D03B681B68002B10D03B681B68D7
:10A3C000102B0CD03B681B68202B08D03B681B6807
:10A3D000302B04D041F272517848FDF7E4FF7B68DE
:10A3E0001B689B68BB60BB6823F4803323F0770352
:10A3F000BB60BB6823F47F43BB607B681B68BA68A3
:10A400009A603B681B68B3F5005F00F0E780B3F526
:10A41000005F00F26F82B3F5805F2DD0B3F5805FEF
:10A4200000F26882702B5DD0702B00F26382602B8B
:10A4300000F08C81602B00F25D82502B00F03581A2
:10A44000502B00F25782402B00F0DC81402B00F2B1
:10A450005182302B00F02782302B00F24B82202BD0
:10A4600000F02182202B00F24582002B00F01B829D
:10A47000102B00F018823DE27B681B68504A934223
:10A4800000F03B827B681B68B3F1804F00F035829F
:10A490007B681B684B4A934200F02F827B681B68E5
:10A4A000494A934200F029827B681B68474A9342DD
:10A4B00000F023827B681B68454A934200F01D82AE
:10A4C0007B681B68434A934200F017827B681B68D5
:10A4D000414A934200F0118241F27E513748FDF724
:10A4E00062FF0AE27B681B68354A934213D07B689F
:10A4F0001B68B3F1804F0ED07B681B68314A9342D2
:10A5000009D07B681B68304A934204D041F28551E0
:10A510002A48FDF748FF3B689B68002B13D03B6837
:10A520009B68B3F5805F0ED03B689B68B3F5005F16
:10A5300009D03B689B68B3F5405F04D041F2885175
:10A540001E48FDF730FF3B685B68B3F5004F14D041
:10A550003B685B68002B10D03B685B68002B0CD01D
:10A560003B685B68022B08D03B685B680A2B04D011
:10A5700041F289511148FDF716FF3B68DB680F2B4C
:10A5800004D941F28A510D48FDF70DFF7B68186828
:10A590003B6899683B685A683B68DB6800F026FEB8
:10A5A0007B681B689B68BB60BB6843F07703BB603C
:10A5B0007B681B68BA689A60A0E100BFD89B02085C
:10A5C000002C014000040040000800400010004042
:10A5D0000040014000440140004801407B681B6886
:10A5E000834A934213D07B681B68B3F1804F0ED02F
:10A5F0007B681B687F4A934209D07B681B687E4A50
:10A60000934204D041F29D517C48FDF7CCFE3B685B
:10A610009B68002B13D03B689B68B3F5805F0ED01E
:10A620003B689B68B3F5005F09D03B689B68B3F556
:10A63000405F04D04FF4AD517048FDF7B4FE3B6865
:10A640005B68B3F5004F14D03B685B68002B10D0FB
:10A650003B685B68002B0CD03B685B68022B08D022
:10A660003B685B680A2B04D041F2A1516348FDF7B7
:10A670009AFE3B68DB680F2B04D941F2A2515F4878
:10A68000FDF791FE7B6818683B6899683B685A68DB
:10A690003B68DB6800F0AAFD7B681B689A687B68F2
:10A6A0001B6842F480429A6028E17B681B68504A2C
:10A6B000934218D07B681B68B3F1804F13D07B683E
:10A6C0001B684C4A93420ED07B681B684A4A9342EF
:10A6D00009D07B681B684A4A934204D041F2B151C9
:10A6E0004648FDF760FE3B685B68B3F5004F14D049
:10A6F0003B685B68002B10D03B685B68002B0CD07C
:10A700003B685B68022B08D03B685B680A2B04D06F
:10A7100041F2B4513948FDF746FE3B68DB680F2B28
:10A7200004D941F2B5513548FDF73DFE7B68186804
:10A730003B6859683B68DB681A4600F0DDFC7B68C3
:10A740001B685021184600F036FDD7E07B681B6877
:10A75000274A934218D07B681B68B3F1804F13D00F
:10A760007B681B68234A93420ED07B681B68224A91
:10A77000934209D07B681B68214A934204D041F27E
:10A78000C1511E48FDF70FFE3B685B68B3F5004FF3
:10A7900014D03B685B68002B10D03B685B68002BD3
:10A7A0000CD03B685B68022B08D03B685B680A2BC7
:10A7B00004D041F2C4511148FDF7F5FD3B68DB6858
:10A7C0000F2B04D941F2C5510C48FDF7ECFD7B6815
:10A7D00018683B6859683B68DB681A4600F0BBFCA8
:10A7E0007B681B686021184600F0E5FC86E000BF2E
:10A7F000002C01400004004000080040D89B0208E3
:10A80000004001407B681B68434A934218D07B6834
:10A810001B68B3F1804F13D07B681B683F4A93429B
:10A820000ED07B681B683E4A934209D07B681B6848
:10A830003C4A934204D041F2D1513B48FDF7B3FD6D
:10A840003B685B68B3F5004F14D03B685B68002B36
:10A8500010D03B685B68002B0CD03B685B68022B18
:10A8600008D03B685B680A2B04D041F2D4512E48D3
:10A87000FDF799FD3B68DB680F2B04D941F2D551F8
:10A880002948FDF790FD7B6818683B6859683B686C
:10A89000DB681A4600F030FC7B681B6840211846D4
:10A8A00000F089FC2AE07B681B681B4A934218D0A1
:10A8B0007B681B68B3F1804F13D07B681B68174A15
:10A8C00093420ED07B681B68154A934209D07B687F
:10A8D0001B68144A934204D041F2E4511248FDF738
:10A8E00062FD7B681A683B681B681946104600F0D9
:10A8F00062FC03E00123FB7300E000BF7B680122E0
:10A9000083F83D207B68002283F83C20FB7B1846BF
:10A910001037BD4680BD00BF002C01400004004040
:10A920000008004000400140D89B020880B483B07A
:10A9300000AF786000BF0C37BD465DF8047B704700
:10A9400080B483B000AF786000BF0C37BD465DF8BF
:10A95000047B704780B483B000AF786000BF0C37D1
:10A96000BD465DF8047B704780B483B000AF78606B
:10A9700000BF0C37BD465DF8047B704780B485B0DE
:10A9800000AF786039607B681B68FB607B683C4A7D
:10A9900093420BD07B68B3F1804F07D07B68394A74
:10A9A000934203D07B68384A934208D1FB6823F076
:10A9B0007003FB603B685B68FA681343FB607B686D
:10A9C0002F4A934217D07B68B3F1804F13D07B6836
:10A9D0002C4A93420FD07B682B4A93420BD07B6862
:10A9E0002A4A934207D07B68294A934203D07B6866
:10A9F000284A934208D1FB6823F44073FB603B680C
:10AA0000DB68FA681343FB60FB6823F080023B6855
:10AA10005B691343FB607B68FA681A603B689A685D
:10AA20007B68DA623B681A687B689A627B68144AC2
:10AA300093420BD07B68154A934207D07B68144A37
:10AA4000934203D07B68134A934203D13B681A694F
:10AA50007B681A637B6801225A617B681B6903F07B
:10AA60000103012B05D17B681B6923F001027B6880
:10AA70001A6100BF1437BD465DF8047B704700BF04
:10AA8000002C01400004004000080040004001404C
:10AA9000004401400048014080B586B000AF7860B6
:10AAA00039607B681B6A7B617B681B6A23F001024B
:10AAB0007B681A627B685B683B617B689B69FB60B3
:10AAC000FB6823F4803323F07003FB60FB6823F002
:10AAD0000303FB603B681B68FA681343FB607B69F8
:10AAE00023F002037B613B689B687A6913437B61B7
:10AAF0007B683C4A93420BD07B683B4A934207D029
:10AB00007B683A4A934203D07B68394A934219D111
:10AB10003B68DB68002B08D03B68DB68082B04D05F
:10AB200041F692313348FDF73EFC7B6923F0080380
:10AB30007B613B68DB687A6913437B617B6923F047
:10AB400004037B617B68274A93420BD07B68264ACB
:10AB5000934207D07B68254A934203D07B68244AFE
:10AB600093422DD13B689B69B3F5007F08D03B68C9
:10AB70009B69002B04D041F69F311E48FDF713FC62
:10AB80003B685B69B3F5807F08D03B685B69002B4D
:10AB900004D04FF4DD511748FDF705FC3B6923F461
:10ABA00080733B613B6923F400733B613B685B69E5
:10ABB0003A6913433B613B689B693A6913433B61C4
:10ABC0007B683A695A607B68FA689A613B685A68A0
:10ABD0007B685A637B687A691A6200BF1837BD4682
:10ABE00080BD00BF002C01400040014000440140F6
:10ABF00000480140D89B020880B586B000AF78605D
:10AC000039607B681B6A7B617B681B6A23F01002DA
:10AC10007B681A627B685B683B617B689B69FB6051
:10AC2000FB6823F0807323F4E043FB60FB6823F4AC
:10AC30004073FB603B681B681B02FA681343FB60B0
:10AC40007B6923F020037B613B689B681B017A6969
:10AC500013437B617B68374A93421AD13B68DB68B8
:10AC6000002B08D03B68DB68082B04D041F6DE31AE
:10AC70003148FDF798FB7B6923F080037B613B68DB
:10AC8000DB681B017A6913437B617B6923F0400316
:10AC90007B617B68274A93420BD07B68274A9342AB
:10ACA00007D07B68264A934203D07B68254A9342AB
:10ACB0002FD13B689B69B3F5007F08D03B689B6947
:10ACC000002B04D041F6EB311B48FDF76CFB3B68D1
:10ACD0005B69B3F5807F08D03B685B69002B04D0CB
:10ACE00041F6EC311448FDF75EFB3B6923F48063C9
:10ACF0003B613B6923F400633B613B685B699B00FC
:10AD00003A6913433B613B689B699B003A69134373
:10AD10003B617B683A695A607B68FA689A613B6874
:10AD20005A687B689A637B687A691A6200BF183731
:10AD3000BD4680BD002C0140D89B02080040014068
:10AD4000004401400048014080B586B000AF786003
:10AD500039607B681B6A7B617B681B6A23F48072A5
:10AD60007B681A627B685B683B617B68DB69FB60C0
:10AD7000FB6823F4803323F07003FB60FB6823F04F
:10AD80000303FB603B681B68FA681343FB607B6945
:10AD900023F400737B613B689B681B027A69134351
:10ADA0007B617B68374A93421AD13B68DB68002B92
:10ADB00008D03B68DB68082B04D041F62B413248B1
:10ADC000FDF7F1FA7B6923F400637B613B68DB6884
:10ADD0001B027A6913437B617B6923F480637B6187
:10ADE0007B68284A93420BD07B68284A934207D05D
:10ADF0007B68274A934203D07B68264A93422FD12F
:10AE00003B689B69B3F5007F08D03B689B69002BCA
:10AE100004D041F639411C48FDF7C5FA3B685B692F
:10AE2000B3F5807F08D03B685B69002B04D041F606
:10AE30003A411548FDF7B7FA3B6923F480533B616B
:10AE40003B6923F400533B613B685B691B013A6932
:10AE500013433B613B689B691B013A6913433B61A8
:10AE60007B683A695A607B68FA68DA613B685A68BD
:10AE70007B68DA637B687A691A6200BF1837BD465F
:10AE800080BD00BF002C0140D89B0208004001405B
:10AE9000004401400048014080B586B000AF7860B2
:10AEA00039607B681B6A3B617B681B6A23F48052B4
:10AEB0007B681A627B685B687B617B68DB69FB602F
:10AEC000FB6823F0807323F4E043FB60FB6823F40A
:10AED0004073FB603B681B681B02FA681343FB600E
:10AEE0003B6923F400533B613B689B681B033A6951
:10AEF00013433B617B681C4A93420BD07B681B4A1F
:10AF0000934207D07B681A4A934203D07B68194A60
:10AF1000934217D13B685B69B3F5807F08D03B68EB
:10AF20005B69002B04D041F67B411348FDF73BFAE7
:10AF30007B6923F480437B613B685B699B017A6991
:10AF400013437B617B687A695A607B68FA68DA61CF
:10AF50003B685A687B681A647B683A691A6200BF6A
:10AF60001837BD4680BD00BF002C014000400140A5
:10AF70000044014000480140D89B020880B487B0DB
:10AF800000AF786039607B681B6A3B617B681B6A35
:10AF900023F480327B681A627B685B687B617B6824
:10AFA0005B6DFB60FB6823F4803323F07003FB6070
:10AFB0003B681B68FA681343FB603B6923F400336A
:10AFC0003B613B689B681B043A6913433B617B68A8
:10AFD000154A93420BD07B68144A934207D07B6892
:10AFE000134A934203D07B68124A934209D17B698A
:10AFF00023F480337B613B685B691B027A691343EE
:10B000007B617B687A695A607B68FA685A653B683D
:10B010005A687B689A657B683A691A6200BF1C3778
:10B02000BD465DF8047B7047002C014000400140A4
:10B03000004401400048014080B487B000AF786010
:10B0400039607B681B6A3B617B681B6A23F4801252
:10B050007B681A627B685B687B617B685B6DFB6009
:10B06000FB6823F0807323F4E043FB603B681B68BC
:10B070001B02FA681343FB603B6923F400133B6136
:10B080003B689B681B053A6913433B617B68164A22
:10B0900093420BD07B68154A934207D07B68144AD1
:10B0A000934203D07B68134A934209D17B6923F40E
:10B0B00080237B613B685B699B027A6913437B61F8
:10B0C0007B687A695A607B68FA685A653B685A6897
:10B0D0007B68DA657B683A691A6200BF1C37BD4637
:10B0E0005DF8047B704700BF002C01400040014028
:10B0F000004401400048014080B487B000AFF860D0
:10B10000B9607A60FB681B6A7B61FB681B6A23F08D
:10B110000102FB681A62FB689B693B613B6923F093
:10B12000F0033B617B681B013A6913433B617B6918
:10B1300023F00A037B617A69BB6813437B61FB6878
:10B140003A699A61FB687A691A6200BF1C37BD468A
:10B150005DF8047B704780B487B000AFF860B960D9
:10B160007A60FB681B6A7B61FB681B6A23F0100234
:10B17000FB681A62FB689B693B613B6923F470437F
:10B180003B617B681B033A6913433B617B6923F096
:10B19000A0037B61BB681B017A6913437B61FB6879
:10B1A0003A699A61FB687A691A6200BF1C37BD462A
:10B1B0005DF8047B704780B485B000AF786039607B
:10B1C0007B689B68FB60FB6823F07003FB603A6858
:10B1D000FB68134343F00703FB607B68FA689A60DF
:10B1E00000BF1437BD465DF8047B704780B487B05C
:10B1F00000AFF860B9607A603B60FB689B687B6178
:10B200007B6923F47F437B613B681A027B681A43A6
:10B21000BB6813437A6913437B61FB687A699A6060
:10B2200000BF1C37BD465DF8047B704780B586B013
:10B2300000AFF860B9607A60FB682B4A93421CD07B
:10B24000FB68B3F1804F18D0FB68284A934214D0B2
:10B25000FB68274A934210D0FB68264A93420CD0E1
:10B26000FB68254A934208D0FB68244A934204D0E5
:10B2700041F6DA612248FDF796F8BB68002B16D03C
:10B28000BB68042B13D0BB68082B10D0BB680C2BF9
:10B290000DD0BB68102B0AD0BB68142B07D0BB683D
:10B2A0003C2B04D041F6DB611548FDF77CF8BB6808
:10B2B00003F01F03012202FA03F37B61FB681A6AA1
:10B2C0007B69DB431A40FB681A62FB681A6ABB6839
:10B2D00003F01F03796801FA03F31A43FB681A624B
:10B2E00000BF1837BD4680BD002C0140000400405F
:10B2F0000008004000400140004401400048014077
:10B30000D89B020880B584B000AF786039607B6854
:10B310001B68884A93421DD07B681B68B3F1804F3D
:10B3200018D07B681B68844A934213D07B681B68E3
:10B33000824A93420ED07B681B68814A934209D0AF
:10B340007B681B687F4A934204D040F2AC717E4810
:10B35000FDF729F83B681B68002B20D03B681B6871
:10B36000102B1CD03B681B68202B18D03B681B6837
:10B37000302B14D03B681B68402B10D03B681B68F7
:10B38000502B0CD03B681B68602B08D03B681B68B7
:10B39000702B04D040F2AD716B48FDF704F83B68A8
:10B3A0009B68802B08D03B689B68002B04D040F240
:10B3B000AE716548FCF7F7FF7B6893F83C30012BD2
:10B3C00001D10223B2E07B68012283F83C207B6834
:10B3D000022283F83D207B681B685B68FB607B680A
:10B3E0001B689B68BB607B681B68524A934261D1B3
:10B3F0003B685B68002B54D03B685B68B3F5801FEB
:10B400004FD03B685B68B3F5001F4AD03B685B6870
:10B41000B3F5401F45D03B685B68B3F5800F40D063
:10B420003B685B68B3F5A00F3BD03B685B68B3F546
:10B43000C00F36D03B685B68B3F5C00F31D03B68B6
:10B440005B68B3F5E00F2CD03B685B68B3F5000F89
:10B4500027D03B685B68B3F5100F22D03B685B6870
:10B46000B3F5200F1DD03B685B68B3F5300F18D0E3
:10B470003B685B68B3F5400F13D03B685B68B3F57E
:10B48000500F0ED03B685B68B3F5600F09D03B6886
:10B490005B68B3F5700F04D040F2C1712A48FCF725
:10B4A00082FFFB6823F47003FB603B685B68FA680B
:10B4B0001343FB60FB6823F07003FB603B681B6871
:10B4C000FA681343FB607B681B68FA685A607B6804
:10B4D0001B68184A934213D07B681B68B3F1804FF6
:10B4E0000ED07B681B68144A934209D07B681B68A6
:10B4F000124A934204D07B681B68124A93420CD1D3
:10B50000BB6823F08003BB603B689B68BA68134349
:10B51000BB607B681B68BA689A607B68012283F80D
:10B520003D207B68002283F83C200023184610371A
:10B53000BD4680BD002C01400004004000080040D2
:10B540000010004000400140109C020880B483B00D
:10B5500000AF786000BF0C37BD465DF8047B7047D4
:10B5600080B483B000AF786000BF0C37BD465DF893
:10B57000047B704780B483B000AF786000BF0C37A5
:10B58000BD465DF8047B704780B483B000AF78603F
:10B5900000BF0C37BD465DF8047B704780B483B0B4
:10B5A00000AF786000BF0C37BD465DF8047B704784
:10B5B00080B59AB000AF7860002387F86730002329
:10B5C0003B660023BB607B68002B01D1012397E21F
:10B5D0007B681B68B3F1A04F08D07B681B688E4A5C
:10B5E000934203D0F2218D48FCF7DDFE7B685B6857
:10B5F000002B12D07B685B68B3F5803F0DD07B6871
:10B600005B68B3F5003F08D07B685B68B3F5403FEB
:10B6100003D0F3218148FCF7C6FE7B689B68002BB2
:10B620000FD07B689B68082B0BD07B689B68102B26
:10B6300007D07B689B68182B03D0F4217748FCF770
:10B64000B2FE7B68DB68002B07D07B68DB68202BB1
:10B6500003D0F5217148FCF7A6FE7B681B69002B1F
:10B6600007D07B681B69012B03D0F6216B48FCF7E0
:10B670009AFE7B685B7E002B07D07B685B7E012B8C
:10B6800003D0F7216548FCF78EFE7B68DB6A002B50
:10B6900012D07B68DB6AB3F5806F0DD07B68DB6A04
:10B6A000B3F5006F08D07B68DB6AB3F5406F03D059
:10B6B000F8215A48FCF777FE7B689B6A002B45D03F
:10B6C0007B689B6A402B41D07B689B6A802B3DD076
:10B6D0007B689B6AC02B39D07B689B6AB3F5807FFF
:10B6E00034D07B689B6AB3F5A07F2FD07B689B6AC0
:10B6F000B3F5C07F2AD07B689B6AB3F5107F25D055
:10B700007B689B6AB3F5207F20D07B689B6AB3F58A
:10B71000307F1BD07B689B6AB3F5407F16D07B6877
:10B720009B6AB3F5507F11D07B689B6AB3F5607F4D
:10B730000CD07B689B6AB3F5707F07D07B689B6AEF
:10B74000012B03D0F9213548FCF72DFE7B6893F8D7
:10B750003030002B08D07B6893F83030012B03D0B9
:10B76000FA212E48FCF71FFE7B685B69042B07D08B
:10B770007B685B69082B03D0FB212848FCF713FE8C
:10B780007B685B6B012B07D07B685B6B002B03D066
:10B79000FC212248FCF707FE7B681B7E002B07D0AC
:10B7A0007B681B7E012B03D0FD211C48FCF7FBFDB1
:10B7B0007B681B69002B33D07B68DB69002B03D0CF
:10B7C0007B68DB69102B04D940F201111348FCF7A8
:10B7D000EAFD7B6893F82030002B09D07B6893F852
:10B7E0002030012B04D04FF481710C48FCF7DBFDB5
:10B7F0007B6893F82030002B12D07B685B6A002BAB
:10B8000003D07B685B6A082B0AD940F20511034814
:10B81000FCF7C9FD04E000BF00010050489C02088D
:10B820007B681B6C03F01003002B76D17B681B6CCC
:10B83000002B52D17B6800225A647B680022DA64B4
:10B840007B6800229A647B68002283F83C20786839
:10B85000FCF72CFF7B681B689B6803F08053002B70
:10B860003BD1786801F05CFC034687F867307B6861
:10B870001B6C03F01003002B2FD197F86730002BBF
:10B880002BD17B681B6C23F4885323F0020343F015
:10B8900002027B681A647B681B689A687B681B6875
:10B8A00022F040529A607B681B689A687B681B682C
:10B8B00042F080529A60944B1B68944AA2FB032387
:10B8C0009A0C13469B0013445B00BB6002E0BB680C
:10B8D000013BBB60BB68002BF9D17B681B689B6890
:10B8E00003F08053002B07D07B681B689B6803F034
:10B8F0000053B3F1005F10D17B681B6C23F012037F
:10B9000043F010027B681A647B685B6C43F00102B1
:10B910007B685A64012387F867307B681B6C03F0EF
:10B920001003002B40F0DF8097F86730002B40F0C9
:10B93000DA807B681B689B6803F00403002B40F0EF
:10B94000D2807B681B6C23F4817343F002027B6816
:10B950001A646F4BFB657B681B68B3F1A04F02D183
:10B960006C4BFB6002E04FF0A043FB607B681B6800
:10B970009B6803F00303012B08D17B681B681B68DD
:10B9800003F00103012B01D1012300E00023002B70
:10B990001CD1FB68002B10D0FB689B6803F00303ED
:10B9A000012B07D1FB681B6803F00103012B01D1B8
:10B9B000012300E00023002B08D1FB6D9B6823F4DA
:10B9C00040327B685B681A43FB6D9A607B685B7EE4
:10B9D0005B037A68526B012A02D04FF4805200E078
:10B9E00000221A437B68DB681A437B689B68134319
:10B9F0003A6E13433B667B6893F82030012B1BD1D2
:10BA00007B685B7E002B09D17B685B6A013B5A0433
:10BA10003B6E134343F480333B660DE07B681B6C45
:10BA200023F0220343F020027B681A647B685B6C7E
:10BA300043F001027B685A647B689B6A012B07D044
:10BA40007B689A6A7B68DB6A13433A6E13433B66F2
:10BA50007B681B689B6803F00C03002B14D17B6888
:10BA60001B68DB687A68126823F4804323F00203C2
:10BA7000D3607B681B7E9A037B6893F830305B0051
:10BA800013433A6E13433B667B681B68DA68224BAC
:10BA900013407A681268396E0B43D3607B681B6968
:10BAA000012B0CD17B681B681B6B23F00F017B689B
:10BAB000DB695A1E7B681B680A431A6307E07B68D0
:10BAC0001B681A6B7B681B6822F00F021A637B6885
:10BAD00000225A647B681B6C23F0030343F00102CD
:10BAE0007B681A640AE07B681B6C23F0120343F046
:10BAF00010027B681A64012387F8673097F8673073
:10BB000018466837BD4680BD0800002083DE1B4311
:10BB1000000300500001005007C0F0FF80B584B062
:10BB200000AF78600023FB737B681B68B3F1A04F04
:10BB300009D07B681B681B4A934204D040F2A6518F
:10BB40001948FCF730FC7B6893F83C30012B01D19D
:10BB5000022323E07B68012283F83C206C21786873
:10BB600001F044FB0346FB73FB7B002B11D178688B
:10BB700001F0D6FA0346FB73FB7B002B09D17B68EF
:10BB80001B6C23F4885323F0010343F001027B680C
:10BB90001A647B68002283F83C20FB7B1846103730
:10BBA000BD4680BD00010050489C020880B586B0AB
:10BBB00000AF7860396000233B617B681B68B3F19C
:10BBC000A04F09D07B681B68654A934204D040F2BD
:10BBD00012616448FCF7E7FB7B685B69082B02D1C4
:10BBE00008237B612EE0604BFB60FB689B6803F0E1
:10BBF0001F03002B12D17B681B68DB6803F0010375
:10BC0000012B1DD17B681B6C43F020027B681A64FA
:10BC10007B68002283F83C2001239DE0FB689B6841
:10BC200003F44043002B0BD07B681B6C43F02002D5
:10BC30007B681A647B68002283F83C2001238BE038
:10BC40000C237B61484B9B6803F01F03002B04D03F
:10BC50007B681B68B3F1A04F04D17B681B68DB686D
:10BC60003B6103E04FF0A043DB683B6101F0BEFBAA
:10BC7000B86021E03B68B3F1FF3F1DD03B68002B6B
:10BC800007D001F0B3FB0246BB68D31A3A689A4268
:10BC900012D27B681B681A687B691340002B0BD19A
:10BCA0007B681B6C43F004027B681A647B6800228B
:10BCB00083F83C2003234FE07B681B681A687B698C
:10BCC0001340002BD6D07B681B6C43F400727B685A
:10BCD0001A647B681B68DB6803F44063002B31D176
:10BCE0003B6903F40053002B2CD17B681B681B6855
:10BCF00003F00803082B25D17B681B689B6803F0C1
:10BD00000403002B12D17B681B6C23F480727B68C8
:10BD10001A647B681B6C03F48053002B12D17B6880
:10BD20001B6C43F001027B681A640BE07B681B6CA0
:10BD300043F020027B681A647B685B6C43F001026D
:10BD40007B685A643B6903F48043002B03D17B6812
:10BD50001B687A691A60002318461837BD4680BDF3
:10BD600000010050489C02080003005080B584B0D8
:10BD700000AF78600023FB737B681B68B3F1A04FB2
:10BD800009D07B681B686E4A934204D040F60401D8
:10BD90006C48FCF708FB7B681B689B6803F0040396
:10BDA000002B40F0C6807B6893F83C30012B01D11A
:10BDB0000223C1E07B68012283F83C20786801F00F
:10BDC0004BF90346FB73FB7B002B40F0AD807B6897
:10BDD0001B6C23F4706323F0010343F480727B68CF
:10BDE0001A64594B9B6803F01F03002B04D07B6837
:10BDF0001B68B3F1A04F15D17B681B6C23F4801234
:10BE00007B681A647B681B68DB6803F00073002B97
:10BE100027D07B681B6C23F4405343F480527B682B
:10BE20001A641EE07B681B6C43F480127B681A6402
:10BE30007B681B68B3F1A04F04D07B681B68404A45
:10BE400093420ED14FF0A043DB6803F00073002B48
:10BE500007D07B681B6C23F4405343F480527B680B
:10BE60001A647B681B6C03F48053B3F5805F06D1C2
:10BE70007B685B6C23F006027B685A6402E07B6897
:10BE800000225A647B68002283F83C207B681B6890
:10BE90001C221A607B685B69082B10D17B681B68C9
:10BEA0005A687B681B6822F004025A607B681B6832
:10BEB0005A687B681B6842F008025A6008E07B6899
:10BEC0001B685A687B681B6842F00C025A6000BF0E
:10BED0007B685B6B012B07D17B681B685A687B68AA
:10BEE0001B6822F010025A60174B9B6803F01F0377
:10BEF000002B10D0144B9B6803F01F03052B0AD0B6
:10BF0000114B9B6803F01F03092B04D07B681B684F
:10BF1000B3F1A04F0FD17B681B689A687B681B68E0
:10BF200042F004029A6006E07B68002283F83C201D
:10BF300001E00223FB73FB7B18461037BD4680BD32
:10BF400000010050489C02080003005080B582B0F8
:10BF500000AF78607B681B68B3F1A04F09D07B68A5
:10BF60001B68074A934204D040F601310548FCF7AC
:10BF70001AFA7B681B681B6C18460837BD4680BDE3
:10BF800000010050489C020880B588B000AF78607E
:10BF90000023FB610023BB6100237B617B681B687E
:10BFA0001B683B617B681B685B68FB607B681B6888
:10BFB000B3F1A04F09D07B681B688E4A934204D02E
:10BFC00040F642318C48FCF7EEF97B685B7E002B33
:10BFD00008D07B685B7E012B04D040F64331864855
:10BFE000FCF7E1F97B685B69042B08D07B685B692F
:10BFF000082B04D040F644317F48FCF7D4F93B6964
:10C0000003F00403002B04D0FB6803F00403002BAF
:10C0100009D13B6903F00803002B76D0FB6803F0DD
:10C020000803002B71D07B681B6C03F01003002BFE
:10C0300005D17B681B6C43F400727B681A646F4BFC
:10C040009B6803F01F03002B10D06C4B9B6803F020
:10C050001F03052B0AD0694B9B6803F01F03092BB4
:10C0600004D07B681B68B3F1A04F04D17B681B68C8
:10C07000DB68BB6103E04FF0A043DB68BB617B681A
:10C080001B68DB6803F44063002B37D1BB6903F402
:10C090000053002B32D13B6903F00803002B2DD055
:10C0A0007B681B689B6803F00403002B1AD17B6834
:10C0B0001B685A687B681B6822F00C025A607B6818
:10C0C0001B6C23F480727B681A647B681B6C03F41E
:10C0D0008053002B12D17B681B6C43F001027B68FC
:10C0E0001A640BE07B681B6C43F010027B681A64D7
:10C0F0007B685B6C43F001027B685A64786818F0D7
:10C10000BBFB7B681B680C221A603B6903F02003B1
:10C11000002B04D0FB6803F02003002B0BD13B69FC
:10C1200003F04003002B00F0A980FB6803F04003FC
:10C13000002B00F0A3807B681B6C43F400527B68EB
:10C140001A642E4B9B6803F01F03002B10D02B4B5F
:10C150009B6803F01F03052B0AD0284B9B6803F054
:10C160001F03092B04D07B681B68B3F1A04F04D1D7
:10C170007B681B68DB68BB6103E04FF0A043DB68B2
:10C18000BB617B681B68DB6C03F0C003002B6ED1C6
:10C19000BB6903F00073002B0BD07B681B68DB6866
:10C1A00003F44063002B62D1BB6903F40053002BFE
:10C1B0005DD13B6903F04003002B58D00F4B9B68C7
:10C1C00003F01F03002B10D00C4B9B6803F01F03E0
:10C1D000062B0AD0094B9B6803F01F03072B04D0E2
:10C1E0007B681B68B3F1A04F0AD17B681B68DB68D2
:10C1F0007B6109E000010050489C020800030050E8
:10C200004FF0A043DB687B617B6903F40013002BD4
:10C210002DD17B681B689B6803F00803002B1AD1A3
:10C220007B681B685A687B681B6822F060025A6052
:10C230007B681B6C23F480527B681A647B681B6CE0
:10C2400003F48073002B12D17B681B6C43F0010256
:10C250007B681A640BE07B681B6C43F010027B6800
:10C260001A647B685B6C43F001027B685A647868EF
:10C2700000F040F97B681B6860221A603B6903F09C
:10C280008003002B11D0FB6803F08003002B0CD03F
:10C290007B681B6C43F480327B681A647868FFF714
:10C2A00073F97B681B6880221A603B6903F4807312
:10C2B000002B12D0FB6803F48073002B0DD07B6839
:10C2C0001B6C43F400327B681A64786800F026F92E
:10C2D0007B681B684FF480721A603B6903F400733B
:10C2E000002B12D0FB6803F40073002B0DD07B6889
:10C2F0001B6C43F480227B681A64786800F018F99C
:10C300007B681B684FF400721A603B6903F01003EE
:10C31000002B3BD0FB6803F01003002B36D07B686A
:10C320005B6B012B02D10123FB6119E0284BBB6041
:10C33000BB689B6803F01F03002B09D17B681B6857
:10C34000DB6803F00103012B0AD10123FB6107E045
:10C35000BB689B6803F44043002B01D00123FB61C1
:10C36000FB69012B0ED17B681B6C43F480627B68F8
:10C370001A647B685B6C43F002027B685A647868DD
:10C38000FFF70CF97B681B6810221A603B6903F405
:10C390008063002B18D0FB6803F48063002B13D05C
:10C3A0007B681B6C43F480427B681A647B685B6C1F
:10C3B00043F008027B685A647B681B684FF4806214
:10C3C0001A60786800F0A0F800BF2037BD4680BD35
:10C3D0000003005080B584B000AF7860396000235E
:10C3E000FB737B681B68B3F1A04F09D07B681B68A7
:10C3F0003E4A934204D040F60C513D48FBF7D3FF30
:10C400003B68002B07D03B68012B04D040F60D5150
:10C410003748FBF7C8FF7B6893F83C30012B01D10C
:10C4200002235FE07B68012283F83C20786800F0FB
:10C4300077FE0346FB73FB7B002B4ED17B6801220A
:10C440001A647B681B689A687B681B6822F08042CC
:10C450009A603B68012B07D17B681B689A687B68F0
:10C460001B6842F080429A607B681B689A687B6810
:10C470001B6842F000429A6000F0B8FFB8601CE010
:10C4800000F0B4FF0246BB68D31A0A2B15D97B68AB
:10C490001B689B6803F00043B3F1004F0DD17B682C
:10C4A0001B6C23F0120343F010027B681A647B6854
:10C4B000002283F83C20012314E07B681B689B6802
:10C4C00003F00043B3F1004FDAD07B681B6C23F01C
:10C4D000030343F001027B681A647B68002283F83F
:10C4E0003C20FB7B18461037BD4680BD0001005044
:10C4F000489C020880B483B000AF786000BF0C375E
:10C50000BD465DF8047B704780B483B000AF7860AF
:10C5100000BF0C37BD465DF8047B704780B483B024
:10C5200000AF786000BF0C37BD465DF8047B7047F4
:10C5300080B483B000AF786000BF0C37BD465DF8B3
:10C54000047B704780B59AB000AF786039600023F3
:10C5500087F867300023BB607B681B68B3F1A04F8E
:10C5600009D07B681B68664A934204D041F2B851F7
:10C570006448FBF718FF3B685B68012B40D03B68C1
:10C580005B68022B3CD03B685B68032B38D03B6870
:10C590005B68042B34D03B685B68052B30D03B686C
:10C5A0005B68062B2CD03B685B68072B28D03B6868
:10C5B0005B68082B24D03B685B68092B20D03B6864
:10C5C0005B680A2B1CD03B685B680B2B18D03B6860
:10C5D0005B680C2B14D03B685B680D2B10D03B685C
:10C5E0005B680E2B0CD03B685B680F2B08D03B6858
:10C5F0005B68102B04D041F2B9514248FBF7D3FEDF
:10C600003B689B68002B20D03B689B68012B1CD0AB
:10C610003B689B68022B18D03B689B68032B14D0A7
:10C620003B689B68042B10D03B689B68052B0CD0A3
:10C630003B689B68062B08D03B689B68072B04D09F
:10C6400041F2BA512F48FBF7AEFE3B68DB68002B86
:10C6500008D03B68DB68012B04D041F2BB5129486C
:10C66000FBF7A1FE3B681B69002B14D03B681B69DC
:10C67000012B10D03B681B69022B0CD03B681B6957
:10C68000032B08D03B681B69042B04D041F2BC513A
:10C690001C48FBF788FE7B681B68DB6803F0180307
:10C6A000002B04D13B685B69B3F5805F2CD37B68BA
:10C6B0001B68DB6803F01803082B04D13B685B6937
:10C6C000B3F5806F20D37B681B68DB6803F0180329
:10C6D000102B03D13B685B69FF2B15D97B681B6866
:10C6E000DB6803F01803182B03D13B685B693F2B11
:10C6F0000AD941F2BD510348FBF755FE04E000BFE3
:10C7000000010050489C02083B68DB68012B63D0A5
:10C710003B681B68012B00F09C803B681B68022B68
:10C7200000F097803B681B68032B00F092803B6809
:10C730001B68042B00F08D803B681B68052B00F004
:10C7400088803B681B68062B00F083803B681B6871
:10C75000072B7ED03B681B68082B7AD03B681B6890
:10C76000092B76D03B681B680A2B72D03B681B688C
:10C770000B2B6ED03B681B680C2B6AD03B681B6888
:10C780000D2B66D03B681B680E2B62D03B681B6884
:10C790000F2B5ED03B681B68102B5AD03B681B6880
:10C7A000112B56D03B681B68122B52D03B681B687C
:10C7B0000F2B4ED03B681B68112B4AD03B681B687F
:10C7C000112B46D03B681B68112B42D041F2C5515A
:10C7D0009B48FBF7E8FD3CE03B681B68012B38D029
:10C7E0003B681B68022B34D03B681B68032B30D09E
:10C7F0003B681B68042B2CD03B681B68052B28D09A
:10C800003B681B68062B24D03B681B68072B20D095
:10C810003B681B68082B1CD03B681B68092B18D091
:10C820003B681B680A2B14D03B681B680B2B10D08D
:10C830003B681B680C2B0CD03B681B680D2B08D089
:10C840003B681B680E2B04D041F2C9517C48FBF7B2
:10C85000AAFD7B6893F83C30012B01D10223A5E2AD
:10C860007B68012283F83C207B681B689B6803F08F
:10C870000403002B40F089823B685B68042B1CD8C2
:10C880007B681B68196B3B685A6813465B0013444E
:10C890005B001A461F239340DB4319403B6818682E
:10C8A0003B685A6813465B0013445B0000FA03F2CE
:10C8B0007B681B680A431A6363E03B685B68092B6B
:10C8C0001ED87B681B68596B3B685A6813465B002F
:10C8D00013445B001E3B1F2202FA03F3DB431940A3
:10C8E0003B6818683B685A6813465B0013445B005A
:10C8F0001E3B00FA03F27B681B680A435A6340E060
:10C900003B685B680E2B1ED87B681B68996B3B6885
:10C910005A6813465B0013445B003C3B1F2202FA3B
:10C9200003F3DB4319403B6818683B685A681346B9
:10C930005B0013445B003C3B00FA03F27B681B681E
:10C940000A439A631DE07B681B68D96B3B685A6891
:10C9500013465B0013445B005A3B1F2202FA03F3A9
:10C96000DB4319403B6818683B685A6813465B0014
:10C9700013445B005A3B00FA03F27B681B680A43CE
:10C98000DA637B681B689B6803F00C03002B40F0A4
:10C99000E6803B681B68092B1CD97B681B6899697A
:10C9A0003B681A6813465B0013441E3B072202FAD9
:10C9B00003F3DB4319403B6898683B681A681346E9
:10C9C0005B0013441E3B00FA03F27B681B680A43BA
:10C9D0009A6119E07B681B6859693B681A681346BD
:10C9E0005B001344072202FA03F3DB4319403B6860
:10C9F00098683B681A6813465B00134400FA03F218
:10CA00007B681B680A435A613B685A697B681B68EC
:10CA1000DB68DB0803F003035B0002FA03F33B6609
:10CA20003B681B69013B032B50D801A252F823F04D
:10CA300045CA000867CA000889CA0008ABCA0008CE
:10CA4000489C02087B681B681A6E944B13403A6836
:10CA5000126891063A6E0A431A437B681B6842F0DB
:10CA600000421A667EE07B681B685A6E8B4B13404F
:10CA70003A68126891063A6E0A431A437B681B684B
:10CA800042F000425A666DE07B681B689A6E834BE9
:10CA900013403A68126891063A6E0A431A437B685B
:10CAA0001B6842F000429A665CE07B681B68DA6EA5
:10CAB0007A4B13403A68126891063A6E0A431A4359
:10CAC0007B681B6842F00042DA664BE07B681B68BB
:10CAD0001B6E03F0F8423B681B689B069A4207D125
:10CAE0007B681B681A6E7B681B6822F000421A661E
:10CAF0007B681B685B6E03F0F8423B681B689B0613
:10CB00009A4207D17B681B685A6E7B681B6822F0CB
:10CB100000425A667B681B689B6E03F0F8423B68D4
:10CB20001B689B069A4207D17B681B689A6E7B68DC
:10CB30001B6822F000429A667B681B68DB6E03F07C
:10CB4000F8423B681B689B069A420AD17B681B68C7
:10CB5000DA6E7B681B6822F00042DA6601E000BFF3
:10CB600000E000BF7B681B689B6803F00303012B98
:10CB700008D17B681B681B6803F00103012B01D1FE
:10CB8000012300E00023002B40F00A813B68DB68B2
:10CB9000012B0FD07B681B68D3F8B0103B681B6873
:10CBA000012202FA03F3DA437B681B680A40C3F8E8
:10CBB000B02049E07B681B68D3F8B0103B681B6865
:10CBC00001229A407B681B680A43C3F8B0203B6887
:10CBD0001B68092B1CD97B681B6899693B681A681C
:10CBE00013465B0013441B3B072202FA03F3DB43AB
:10CBF00019403B6898683B681A6813465B00134409
:10CC00001B3B00FA03F27B681B680A439A611BE036
:10CC10007B681B6859693B681B685A1C13465B009C
:10CC20001344072202FA03F3DB4319403B68986878
:10CC30003B681B685A1C13465B00134400FA03F25E
:10CC40007B681B680A435A61154BFB653B681B6890
:10CC5000102B05D1FB6D9B6803F40003002B15D04E
:10CC60003B681B68112B05D1FB6D9B6803F080733B
:10CC7000002B0BD03B681B68122B40F09180FB6DA2
:10CC80009B6803F48003002B40F08A807B681B685C
:10CC9000B3F1A04F08D1034BFB6008E000F0FF8325
:10CCA00000030050000100504FF0A043FB607B6880
:10CCB0001B689B6803F00303012B08D17B681B688A
:10CCC0001B6803F00103012B01D1012300E00023C5
:10CCD000002B50D1FB68002B10D0FB689B6803F041
:10CCE0000303012B07D1FB681B6803F00103012B31
:10CCF00001D1012300E00023002B3CD13B681B68DD
:10CD0000102B1DD17B681B68B3F1A04F18D1FB6DB0
:10CD10009B6843F40002FB6D9A60264B1B68264A11
:10CD2000A2FB03239A0C13469B0013445B00BB60D9
:10CD300002E0BB68013BBB60BB68002BF9D12EE071
:10CD40003B681B68112B0BD17B681B68B3F1A04FAC
:10CD500006D1FB6D9B6843F08072FB6D9A601EE00C
:10CD60003B681B68122B1AD1FB6D9B6843F4800251
:10CD7000FB6D9A6013E07B681B6C43F020027B68BC
:10CD80001A64012387F867300AE07B681B6C43F064
:10CD900020027B681A64012387F8673000E000BF37
:10CDA0007B68002283F83C2097F867301846683784
:10CDB000BD4680BD0800002083DE1B4380B598B0CF
:10CDC00000AF78603960002387F85F307B681B68AC
:10CDD000B3F1A04F04D041F695319148FBF7E3FA47
:10CDE0003B681B68002B20D03B681B68012B1CD0C4
:10CDF0003B681B68022B18D03B681B68032B14D0C0
:10CE00003B681B68052B10D03B681B68062B0CD0B9
:10CE10003B681B68072B08D03B681B68092B04D0B4
:10CE200041F696317E48FBF7BEFA3B681B68002B43
:10CE300052D03B685B68002B0ED03B685B68B3F553
:10CE4000004F09D03B685B68B3F5404F04D041F612
:10CE500099317348FBF7A7FA3B689B68002B3BD0DE
:10CE60003B689B68B3F5807F36D03B689B68B3F521
:10CE7000007F31D03B689B68B3F5407F2CD03B6886
:10CE80009B68B3F5806F27D03B689B68B3F5A06FB4
:10CE900022D03B689B68B3F5C06F1DD03B689B6890
:10CEA000B3F5E06F18D03B689B68B3F5006F13D003
:10CEB0003B689B68B3F5106F0ED03B689B68B3F579
:10CEC000206F09D03B689B68B3F5306F04D041F602
:10CED0009A315348FBF767FA7B681B68B3F1A04FA0
:10CEE00002D1504BBB6002E04FF0A043BB60BB6877
:10CEF000002B01D10123AAE07B6893F83C30012B81
:10CF000001D10223A3E07B68012283F83C207B68E7
:10CF10001B689B6803F00403002B40F08780BB680C
:10CF20009B6803F00403002B40F080803E4BBB6500
:10CF30003B681B68002B40D0BB6D9B6823F46042AC
:10CF40003B6859687B6893F830305B030B431A43A6
:10CF5000BB6D9A607B681B689B6803F00303012B21
:10CF600008D17B681B681B6803F00103012B01D10A
:10CF7000012300E00023002B62D1BB689B6803F013
:10CF80000303012B07D1BB681B6803F00103012BCE
:10CF900001D1012300E00023002B51D1BB6D9B6820
:10CFA00023F4716323F00F033A6811683A689268BA
:10CFB0000A431A43BB6D9A6042E0BB6D9B6823F441
:10CFC0006042BB6D9A607B681B689B6803F003033B
:10CFD000012B08D17B681B681B6803F00103012B40
:10CFE00001D1012300E00023002B29D1BB689B68FD
:10CFF00003F00303012B07D1BB681B6803F0010397
:10D00000012B01D1012300E00023002B18D1BB6DBF
:10D010009B6823F4716323F00F03BA6D93600FE0F4
:10D02000489C020800010050000300507B681B6C04
:10D0300043F020027B681A64012387F85F3000E028
:10D0400000BF7B68002283F83C2097F85F301846C9
:10D050006037BD4680BD00BF80B584B000AF78604A
:10D060000023FB607B681B689B6803F00303012BB4
:10D0700008D17B681B681B6803F00103012B01D1F9
:10D08000012300E00023002B43D17B681B689A68D2
:10D09000224B1340002B0DD07B681B6C43F0100219
:10D0A0007B681A647B685B6C43F001027B685A649E
:10D0B00001232FE07B681B689A687B681B6842F03D
:10D0C00001029A6000F092F9F8601BE000F08EF91E
:10D0D0000246FB68D31A022B14D97B681B681B68B5
:10D0E00003F00103012B0DD07B681B6C43F0100291
:10D0F0007B681A647B685B6C43F001027B685A644E
:10D10000012307E07B681B681B6803F00103012B08
:10D11000DCD1002318461037BD4680BD3F0000809B
:10D1200080B584B000AF78600023FB607B681B682B
:10D130009B6803F00303012B08D17B681B681B6805
:10D1400003F00103012B01D1012300E00023002B98
:10D1500047D07B681B689B6803F00D03012B0FD140
:10D160007B681B689A687B681B6842F002029A60C1
:10D170007B681B6803221A6000F038F9F86029E028
:10D180007B681B6C43F010027B681A647B685B6CE5
:10D1900043F001027B685A64012323E000F026F982
:10D1A0000246FB68D31A022B14D97B681B689B6864
:10D1B00003F00103012B0DD17B681B6C43F01002BF
:10D1C0007B681A647B685B6C43F001027B685A647D
:10D1D000012307E07B681B689B6803F00103012BB8
:10D1E000DCD0002318461037BD4680BD80B586B020
:10D1F00000AF7860396000237B610023FB6000236F
:10D200003B617B681B68B3F1A04F09D07B681B684A
:10D210005E4A934204D041F6EF415D48FBF7C3F804
:10D220003B680C2B0AD03B68602B07D03B686C2B0B
:10D2300004D041F6F0415648FBF7B5F87B681B680F
:10D240009B6803F00C03002B00F09B807B681B683D
:10D25000DB6803F00073B3F1007F2AD17B685B7E4B
:10D26000012B26D17B681B7E012B22D10C233B6036
:10D2700014E03B69474A93420DD97B681B6C43F02D
:10D2800010027B681A647B685B6C43F001027B6868
:10D290005A64012376E03B6901333B617B681B687C
:10D2A0001B6803F04003402BE3D17B681B684022DE
:10D2B0001A603B68602B15D07B681B689B6803F085
:10D2C0000403042B0ED17B681B689B6803F00203E8
:10D2D000002B07D17B681B689A687B681B6842F04B
:10D2E00010029A603B680C2B15D07B681B689B680A
:10D2F00003F00803082B0ED17B681B689B6803F0C2
:10D300000203002B07D17B681B689A687B681B6847
:10D3100042F020029A603B68602B05D03B686C2B82
:10D3200005D10C237B6105E008237B6102E0042327
:10D330007B6100BF00F05AF8F8601BE000F056F87F
:10D340000246FB68D31A0B2B14D97B681B689A68BA
:10D350007B691340002B0DD07B681B6C43F01002DF
:10D360007B681A647B685B6C43F001027B685A64DB
:10D37000012307E07B681B689A687B691340002BD8
:10D38000DCD1002318461837BD4680BD000100508F
:10D39000489C0208FF93090080B500AF084B1B684A
:10D3A000074A43F010031360032002F09FFE0F2092
:10D3B000FBF7DEFFFBF7B8FF0023184680BD00BF78
:10D3C0000020024080B400AF064B1B781A46064B83
:10D3D0001B681344044A136000BFBD465DF8047B1C
:10D3E000704700BF04000020080A002080B400AF8E
:10D3F000034B1B681846BD465DF8047B704700BFB1
:10D40000080A002080B584B000AF7860FFF7EEFF17
:10D41000B8607B68FB60FB68B3F1FF3F05D00A4B47
:10D420001B781A46FB681344FB6000BFFFF7DEFF62
:10D430000246BB68D31AFA689A42F7D800BF00BF09
:10D440001037BD4680BD00BF0400002080B5ADF59B
:10D45000007D00AF07F50073A3F5FE73186007F5B4
:10D460000073A3F5FE731B68002B02D1012301F0AA
:10D470009AB907F50073A3F5FE731B681B68002BB0
:10D480002CD007F50073A3F5FE731B681B6803F02F
:10D490000103002B22D107F50073A3F5FE731B686F
:10D4A0001B6803F00203002B18D107F50073A3F5E6
:10D4B000FE731B681B6803F00803002B0ED107F5F1
:10D4C0000073A3F5FE731B681B6803F00403002BB5
:10D4D00004D140F24911BA48FAF765FF07F5007325
:10D4E000A3F5FE731B681B6803F00103002B00F01B
:10D4F0009D8107F50073A3F5FE731B685B68002B25
:10D5000016D007F50073A3F5FE731B685B68B3F5CF
:10D51000803F0DD007F50073A3F5FE731B685B68B1
:10D52000B3F5A02F04D040F24F11A548FAF73BFF06
:10D53000A44B5B6803F00C03042B0CD0A14B5B687D
:10D5400003F00C03082B5CD19E4B5B6803F4803323
:10D55000B3F5803F55D14FF40033C7F8F031D7F819
:10D56000F03193FAA3F3C7F8EC31D7F8EC31B3FA02
:10D5700083F3DBB25B09DBB243F00103DBB2012BC7
:10D5800002D1904B1B6815E04FF40033C7F8E83127
:10D59000D7F8E83193FAA3F3C7F8E4314FF4003336
:10D5A000C7F8E031D7F8E03193FAA3F3C7F8DC31DC
:10D5B000844B5B6A4FF40032C7F8D821D7F8D821E2
:10D5C00092FAA2F2C7F8D421D7F8D421B2FA82F2A3
:10D5D000D2B242F02002D2B202F01F02012101FABF
:10D5E00002F21340002B00F0208107F50073A3F531
:10D5F000FE731B685B68002B40F01781012301F06C
:10D60000D2B807F50073A3F5FE731B685B68B3F52A
:10D61000803F06D16B4B1B686A4A43F4803313602A
:10D6200036E007F50073A3F5FE731B685B68002BFB
:10D630000CD1644B1B68634A23F480331360614B45
:10D640001B68604A23F48023136021E007F5007310
:10D65000A3F5FE731B685B68B3F5A02F0CD1594B83
:10D660001B68584A43F480231360564B1B68554A85
:10D6700043F4803313600BE0524B1B68514A23F490
:10D68000803313604F4B1B684E4A23F48023136092
:10D690004C4BDB6A23F00F0207F50073A3F5FE7312
:10D6A0001B689B6847491343CB6207F50073A3F5DA
:10D6B000FE731B685B68002B59D0FFF797FEC7F815
:10D6C000F8010AE0FFF792FE0246D7F8F831D31AC4
:10D6D000642B02D9032301F066B84FF40033C7F876
:10D6E000D031D7F8D03193FAA3F3C7F8CC31D7F8BB
:10D6F000CC31B3FA83F3DBB25B09DBB243F0010355
:10D70000DBB2012B02D12F4B1B6815E04FF4003325
:10D71000C7F8C831D7F8C83193FAA3F3C7F8C431B2
:10D720004FF40033C7F8C031D7F8C03193FAA3F3F0
:10D73000C7F8BC31234B5B6A4FF40032C7F8B821FD
:10D74000D7F8B82192FAA2F2C7F8B421D7F8B421D9
:10D75000B2FA82F2D2B242F02002D2B202F01F023A
:10D76000012101FA02F21340002BABD05EE0FFF77B
:10D770003DFEC7F8F8010AE0FFF738FE0246D7F889
:10D78000F831D31A642B02D9032301F00CB84FF4FB
:10D790000033C7F8B031D7F8B03193FAA3F3C7F824
:10D7A000AC31D7F8AC31B3FA83F3DBB25B09DBB24F
:10D7B00043F00103DBB2012B06D1024B1B6819E0D9
:10D7C000809C0208001002404FF40033C7F8A831D3
:10D7D000D7F8A83193FAA3F3C7F8A4314FF4003374
:10D7E000C7F8A031D7F8A03193FAA3F3C7F89C315A
:10D7F000C04B5B6A4FF40032C7F89821D7F89821E4
:10D8000092FAA2F2C7F89421D7F89421B2FA82F2E0
:10D81000D2B242F02002D2B202F01F02012101FA7C
:10D8200002F21340002BA7D100E000BF07F5007300
:10D83000A3F5FE731B681B6803F00203002B00F0C6
:10D84000A28107F50073A3F5FE731B681B69002B0B
:10D850000CD007F50073A3F5FE731B681B69012B41
:10D8600004D040F28711A448FAF79DFD07F5007334
:10D87000A3F5FE731B685B691F2B04D94FF4C471B9
:10D880009D48FAF790FD9B4B5B6803F00C03002B5F
:10D890000BD0984B5B6803F00C03082B72D1954BAF
:10D8A0005B6803F48033002B6CD10223C7F89031FE
:10D8B000D7F8903193FAA3F3C7F88C31D7F88C31AD
:10D8C000B3FA83F3DBB25B09DBB243F00103DBB2F3
:10D8D000012B02D1874B1B6813E00223C7F8883164
:10D8E000D7F8883193FAA3F3C7F884310223C7F835
:10D8F0008031D7F8803193FAA3F3C7F87C317D4BA0
:10D900005B6A0222C7F87821D7F8782192FAA2F24E
:10D91000C7F87421D7F87421B2FA82F2D2B242F079
:10D920002002D2B202F01F02012101FA02F21340DA
:10D93000002B0AD007F50073A3F5FE731B681B6963
:10D94000012B02D0012300F02EBF6A4B1B6823F08D
:10D95000F80207F50073A3F5FE731B685B69F821F5
:10D96000C7F87011D7F8701191FAA1F1C7F86C11CE
:10D97000D7F86C11B1FA81F1C9B28B405D491343FC
:10D980000B6000E107F50073A3F5FE731B681B69CC
:10D99000002B00F088800123C7F86831D7F8683180
:10D9A00093FAA3F3C7F86431D7F86431B3FA83F379
:10D9B000DBB203F1845303F584139B001A46012361
:10D9C0001360FFF713FDC7F8F8010AE0FFF70EFD3B
:10D9D0000246D7F8F831D31A022B02D9032300F0FC
:10D9E000E2BE0223C7F86031D7F8603193FAA3F39F
:10D9F000C7F85C31D7F85C31B3FA83F3DBB25B096B
:10DA0000DBB243F00103DBB2012B02D1394B1B68BF
:10DA100013E00223C7F85831D7F8583193FAA3F32B
:10DA2000C7F854310223C7F85031D7F8503193FA70
:10DA3000A3F3C7F84C312F4B5B6A0222C7F8482189
:10DA4000D7F8482192FAA2F2C7F84421D7F8442126
:10DA5000B2FA82F2D2B242F02002D2B202F01F0237
:10DA6000012101FA02F21340002BAFD0214B1B68B9
:10DA700023F0F80207F50073A3F5FE731B685B69DA
:10DA8000F821C7F84011D7F8401191FAA1F1C7F871
:10DA90003C11D7F83C11B1FA81F1C9B28B4015495C
:10DAA00013430B606FE00123C7F83831D7F83831E2
:10DAB00093FAA3F3C7F83431D7F83431B3FA83F3C8
:10DAC000DBB203F1845303F584139B001A46002351
:10DAD0001360FFF78BFCC7F8F8010FE0FFF786FC37
:10DAE0000246D7F8F831D31A022B07D9032300F0E6
:10DAF0005ABE00BF00100240809C02080223C7F8F3
:10DB00003031D7F8303193FAA3F3C7F82C31D7F876
:10DB10002C31B3FA83F3DBB25B09DBB243F00103D0
:10DB2000DBB2012B02D1814B1B6813E00223C7F843
:10DB30002831D7F8283193FAA3F3C7F82431022308
:10DB4000C7F82031D7F8203193FAA3F3C7F81C3176
:10DB5000764B5B6A0222C7F81821D7F8182192FA8F
:10DB6000A2F2C7F81421D7F81421B2FA82F2D2B285
:10DB700042F02002D2B202F01F02012101FA02F2A9
:10DB80001340002BAAD107F50073A3F5FE731B68A1
:10DB90001B6803F00803002B00F02B8107F50073CE
:10DBA000A3F5FE731B689B69002B0CD007F500736F
:10DBB000A3F5FE731B689B69012B04D04FF4E4713D
:10DBC0005B48FAF7F0FB07F50073A3F5FE731B68DB
:10DBD0009B69002B79D00123C7F81031D7F8103199
:10DBE00093FAA3F3C7F80C31D7F80C31B3FA83F3E7
:10DBF000DBB21A464F4B13449B001A4601231360B5
:10DC0000FFF7F4FBC7F8F8010AE0FFF7EFFB024665
:10DC1000D7F8F831D31A022B02D9032300F0C3BD81
:10DC20000223C7F80831D7F8083193FAA3F3C7F8ED
:10DC3000043107F50073A3F5807302221A6007F51B
:10DC40000073A3F580731B6893FAA3F207F50073C2
:10DC5000A3F582731A6007F50073A3F5847302229B
:10DC60001A6007F50073A3F584731B6893FAA3F297
:10DC700007F50073A3F586731A602C4B5A6A07F5F3
:10DC80000073A3F588730221196007F50073A3F5EB
:10DC900088731B6893FAA3F107F50073A3F58A73E1
:10DCA000196007F50073A3F58A731B68B3FA83F351
:10DCB000DBB243F06003DBB203F01F03012101FA82
:10DCC00003F31340002BA0D093E007F50073A3F5F6
:10DCD0008C7301221A6007F50073A3F58C731B681F
:10DCE00093FAA3F207F50073A3F58E731A6007F594
:10DCF0000073A3F58E731B68B3FA83F3DBB21A4685
:10DD00000C4B13449B001A4600231360FFF76EFB75
:10DD1000C7F8F80110E0FFF769FB0246D7F8F831C1
:10DD2000D31A022B08D9032300F03DBD0010024096
:10DD3000809C02082081901007F50073A3F5907372
:10DD400002221A6007F50073A3F590731B6893FA1B
:10DD5000A3F207F50073A3F592731A6007F5007339
:10DD6000A3F5947302221A6007F50073A3F5947368
:10DD70001B6893FAA3F207F50073A3F596731A6074
:10DD800007F50073A3F5987302221A6007F5007374
:10DD9000A3F598731B6893FAA3F207F50073A3F534
:10DDA0009A731A60B84B5A6A07F50073A3F59C730F
:10DDB0000221196007F50073A3F59C731B6893FAA1
:10DDC000A3F107F50073A3F59E73196007F50073BF
:10DDD000A3F59E731B68B3FA83F3DBB243F06003D1
:10DDE000DBB203F01F03012101FA03F31340002B00
:10DDF00091D107F50073A3F5FE731B681B6803F050
:10DE00000403002B00F0C081002387F8FF3107F5E1
:10DE10000073A3F5FE731B68DB68002B14D007F5B5
:10DE20000073A3F5FE731B68DB68012B0CD007F5AC
:10DE30000073A3F5FE731B68DB68052B04D04FF459
:10DE4000FA719248FAF7AFFA8F4BDB6903F080530F
:10DE5000002B16D18C4BDB698B4A43F08053D36186
:10DE6000894BDB6903F0805207F50073A3F5FC735F
:10DE70001A6007F50073A3F5FC731B68012387F88C
:10DE8000FF31834B1B6803F48073002B1BD1804B45
:10DE90001B687F4A43F480731360FFF7A7FAC7F843
:10DEA000F8010AE0FFF7A2FA0246D7F8F831D31AD0
:10DEB000642B02D9032300F076BC754B1B6803F476
:10DEC0008073002BEED007F50073A3F5FE731B687B
:10DED000DB68012B06D16C4B1B6A6B4A43F00103D4
:10DEE000136235E007F50073A3F5FE731B68DB686A
:10DEF000002B0CD1644B1B6A634A23F001031362AD
:10DF0000614B1B6A604A23F00403136220E007F5AB
:10DF10000073A3F5FE731B68DB68052B0CD15A4B0D
:10DF20001B6A594A43F004031362574B1B6A564A53
:10DF300043F0010313620BE0534B1B6A524A23F078
:10DF400001031362504B1B6A4F4A23F00403136210
:10DF500007F50073A3F5FE731B68DB68002B00F068
:10DF60008280FFF743FAC7F8F8010CE0FFF73EFAAA
:10DF70000246D7F8F831D31A41F28832934202D9D7
:10DF8000032300F010BC07F50073A3F5A073022271
:10DF90001A6007F50073A3F5A0731B6893FAA3F248
:10DFA00007F50073A3F5A2731A6007F50073A3F5D4
:10DFB000A47302221A6007F50073A3F5A4731B680B
:10DFC00093FAA3F207F50073A3F5A6731A6007F599
:10DFD0000073A3F5A6731B68B3FA83F3DBB25B0986
:10DFE000DBB243F00203DBB2022B02D1264B1B6AE9
:10DFF00013E007F50073A3F5A87302221A6007F572
:10E000000073A3F5A8731B6893FAA3F207F50073D6
:10E01000A3F5AA731A601C4B5B6A07F50072A2F5A0
:10E02000AC720221116007F50072A2F5AC721268A1
:10E0300092FAA2F107F50072A2F5AE72116007F52F
:10E040000072A2F5AE721268B2FA82F2D2B242F057
:10E050004002D2B202F01F02012101FA02F2134083
:10E06000002B83D086E0FFF7C1F9C7F8F80111E073
:10E07000FFF7BCF90246D7F8F831D31A41F28832DB
:10E08000934207D903238EE300100240809C0208CC
:10E090000070004007F50073A3F5B07302221A6008
:10E0A00007F50073A3F5B0731B6893FAA3F207F5A5
:10E0B0000073A3F5B2731A6007F50073A3F5B47388
:10E0C00002221A6007F50073A3F5B4731B6893FA74
:10E0D000A3F207F50073A3F5B6731A6007F5007392
:10E0E000A3F5B6731B68B3FA83F3DBB25B09DBB24B
:10E0F00043F00203DBB2022B02D1BB4B1B6A13E0DD
:10E1000007F50073A3F5B87302221A6007F50073D0
:10E11000A3F5B8731B6893FAA3F207F50073A3F590
:10E12000BA731A60B04B5B6A07F50072A2F5BC7255
:10E130000221116007F50072A2F5BC72126892FA12
:10E14000A2F107F50072A2F5BE72116007F5007228
:10E15000A2F5BE721268B2FA82F2D2B242F0400266
:10E16000D2B202F01F02012101FA02F21340002B89
:10E170007FF47EAF97F8FF31012B05D19A4BDB6915
:10E18000994A23F08053D36107F50073A3F5FE731A
:10E190001B68DB69002B14D007F50073A3F5FE7331
:10E1A0001B68DB69012B0CD007F50073A3F5FE7328
:10E1B0001B68DB69022B04D04FF40E718B48FAF711
:10E1C000F2F807F50073A3F5FE731B68DB69002BFB
:10E1D00000F0E882844B5B6803F00C03082B00F02E
:10E1E000B68207F50073A3F5FE731B68DB69022B8B
:10E1F00040F0078207F50073A3F5FE731B681B6AE6
:10E20000002B0DD007F50073A3F5FE731B681B6A86
:10E21000B3F5803F04D040F241217448FAF7C3F8C7
:10E2200007F50073A3F5FE731B685B6A002B00F013
:10E23000838007F50073A3F5FE731B685B6AB3F573
:10E24000802F79D007F50073A3F5FE731B685B6A16
:10E25000B3F5002F70D007F50073A3F5FE731B68AC
:10E260005B6AB3F5402F67D007F50073A3F5FE7323
:10E270001B685B6AB3F5801F5ED007F50073A3F5DA
:10E28000FE731B685B6AB3F5A01F55D007F50073DA
:10E29000A3F5FE731B685B6AB3F5C01F4CD007F58E
:10E2A0000073A3F5FE731B685B6AB3F5E01F43D0F0
:10E2B00007F50073A3F5FE731B685B6AB3F5001FD7
:10E2C0003AD007F50073A3F5FE731B685B6AB3F5DC
:10E2D000101F31D007F50073A3F5FE731B685B6A4E
:10E2E000B3F5201F28D007F50073A3F5FE731B6854
:10E2F0005B6AB3F5301F1FD007F50073A3F5FE73FB
:10E300001B685B6AB3F5401F16D007F50073A3F5D1
:10E31000FE731B685B6AB3F5501F0DD007F50073E1
:10E32000A3F5FE731B685B6AB3F5601F04D040F26F
:10E3300042212E48FAF737F807F50073A3F5C073AA
:10E340004FF080721A6007F50073A3F5C0731B6865
:10E3500093FAA3F207F50073A3F5C2731A6007F5E9
:10E360000073A3F5C2731B68B3FA83F3DBB203F146
:10E37000845303F584139B001A4600231360FFF7B0
:10E3800035F8C7F8F80109E0FFF730F80246D7F88A
:10E39000F831D31A022B01D9032304E207F50073E5
:10E3A000A3F5C4734FF000721A6007F50073A3F56C
:10E3B000C4731B6893FAA3F207F50073A3F5C67341
:10E3C0001A6007F50073A3F5C6731B68B3FA83F3ED
:10E3D000DBB25B09DBB243F00103DBB2012B07D1F7
:10E3E000014B1B682CE000BF00100240809C02081B
:10E3F00007F50073A3F5C8734FF000721A6007F5B4
:10E400000073A3F5C8731B6893FAA3F207F50073B2
:10E41000A3F5CA731A6007F50073A3F5CC734FF028
:10E4200000721A6007F50073A3F5CC731B6893FAAA
:10E43000A3F207F50073A3F5CE731A60C94B5B6AAC
:10E4400007F50072A2F5D0724FF00071116007F568
:10E450000072A2F5D072126892FAA2F107F500726A
:10E46000A2F5D272116007F50072A2F5D27212689D
:10E47000B2FA82F2D2B242F02002D2B202F01F020D
:10E48000012101FA02F21340002B7FF47DAFB54B5E
:10E490005B6823F4741207F50073A3F5FE731B6821
:10E4A000596A07F50073A3F5FE731B681B6A0B43DB
:10E4B000AC4913434B6007F50073A3F5D4734FF0D9
:10E4C00080721A6007F50073A3F5D4731B6893FA82
:10E4D000A3F207F50073A3F5D6731A6007F500736E
:10E4E000A3F5D6731B68B3FA83F3DBB203F184534D
:10E4F00003F584139B001A4601231360FEF776FF91
:10E50000C7F8F80109E0FEF771FF0246D7F8F831C5
:10E51000D31A022B01D9032345E107F50073A3F5B4
:10E52000D8734FF000721A6007F50073A3F5D87323
:10E530001B6893FAA3F207F50073A3F5DA731A6068
:10E5400007F50073A3F5DA731B68B3FA83F3DBB244
:10E550005B09DBB243F00103DBB2012B02D1814B3B
:10E560001B6827E007F50073A3F5DC734FF000721A
:10E570001A6007F50073A3F5DC731B6893FAA3F226
:10E5800007F50073A3F5DE731A6007F50073A3F5B2
:10E59000E0734FF000721A6007F50073A3F5E073A3
:10E5A0001B6893FAA3F207F50073A3F5E2731A60F0
:10E5B0006C4B5B6A07F50072A2F5E4724FF00071D4
:10E5C000116007F50072A2F5E472126892FAA2F1E6
:10E5D00007F50072A2F5E672116007F50072A2F568
:10E5E000E6721268B2FA82F2D2B242F02002D2B2DD
:10E5F00002F01F02012101FA02F21340002B82D027
:10E60000D0E007F50073A3F5E8734FF080721A604D
:10E6100007F50073A3F5E8731B6893FAA3F207F5F7
:10E620000073A3F5EA731A6007F50073A3F5EA73A4
:10E630001B68B3FA83F3DBB203F1845303F584134D
:10E640009B001A4600231360FEF7D0FEC7F8F801BE
:10E6500009E0FEF7CBFE0246D7F8F831D31A022BB9
:10E6600001D903239FE007F50073A3F5EC734FF086
:10E6700000721A6007F50073A3F5EC731B6893FA38
:10E68000A3F207F50073A3F5EE731A6007F50073A4
:10E69000A3F5EE731B68B3FA83F3DBB25B09DBB25D
:10E6A00043F00103DBB2012B02D12E4B1B6827E0A4
:10E6B00007F50073A3F5F0734FF000721A6007F5C9
:10E6C0000073A3F5F0731B6893FAA3F207F50073C8
:10E6D000A3F5F2731A6007F50073A3F5F4734FF016
:10E6E00000721A6007F50073A3F5F4731B6893FAC0
:10E6F000A3F207F50073A3F5F6731A60194B5B6A72
:10E7000007F50072A2F5F8724FF00071116007F57D
:10E710000072A2F5F872126892FAA2F107F500727F
:10E72000A2F5FA72116007F50072A2F5FA7212688A
:10E73000B2FA82F2D2B242F02002D2B202F01F024A
:10E74000012101FA02F21340002B82D12AE007F5E1
:10E750000073A3F5FE731B68DB69012B04D1012351
:10E7600021E000BF00100240114B5B68C7F8F43194
:10E77000D7F8F43103F4803207F50073A3F5FE7384
:10E780001B681B6A9A420BD1D7F8F43103F470125C
:10E7900007F50073A3F5FE731B685B6A9A4201D00C
:10E7A000012300E00023184607F50077BD4680BD31
:10E7B0000010024080B59EB000AF78603960002341
:10E7C0007B677B68002B01D1012305E27B681B6816
:10E7D00003F00103002B16D17B681B6803F00203D2
:10E7E000002B10D17B681B6803F00403002B0AD1B7
:10E7F0007B681B6803F00803002B04D140F2C121A1
:10E800009A48F9F7D0FD3B68002B0AD03B68012BF2
:10E8100007D03B68022B04D040F2C2219348F9F79D
:10E82000C2FD934B1B6803F007033A689A4210D964
:10E830008F4B1B6823F007028D493B6813430B6025
:10E840008B4B1B6803F007033A689A4201D00123FF
:10E85000C2E17B681B6803F00203002B31D07B68A8
:10E860009B68002B24D07B689B68802B20D07B6822
:10E870009B68902B1CD07B689B68A02B18D07B6872
:10E880009B68B02B14D07B689B68C02B10D07B6832
:10E890009B68D02B0CD07B689B68E02B08D07B68F2
:10E8A0009B68F02B04D040F2D9217048F9F77BFD2A
:10E8B000704B5B6823F0F0027B689B686D491343E3
:10E8C0004B607B681B6803F00103002B00F0F580B0
:10E8D0007B685B68002B0CD07B685B68012B08D0E1
:10E8E0007B685B68022B04D04FF438715F48F9F7FE
:10E8F0005AFD7B685B68012B3DD14FF400333B67C9
:10E900003B6F93FAA3F3FB66FB6EB3FA83F3DBB2C0
:10E910005B09DBB243F00103DBB2012B02D1554BA3
:10E920001B680FE04FF40033BB66BB6E93FAA3F392
:10E930007B664FF400333B663B6E93FAA3F3FB65B3
:10E940004C4B5B6A4FF40032BA65BA6D92FAA2F290
:10E950007A657A6DB2FA82F2D2B242F02002D2B275
:10E9600002F01F02012101FA02F21340002B40F0D5
:10E970008380012330E17B685B68022B3CD14FF040
:10E9800000733B653B6D93FAA3F3FB64FB6CB3FA36
:10E9900083F3DBB25B09DBB243F00103DBB2012B93
:10E9A00002D1344B1B680FE04FF00073BB64BB6CAB
:10E9B00093FAA3F37B644FF000733B643B6C93FAD0
:10E9C000A3F3FB632B4B5B6A4FF00072BA63BA6B25
:10E9D00092FAA2F27A637A6BB2FA82F2D2B242F07F
:10E9E0002002D2B202F01F02012101FA02F213400A
:10E9F000002B41D10123EFE002233B633B6B93FAF1
:10EA0000A3F3FB62FB6AB3FA83F3DBB25B09DBB20D
:10EA100043F00103DBB2012B02D1164B1B680DE062
:10EA20000223BB62BB6A93FAA3F37B6202233B62BD
:10EA30003B6A93FAA3F3FB610E4B5B6A0222BA6155
:10EA4000BA6992FAA2F27A617A69B2FA82F2D2B221
:10EA500042F02002D2B202F01F02012101FA02F2BA
:10EA60001340002B08D10123B6E000BF809C0208B0
:10EA70000020024000100240594B5B6823F0030263
:10EA80007B685B68564913434B60FEF7AFFC7867C1
:10EA90000AE0FEF7ABFC02467B6FD31A41F28832E4
:10EAA000934201D9032397E04D4B5B6803F00C02BE
:10EAB0007B685B689B009A42EBD14A4B1B6803F072
:10EAC00007033A689A4210D2464B1B6823F00702AC
:10EAD00044493B6813430B60424B1B6803F0070338
:10EAE0003A689A4201D0012376E07B681B6803F004
:10EAF0000403002B25D07B68DB68002B18D07B68D3
:10EB0000DB68B3F5806F13D07B68DB68B3F5A06F6B
:10EB10000ED07B68DB68B3F5C06F09D07B68DB681B
:10EB2000B3F5E06F04D04FF447712F48F9F73BFC81
:10EB30002B4B5B6823F4E0627B68DB682849134356
:10EB40004B607B681B6803F00803002B26D07B68B2
:10EB50001B69002B18D07B681B69B3F5806F13D03D
:10EB60007B681B69B3F5A06F0ED07B681B69B3F59A
:10EB7000C06F09D07B681B69B3F5E06F04D040F229
:10EB800023311948F9F70FFC154B5B6823F46052E9
:10EB90007B681B69DB00124913434B6000F02CF8C3
:10EBA00001460F4B5B6803F0F003F0223A613A69CB
:10EBB00092FAA2F2FA60FA68B2FA82F2D2B2D340C2
:10EBC0000A4AD35C21FA03F3094A1360094B1B6814
:10EBD0001846FAF7CDFB002318467837BD4680BDAE
:10EBE0000010024000200240809C0208949F02080E
:10EBF000080000200000002080B487B000AF002390
:10EC0000FB600023BB6000237B6100237B6000234B
:10EC10003B611E4B5B68FB60FB6803F00C03042B3D
:10EC200002D0082B03D026E0194B3B6126E0FB689D
:10EC30009B0C03F00F03174AD35C7B60134BDB6A1A
:10EC400003F00F03144AD35CBB60FB6803F480330A
:10EC5000002B08D00E4ABB68B2FBF3F27B6802FBC4
:10EC600003F37B6104E07B680C4A02FB03F37B61E6
:10EC70007B693B6102E0064B3B6100BF3B69184684
:10EC80001C37BD465DF8047B704700BF0010024092
:10EC900000127A00749F0208849F020800093D0058
:10ECA00080B400AF034B1B681846BD465DF8047B7B
:10ECB000704700BF0800002080B582B000AFFFF7AA
:10ECC000EFFF01460B4B5B6803F4E0634FF4E06237
:10ECD0007A607A6892FAA2F23A603A68B2FA82F2FC
:10ECE000D2B2D340044AD35C21FA03F31846083762
:10ECF000BD4680BD00100240A49F020880B582B0CE
:10ED000000AFFFF7CDFF01460B4B5B6803F4605388
:10ED10004FF460527A607A6892FAA2F23A603A68E6
:10ED2000B2FA82F2D2B2D340044AD35C21FA03F39E
:10ED300018460837BD4680BD00100240A49F020857
:10ED400080B582B000AF786039607B68002B04D159
:10ED500040F285411848F9F726FB3B68002B04D1A7
:10ED600040F286411448F9F71EFB7B680F221A60B7
:10ED7000124B5B6803F003027B685A600F4B5B68C1
:10ED800003F0F0027B689A600C4B5B6803F4E0626E
:10ED90007B68DA60094B5B68DB0803F4E0627B6840
:10EDA0001A61074B1B6803F007023B681A6000BF3B
:10EDB0000837BD4680BD00BF809C0208001002409D
:10EDC0000020024080B592B000AF786000233B6421
:10EDD0000023FB63002387F847307B681B68624A87
:10EDE000934203D970216148F9F7DDFA7B681B680B
:10EDF00003F48033002B00F0F1807B685B68002B0C
:10EE000012D07B685B68B3F5807F0DD07B685B6850
:10EE1000B3F5007F08D07B685B68B3F5407F03D013
:10EE200076215248F9F7BFFA514BDB6903F0805362
:10EE3000002B0ED14E4BDB694D4A43F08053D3611A
:10EE40004B4BDB6903F08053BB60BB68012387F841
:10EE50004730484B1B6803F48073002B18D1454B97
:10EE60001B68444A43F480731360FEF7BFFA3864AA
:10EE700008E0FEF7BBFA02463B6CD31A642B01D9BB
:10EE800003234FE23B4B1B6803F48073002BF0D04D
:10EE9000374B1B6A03F44073FB63FB6B002B00F0E2
:10EEA0008A807B685B6803F44073FA6B9A4200F0D7
:10EEB00082802F4B1B6A23F44073FB634FF4803333
:10EEC0003B633B6B93FAA3F3FB62FB6AB3FA83F3F6
:10EED000DBB21A46284B13449B001A4601231360E9
:10EEE0004FF48033BB63BB6B93FAA3F37B637B6B01
:10EEF000B3FA83F3DBB21A461F4B13449B001A4646
:10EF0000002313601A4AFB6B1362FB6B03F00103CF
:10EF1000002B50D0FEF76AFA38640AE0FEF766FA72
:10EF200002463B6CD31A41F28832934201D9032343
:10EF3000F8E10223BB62BB6A93FAA3F37B6202236C
:10EF40003B623B6A93FAA3F3FB61FB69B3FA83F379
:10EF5000DBB25B09DBB243F00203DBB2022B0DD163
:10EF6000034B1B6A12E000BFFF120300B89C0208AB
:10EF70000010024000700040008190100223BB612D
:10EF8000BB6993FAA3F37B61894B5B6A02223A6106
:10EF90003A6992FAA2F2FA60FA68B2FA82F2D2B24E
:10EFA00042F04002D2B202F01F02012101FA02F245
:10EFB0001340002BB2D07E4B1B6A23F440727B6857
:10EFC0005B687B4913430B6297F84730012B05D1EF
:10EFD000774BDB69764A23F08053D3617B681B68EB
:10EFE00003F00103002B1CD07B689B68002B0FD023
:10EFF0007B689B68012B0BD07B689B68022B07D03A
:10F000007B689B68032B03D0BC216A48F9F7CBF9D6
:10F01000674B1B6B23F003027B689B6864491343B7
:10F020000B637B681B6803F00203002B1FD07B6817
:10F03000DB68002B12D07B68DB68B3F5803F0DD016
:10F040007B68DB68B3F5003F08D07B68DB68B3F50D
:10F05000403F03D0C7215748F9F7A5F9544B1B6B24
:10F0600023F440327B68DB68514913430B637B68B0
:10F070001B6803F00403002B1FD07B681B69002B67
:10F0800012D07B681B69B3F5802F0DD07B681B699C
:10F09000B3F5002F08D07B681B69B3F5402F03D070
:10F0A000D3214448F9F77FF9414B1B6B23F44022ED
:10F0B0007B681B693E4913430B637B681B6803F045
:10F0C0002003002B14D07B68DB69002B07D07B6802
:10F0D000DB69102B03D0DE213648F9F764F9344B95
:10F0E0001B6B23F010027B68DB69314913430B6310
:10F0F0007B681B6803F40033002B15D07B681B6B07
:10F10000B3F5800F07D07B681B6B002B03D0EC217D
:10F110002848F9F748F9264B5B6823F480027B689E
:10F120001B6B234913434B607B681B6803F0400350
:10F13000002B15D07B681B6A002B08D07B681B6AEC
:10F14000202B04D04FF480711A48F9F72CF9184B92
:10F150001B6B23F020027B681B6A154913430B636A
:10F160007B681B6803F00803002B25D07B685B6974
:10F17000002B13D07B685B69B3F5801F0ED07B68D2
:10F180005B69B3F5001F09D07B685B69B3F5401F6D
:10F1900004D040F221110748F9F705F9044B1B6B25
:10F1A00023F440127B685B69014913430B6303E05E
:10F1B00000100240B89C02087B681B6803F0100333
:10F1C000002B20D07B689B69002B13D07B689B6948
:10F1D000B3F5800F0ED07B689B69B3F5000F09D0A3
:10F1E0007B689B69B3F5400F04D040F22B114F4868
:10F1F000F9F7D9F84E4B1B6B23F440027B689B69EF
:10F200004B4913430B637B681B6803F40073002BAB
:10F2100016D07B689B6A002B09D07B689B6AB3F58C
:10F22000000F04D040F23B114048F9F7BCF8404BC6
:10F230005B6823F400027B689B6A3D4913434B6083
:10F240007B681B6803F08003002B4DD07B685B6AF2
:10F25000002B40D07B685B6AB3F5807F3BD07B6836
:10F260005B6AB3F5887F36D07B685B6AB3F5907FC5
:10F2700031D07B685B6AB3F5987F2CD07B685B6A82
:10F28000B3F5A07F27D07B685B6AB3F5A87F22D057
:10F290007B685B6AB3F5B07F1DD07B685B6AB3F5B2
:10F2A000B87F18D07B685B6AB3F5C07F13D07B68EA
:10F2B0005B6AB3F5C87F0ED07B685B6AB3F5D07F1D
:10F2C00009D07B685B6AB3F5D87F04D040F25B114C
:10F2D0001648F9F768F8164BDB6A23F4F8727B6876
:10F2E0005B6A13491343CB627B681B6803F480534A
:10F2F000002B16D07B68DB6A002B09D07B68DB6AA9
:10F30000B3F5807F04D04FF4C6710848F9F74BF885
:10F31000074B1B6B23F480727B68DB6A0449134341
:10F320000B63002318464837BD4680BDB89C0208D1
:10F330000010024080B586B000AF786039600023CD
:10F340007B617B68B3F1904F17D07B68364A93425C
:10F3500013D07B68354A93420FD07B68344A93427E
:10F360000BD07B68334A934207D07B68324A934282
:10F3700003D0B2213148F9F716F83B681B689BB2FD
:10F38000002B05D03B681B681B0C1B04002B03D013
:10F39000B3212A48F9F707F83B685B68002B00F0B7
:10F3A00000823B685B68012B00F0FB813B685B6877
:10F3B000112B00F0F6813B685B68022B00F0F181B5
:10F3C0003B685B68122B00F0EC813B685B68B3F52F
:10F3D000881F00F0E6813B685B68B3F5041F00F00E
:10F3E000E0813B685B68B3F5441F00F0DA813B685D
:10F3F0005B68B3F5901F00F0D4813B685B68B3F5A0
:10F40000081F00F0CE813B685B68B3F5481F00F031
:10F41000C8813B685B68032B00F0C381B4210748B7
:10F42000F8F7C1FFBDE100BF000400480008004834
:10F43000000C00480010004800140048F09C02082E
:10F440003B681A6801217B6901FA03F31340FB60F2
:10F45000FB68002B00F0A2813B685B6803F00303AC
:10F46000012B05D03B685B6803F00303022B40D1FE
:10F470003B68DB68002B0BD03B68DB68012B07D0B7
:10F480003B68DB68032B03D0C3218A48F8F78BFF66
:10F490007B689B683B617B695B00032202FA03F394
:10F4A000DB433A6913403B613B68DA687B695B0088
:10F4B00002FA03F33A6913433B617B683A699A6045
:10F4C0007B685B683B6101227B6902FA03F3DB43E3
:10F4D0003A6913403B613B685B681B0903F001021A
:10F4E0007B6902FA03F33A6913433B617B683A692B
:10F4F0005A603B685B6803F00303032B27D03B682B
:10F500009B68002B0BD03B689B68012B07D03B68A6
:10F510009B68022B03D0D4216648F8F744FF7B6830
:10F52000DB683B617B695B00032202FA03F3DB4388
:10F530003A6913403B613B689A687B695B0002FA59
:10F5400003F33A6913433B617B683A69DA603B68CD
:10F550005B6803F00303022B4FD17B68B3F1904F3C
:10F5600017D07B68544A934213D07B68534A934226
:10F570000FD07B68524A93420BD07B68514A93422A
:10F5800007D07B68504A934203D0E2214948F8F7FC
:10F590000AFF3B681B690C2B0BD93B681B690E2BC0
:10F5A00007D03B681B690F2B03D0E3214148F8F7D4
:10F5B000FAFE7B69DA087B68083253F822303B6137
:10F5C0007B6903F007039B000F2202FA03F3DB437E
:10F5D0003A6913403B613B681A697B6903F0070392
:10F5E0009B0002FA03F33A6913433B617B69DA0833
:10F5F0007B680832396943F822107B681B683B61DD
:10F600007B695B00032202FA03F3DB433A69134090
:10F610003B613B685B6803F003027B695B0002FAB5
:10F6200003F33A6913433B617B683A691A603B68AC
:10F630005B6803F44033002B00F0B080234B9B69E0
:10F64000224A43F001039361204B9B6903F00103BD
:10F65000BB60BB681E4A7B699B08023352F82330AB
:10F660003B617B6903F003039B000F2202FA03F363
:10F67000DB433A6913403B617B68B3F1904F29D07B
:10F680007B680D4A934213D07B680C4A93420DD09D
:10F690007B680B4A934207D07B680A4A934201D1A8
:10F6A000042318E0052316E0032314E0022312E0EC
:10F6B000012310E0F09C0208000400480008004804
:10F6C000000C0048001000480014004800100240E0
:10F6D0000000014000237A6902F003029200934087
:10F6E0003A6913433B6135497B699B0802333A69A8
:10F6F00041F82320324B9B683B61FB68DB433A694E
:10F7000013403B613B685B6803F48013002B03D01C
:10F710003A69FB6813433B61294A3B699360284B74
:10F72000DB683B61FB68DB433A6913403B613B6844
:10F730005B6803F40013002B03D03A69FB681343A2
:10F740003B611F4A3B69D3601D4B5B683B61FB68B3
:10F75000DB433A6913403B613B685B6803F4003369
:10F76000002B03D03A69FB6813433B61144A3B69A1
:10F770005360134B1B683B61FB68DB433A691340E2
:10F780003B613B685B6803F48033002B03D03A692C
:10F79000FB6813433B610A4A3B6913607B69013391
:10F7A0007B613B681A687B6922FA03F3002B7FF4C4
:10F7B00047AE00BF00BF1837BD4680BD0000014006
:10F7C0000004014080B584B000AF78600B467B80B8
:10F7D0007B88002B04D07B881B0C1B04002B04D0DF
:10F7E0004FF4C2710948F8F7DEFD7B681A697B881F
:10F7F0001340002B02D00123FB7301E00023FB73B5
:10F80000FB7B18461037BD4680BD00BFF09C020848
:10F8100080B582B000AF78600B467B8013467B706A
:10F820007B88002B04D07B881B0C1B04002B04D08E
:10F830004FF4D2710D48F8F7B6FD7B78002B07D056
:10F840007B78012B04D040F2A5110848F8F7ABFDF6
:10F850007B78002B03D07A887B689A6102E07A88F3
:10F860007B689A6200BF0837BD4680BDF09C0208E5
:10F8700080B584B000AF78600B467B807B88002B1E
:10F8800004D07B881B0C1B04002B04D04FF4DE71CA
:10F890000A48F8F788FD7B685B69FB607A88FB683B
:10F8A00013401A04FB68D9437B880B401A437B68DA
:10F8B0009A6100BF1037BD4680BD00BFF09C0208B2
:10F8C00080B582B000AF0346FB80084B5A69FB88C5
:10F8D0001340002B06D0054AFB885361FB8818466D
:10F8E0000AF0DEFC00BF0837BD4680BD00040140C1
:10F8F00080B584B000AF78600023FB607B68002B8C
:10F9000001D10123E7E07B681B68754A93423AD036
:10F910007B681B68734A934235D07B681B68724AC8
:10F92000934230D07B681B68704A93422BD07B682F
:10F930001B686F4A934226D07B681B686D4A9342CE
:10F9400021D07B681B686C4A93421CD07B681B6883
:10F950006A4A934217D07B681B68694A934212D067
:10F960007B681B68674A93420DD07B681B68664AB8
:10F97000934208D07B681B68644A934203D093216A
:10F980006348F8F710FD7B685B68002B0CD07B6840
:10F990005B68102B08D07B685B68B3F5804F03D0A1
:10F9A00094215B48F8F7FFFC7B689B68402B07D0ED
:10F9B0007B689B68002B03D095215548F8F7F3FC32
:10F9C0007B68DB68802B07D07B68DB68002B03D06B
:10F9D00096214F48F8F7E7FC7B681B69002B0DD098
:10F9E0007B681B69B3F5807F08D07B681B69B3F522
:10F9F000007F03D097214648F8F7D5FC7B685B6908
:10FA0000002B0DD07B685B69B3F5806F08D07B68F5
:10FA10005B69B3F5006F03D098213D48F8F7C3FC4C
:10FA20007B689B69002B07D07B689B69202B03D0E8
:10FA300099213748F8F7B7FC7B68DB69002B12D0B7
:10FA40007B68DB69B3F5805F0DD07B68DB69B3F55C
:10FA5000005F08D07B68DB69B3F5405F03D09A2173
:10FA60002B48F8F7A0FC7B68022283F821207B68F2
:10FA70001B681B68FB60FB6823F47F5323F0300393
:10FA8000FB607B685A687B689B681A437B68DB680D
:10FA90001A437B681B691A437B685B691A437B685E
:10FAA0009B691A437B68DB691343FA681343FB6065
:10FAB0007B681B68FA681A60786800F0F3F97B6865
:10FAC00000229A637B68012283F821207B68002250
:10FAD00083F82020002318461037BD4680BD00BFA4
:10FAE000080002401C000240300002404400024076
:10FAF000580002406C0002408000024008040240AE
:10FB00001C040240300402404404024058040240F5
:10FB1000289D020880B586B000AFF860B9607A60B1
:10FB20003B600023FB753B68002B03D03B68B3F5BB
:10FB3000803F04D34FF4A6712C48F8F734FCFB68DF
:10FB400093F82030012B01D102234AE0FB68012207
:10FB500083F82020FB6893F82130012B3AD1FB6811
:10FB6000022283F82120FB6800229A63FB681B684D
:10FB70001A68FB681B6822F001021A603B687A6809
:10FB8000B968F86800F05FF9FB68DB6A002B08D001
:10FB9000FB681B681A68FB681B6842F00E021A605B
:10FBA0000FE0FB681B681A68FB681B6842F00A02DA
:10FBB0001A60FB681B681A68FB681B6822F0040265
:10FBC0001A60FB681B681A68FB681B6842F0010238
:10FBD0001A6005E0FB68002283F820200223FB75F1
:10FBE000FB7D18461837BD4680BD00BF289D020822
:10FBF00080B483B000AF78607B68002B01D1012313
:10FC00002EE07B6893F82130022B08D07B68042219
:10FC10009A637B68002283F82020012320E07B6820
:10FC20001B681A687B681B6822F00E021A607B68EA
:10FC30001B681A687B681B6822F001021A607B68E7
:10FC40001A6C7B68DB6B012101FA02F25A607B6857
:10FC5000012283F821207B68002283F820200023E2
:10FC600018460C37BD465DF8047B704780B584B0FC
:10FC700000AF78600023FB737B6893F82130022B80
:10FC800005D07B6804229A630123FB7327E07B681D
:10FC90001B681A687B681B6822F00E021A607B687A
:10FCA0001B681A687B681B6822F001021A607B6877
:10FCB0001A6C7B68DB6B012101FA02F25A607B68E7
:10FCC000012283F821207B68002283F820207B68B2
:10FCD0005B6B002B03D07B685B6B78689847FB7B82
:10FCE00018461037BD4680BD80B584B000AF78603F
:10FCF0007B68DB6B1B68FB607B681B681B68BB60F9
:10FD00007B681B6C04229A40FB681340002B24D0B4
:10FD1000BB6803F00403002B1FD07B681B681B68C3
:10FD200003F02003002B07D17B681B681A687B68EF
:10FD30001B6822F004021A607B681A6C7B68DB6B1C
:10FD4000042101FA02F25A607B68DB6A002B6AD058
:10FD50007B68DB6A7868984765E07B681B6C0222E9
:10FD60009A40FB681340002B2CD0BB6803F00203C1
:10FD7000002B27D07B681B681B6803F02003002B37
:10FD80000BD17B681B681A687B681B6822F00A022B
:10FD90001A607B68012283F821207B681A6C7B68DB
:10FDA000DB6B022101FA02F25A607B68002283F8C1
:10FDB00020207B689B6A002B35D07B689B6A786823
:10FDC000984730E07B681B6C08229A40FB68134020
:10FDD000002B28D0BB6803F00803002B23D07B68DE
:10FDE0001B681A687B681B6822F00E021A607B6829
:10FDF0001A6C7B68DB6B012101FA02F25A607B68A6
:10FE000001229A637B68012283F821207B6800220B
:10FE100083F820207B681B6B002B04D07B681B6B56
:10FE200078689847FFE700BF1037BD4680BD80B4B3
:10FE300083B000AF78607B689B6B18460C37BD467B
:10FE40005DF8047B704780B485B000AFF860B9609E
:10FE50007A603B60FB681A6CFB68DB6B012101FA7E
:10FE600002F25A60FB681B683A685A60FB685B687C
:10FE7000102B08D1FB681B687A689A60FB681B68C6
:10FE8000BA68DA6007E0FB681B68BA689A60FB68CA
:10FE90001B687A68DA6000BF1437BD465DF8047BE2
:10FEA0007047000080B483B000AF78607B681B6847
:10FEB0001A46144B9A420FD87B681B681A46124B9D
:10FEC0001344124AA2FB03231B099A007B681A649D
:10FED0007B680F4ADA630EE07B681B681A460D4B9D
:10FEE00013440A4AA2FB03231B099A007B681A6485
:10FEF0007B68094ADA6300BF0C37BD465DF8047BB6
:10FF0000704700BF07040240F8FFFDBFCDCCCCCC4A
:10FF100000000240F8FBFDBF0004024080B485B041
:10FF200000AF78607B6803F00703FB600C4BDB6875
:10FF3000BB60BA684FF6FF031340BB60FB681A0250
:10FF4000BB68134343F0BF6343F40033BB60044A10
:10FF5000BB68D36000BF1437BD465DF8047B7047B3
:10FF600000ED00E080B400AF044BDB681B0A03F037
:10FF700007031846BD465DF8047B704700ED00E0BE
:10FF800080B483B000AF0346FB7197F90730002BB4
:10FF90000BDBFB7903F01F02074997F907305B0978
:10FFA000012000FA02F241F8232000BF0C37BD46C1
:10FFB0005DF8047B704700BF00E100E080B483B0CF
:10FFC00000AF0346FB7197F90730002B12DBFB797A
:10FFD00003F01F020A4997F907305B09012000FA74
:10FFE00002F2203341F82320BFF34F8F00BFBFF34D
:10FFF0006F8F00BF00BF0C37BD465DF8047B7047B4
:020000040801F1
:1000000000E100E080B483B000AF03463960FB71CB
:1000100097F90730002B0ADB3B68DAB20C4997F9F5
:1000200007301201D2B20B4483F800230AE03B6888
:10003000DAB20849FB7903F00F03043B1201D2B294
:100040000B441A7600BF0C37BD465DF8047B704741
:1000500000E100E000ED00E080B489B000AFF8609E
:10006000B9607A60FB6803F00703FB61FB69C3F1C9
:100070000703042B28BF0423BB61FB690433062B51
:1000800002D9FB69033B00E000237B614FF0FF32A4
:10009000BB6902FA03F3DA43BB681A407B699A40F2
:1000A0004FF0FF317B6901FA03F3D9437B680B40C2
:1000B000134318462437BD465DF8047B70470000A3
:1000C00080B400AFBFF34F8F00BF064BDB6803F473
:1000D000E0620449044B1343CB60BFF34F8F00BF72
:1000E00000BFFDE700ED00E00400FA0580B582B036
:1000F00000AF78607B68072B0FD07B68062B0CD095
:100100007B68052B09D07B68042B06D07B68032B0A
:1001100003D0AB210448F8F746F97868FFF7FEFEF4
:1001200000BF0837BD4680BD609D020880B586B01F
:1001300000AF0346B9607A60FB7300237B617B6884
:100140000F2B03D9C3210E48F8F72DF9BB680F2BED
:1001500003D9C4210A48F8F726F9FFF703FF7861AD
:100160007A68B9687869FFF777FF024697F90F3028
:1001700011461846FFF746FF00BF1837BD4680BD41
:10018000609D020880B582B000AF0346FB7197F90D
:100190000730002B03DAD7210548F8F704F997F95F
:1001A00007301846FFF7ECFE00BF0837BD4680BD9C
:1001B000609D020880B582B000AF0346FB7197F9DD
:1001C0000730002B03DAE7210548F8F7ECF897F938
:1001D00007301846FFF7F2FE00BF0837BD4680BD66
:1001E000609D020880B500AFFFF76AFF80B500AFE1
:1001F000064B5B6903F48033002B05D000F008F850
:10020000024B4FF480325A6100BF80BD00040140B0
:1002100080B400AF00BFBD465DF8047B70470000AE
:10022000F0B587B000AFF860B960C7E900230123DB
:10023000FB750023BB7500237B75454B1B7E012B93
:1002400001D1022380E0424B01221A76FB68012B88
:1002500009D0FB68022B06D0FB68032B03D0B0212A
:100260003C48F8F7A0F8BB68B3F1006F16D33A4BDF
:100270001B88B3F5807F04D1BB68384A93420DD800
:1002800010E0354B1B88802B04D1BB68344A934265
:1002900004D807E0BB68334A934203D9B1212D4803
:1002A000F8F781F84CF2503000F0B2F80346FB75D5
:1002B000FB7D002B44D1FB68012B02D101237B7510
:1002C00007E0FB68022B02D102237B7501E00423C7
:1002D0007B750023BB752DE0BB7D5A00BB6802EB2C
:1002E000030CBB7D1901D7E90023C1F12006A1F160
:1002F000200022FA01F403FA06F6344323FA00F050
:10030000044323FA01F5A3B21946604600F064F8ED
:100310004CF2503000F07CF80346FB75124B1B6921
:10032000114A23F001031361FB7D002B07D1BB7D34
:100330000133BB75BA7D7B7D9A42CDD300E000BF0F
:10034000034B00221A76FB7D18461C37BD46F0BDD4
:10035000100A0020989D0208CCF7FF1FFFFF03083A
:10036000FFFF0108FFFF00080020024080B483B0B7
:1003700000AF0023FB710D4B1B6903F08003002BC2
:100380000DD00A4B0A4A5A60084B0A4A5A60074B7A
:100390001B6903F08003002B01D00123FB71FB7963
:1003A00018460C37BD465DF8047B704700200240BC
:1003B00023016745AB89EFCD80B400AF054B1B69C6
:1003C000044A43F08003136100231846BD465DF8DC
:1003D000047B70470020024080B483B000AF786097
:1003E0000B467B80084B0022DA61084B1B69074AE9
:1003F00043F0010313617B687A881A8000BF0C37D1
:10040000BD465DF8047B7047100A002000200240C2
:1004100080B584B000AF7860FCF7E8FFF86010E0CA
:100420007B68B3F1FF3F0CD07B68002B07D0FCF753
:10043000DDFF0246FB68D31A7A689A4201D2032391
:100440001FE0124BDB6803F00103012BE8D00F4BD8
:10045000DB6803F02003202B02D10C4B2022DA6052
:100460000A4BDB6803F01003102B05D0074BDB6849
:1004700003F00403042B03D100F00AF8012300E089
:10048000002318461037BD4680BD00BF0020024043
:1004900080B483B000AF00237B60144BDB6803F0B3
:1004A0001003102B09D1124BDB6943F00203104AF1
:1004B000D3617B6843F010037B600C4BDB6803F077
:1004C0000403042B09D10A4BDB6943F00103084AFA
:1004D000D3617B6843F004037B60044A7B68D3608C
:1004E00000BF0C37BD465DF8047B7047002002401A
:1004F000100A002080B584B000AF78603960012315
:10050000FB730023BB60624B1B7E012B01D10223D6
:10051000BAE05F4B01221A767B681B68002B07D07C
:100520007B681B68012B03D0A6215A48F7F73BFFD5
:100530007B681B68012B16D14CF25030FFF768FF27
:100540000346002B40F09C8000F0B0F84CF2503095
:10055000FFF75EFF0346FB734F4B1B694E4A23F0C8
:10056000040313618CE07B685B68B3F1006F19D3FF
:100570004A4B1B88B3F5807F05D17B685B68484A8E
:1005800093420FD812E0454B1B88802B05D17B6826
:100590005B68444A934205D808E07B685B68424A3E
:1005A000934203D9BC213B48F7F7FDFE3B4B1B8828
:1005B000B3F5807F0DD17B685A687B689B68DB024E
:1005C0001344013B364A934294BF01230023DBB21C
:1005D0001EE0324B1B88802B0DD17B685A687B68EC
:1005E0009B68DB021344013B2E4A934294BF0123D4
:1005F0000023DBB20CE07B685A687B689B68DB02F7
:100600001344013B284A934294BF01230023DBB2E9
:10061000002B03D1BD211F48F7F7C5FE4CF2503027
:10062000FFF7F6FE0346002B2AD13B684FF0FF325E
:100630001A607B685B68BB6019E0B86800F050F82E
:100640004CF25030FFF7E4FE0346FB73124B1B697C
:10065000114A23F002031361FB7B002B03D03B689C
:10066000BA681A600CE0BB6803F50063BB607B6886
:100670009B68DA027B685B681344BA689A42DCD3F1
:10068000034B00221A76FB7B18461037BD4680BD0F
:10069000100A0020D09D020800200240CCF7FF1F66
:1006A000FFFF0308FFFF0108FFFF000880B400AF51
:1006B000094B0022DA61094B1B69084A43F0040325
:1006C0001361064B1B69054A43F04003136100BFE9
:1006D000BD465DF8047B7047100A002000200240F0
:1006E00080B483B000AF78600B4B0022DA610B4B13
:1006F0001B690A4A43F002031361084A7B6853618D
:10070000064B1B69054A43F04003136100BF0C37D9
:10071000BD465DF8047B7047100A002000200240AF
:1007200080B584B000AF78607B68002B01D10123D5
:1007300009E27B681B688F4A934204D04FF48F71A3
:100740008D48F7F730FE7B681B7E002B08D07B6856
:100750001B7E012B04D040F21F118748F7F723FEC0
:100760007B685B7E002B08D07B685B7E012B04D00E
:100770004FF490718048F7F716FE7B689B7E002B44
:1007800008D07B689B7E012B04D040F221117A486F
:10079000F7F709FE7B68DB7E002B08D07B68DB7EE9
:1007A000012B04D04FF491717348F7F7FCFD7B687F
:1007B0001B7F002B08D07B681B7F012B04D040F2ED
:1007C00023116D48F7F7EFFD7B685B7F002B08D0A6
:1007D0007B685B7F012B04D04FF492716648F7F77A
:1007E000E2FD7B689B68002B13D07B689B68B3F1AC
:1007F000804F0ED07B689B68B3F1004F09D07B68B7
:100800009B68B3F1404F04D040F225115A48F7F7E6
:10081000CAFD7B68DB68002B13D07B68DB68B3F113
:10082000807F0ED07B68DB68B3F1007F09D07B68E6
:10083000DB68B3F1407F04D04FF493714E48F7F773
:10084000B2FD7B681B69002B4FD07B681B69B3F539
:10085000803F4AD07B681B69B3F5003F45D07B6879
:100860001B69B3F5403F40D07B681B69B3F5802F0F
:100870003BD07B681B69B3F5A02F36D07B681B6922
:10088000B3F5C02F31D07B681B69B3F5E02F2CD0B6
:100890007B681B69B3F5002F27D07B681B69B3F514
:1008A000102F22D07B681B69B3F5202F1DD07B68E9
:1008B0001B69B3F5302F18D07B681B69B3F5402F47
:1008C00013D07B681B69B3F5502F0ED07B681B6972
:1008D000B3F5602F09D07B681B69B3F5702F04D086
:1008E00040F227112448F7F75EFD7B685B69002B17
:1008F00027D07B685B69B3F5801F22D07B685B697A
:10090000B3F5001F1DD07B685B69B3F5401F18D09D
:100910007B685B69B3F5800F13D07B685B69B3F5C7
:10092000A00F0ED07B685B69B3F5C00F09D07B6860
:100930005B69B3F5E00F04D04FF494710E48F7F7FC
:1009400032FD7B685B68002B04D07B685B68B3F585
:10095000806F04D940F229110748F7F724FD7B681E
:1009600093F82030DBB2002B08D17868F7F722FF2C
:1009700004E000BF006400400C9E02087B681B6816
:100980001A687B681B6842F001021A60FCF72EFDB2
:10099000F86012E0FCF72AFD0246FB68D31A0A2B26
:1009A0000BD97B685B6A43F400327B685A627B68D0
:1009B000052283F820200123C5E07B681B685B6863
:1009C00003F00103002BE5D07B681B681A687B6885
:1009D0001B6822F002021A60FCF708FDF86012E0C2
:1009E000FCF704FD0246FB68D31A0A2B0BD97B687F
:1009F0005B6A43F400327B685A627B68052283F8A5
:100A0000202001239FE07B681B685B6803F00203E2
:100A1000002BE5D17B681B7E012B08D17B681B680E
:100A20001A687B681B6842F080021A6007E07B68E6
:100A30001B681A687B681B6822F080021A607B685A
:100A40005B7E012B08D17B681B681A687B681B687A
:100A500042F040021A6007E07B681B681A687B68F6
:100A60001B6822F040021A607B689B7E012B08D134
:100A70007B681B681A687B681B6842F020021A605A
:100A800007E07B681B681A687B681B6822F02002FD
:100A90001A607B68DB7E012B08D17B681B681A68B3
:100AA0007B681B6822F010021A6007E07B681B68F5
:100AB0001A687B681B6842F010021A607B681B7F13
:100AC000012B08D17B681B681A687B681B6842F0A1
:100AD00008021A6007E07B681B681A687B681B685D
:100AE00022F008021A607B685B7F012B08D17B68CB
:100AF0001B681A687B681B6842F004021A6007E0F2
:100B00007B681B681A687B681B6822F004021A6005
:100B10007B689A687B68DB681A437B681B691A43A9
:100B20007B685B6942EA03017B685B685A1E7B68ED
:100B30001B680A43DA617B6800225A627B680122E3
:100B400083F82020002318461037BD4680BD00BF23
:100B500080B586B000AF786039607B681B687B61C8
:100B60007B6893F82030FB74FB7C012B03D0FB7C6B
:100B7000022B40F00F813B681B68B3F5803F04D324
:100B800040F252318948F7F70EFC3B685B68B3F5D9
:100B9000803F04D340F253318448F7F704FC3B68AC
:100BA0009B68B3F5803F04D34FF455717F48F7F746
:100BB000FAFB3B68DB68B3F5803F04D340F2553164
:100BC0007A48F7F7F0FB3B689B69002B08D03B683D
:100BD0009B69012B04D040F256317448F7F7E3FBD0
:100BE0003B68DB69002B08D03B68DB69012B04D034
:100BF00040F257316D48F7F7D6FB3B681B69002B75
:100C000008D03B681B69012B04D04FF4567167482C
:100C1000F7F7C9FB3B681B6A002B08D03B681B6ACF
:100C2000012B04D040F259316048F7F7BCFB3B6818
:100C30005B690D2B04D940F25E315C48F7F7B3FBDA
:100C40007B69D3F8003243F001027B69C3F80022CC
:100C50003B685B6903F01F03012202FA03F3FB60A8
:100C60007B69D3F81C22FB68DB431A407B69C3F81D
:100C70001C223B68DB69002B23D17B69D3F80C2253
:100C8000FB68DB431A407B69C3F80C223B68DB68D6
:100C900019043B685B689BB23A68526919437B69E7
:100CA000483243F832103B689B6819043B681B6864
:100CB0009AB23B685B690A4379694833DB000B44AD
:100CC0005A603B68DB69012B22D17B69D3F80C2287
:100CD000FB681A437B69C3F80C223B681B68190444
:100CE0003B685B689BB23A68526919437B6948323A
:100CF00043F832103B689B6819043B68DB689AB282
:100D00003B685B690A4379694833DB000B445A60EE
:100D10003B689B69002B09D17B69D3F80422FB68EF
:100D2000DB431A407B69C3F8042207E07B69D3F8F0
:100D30000422FB681A437B69C3F804223B681B69E1
:100D4000002B09D17B69D3F81422FB68DB431A40DE
:100D50007B69C3F8142207E07B69D3F81422FB688F
:100D60001A437B69C3F814223B681B6A012B07D125
:100D70007B69D3F81C22FB681A437B69C3F81C22E9
:100D80007B69D3F8003223F001027B69C3F80022AB
:100D9000002306E07B685B6A43F480227B685A622A
:100DA000012318461837BD4680BD00BF0C9E0208BF
:100DB00080B584B000AF78607B6893F82030DBB2F8
:100DC000012B2ED17B68022283F820207B681B68D0
:100DD0001A687B681B6822F001021A60FCF706FBA8
:100DE000F86012E0FCF702FB0246FB68D31A0A2BFC
:100DF0000BD97B685B6A43F400327B685A627B687C
:100E0000052283F82020012312E07B681B685B68C1
:100E100003F00103002BE5D17B6800225A62002316
:100E200006E07B685B6A43F400227B685A62012318
:100E300018461037BD4680BD80B588B000AFF86059
:100E4000B9607A603B60FB6893F82030FB77FB6801
:100E50001B689B68BB61BB689B68002B08D0BB68A4
:100E60009B68042B04D040F2BE417F48F7F79BFA01
:100E7000BB68DB68002B08D0BB68DB68022B04D0A2
:100E800040F2BF417848F7F78EFABB681B69082B20
:100E900004D94FF498617448F7F785FABB689B68EA
:100EA000002B0AD1BB681B68B3F5006F0FD340F26B
:100EB000C3416D48F7F777FA09E0BB685B68B3F1A7
:100EC000005F04D340F2C7416748F7F76CFABB688C
:100ED0001B7D002B08D0BB681B7D012B04D040F28A
:100EE000C9416148F7F75FFAFB7F012B03D0FB7F15
:100EF000022B40F0AD80BB6903F08063002B0AD168
:100F0000BB6903F00063002B05D1BB6903F080537C
:100F1000002B00F09580BB691B0E03F003037B617F
:100F200001227B699A403B681A60BB689B68002B72
:100F30000DD1BB681B685A05BB68DB68F968096896
:100F40001A437B6918331B010B441A600FE0BB681E
:100F50005B68DA00BB689B681A43BB68DB68F968AA
:100F600009681A437B6918331B010B441A60FB683C
:100F70001968BB681A697B6918331B010B44043379
:100F80001A60BB681B7D012B11D1FB681A687B6955
:100F900018331B01134404331B68FA68116843F4C7
:100FA00080727B6918331B010B4404331A607B6821
:100FB00007331B781A067B6806331B781B041A4319
:100FC0007B6805331B781B0213437A68043212785E
:100FD0001046FA68116843EA00027B691B010B4462
:100FE00003F5C6731A607B6803331B781A067B68A7
:100FF00002331B781B041A437B6801331B781B02E6
:1010000013437A6812781046FA68116843EA0002BE
:101010007B691B010B4403F5C4731A60FB681A68F3
:101020007B6918331B0113441B68FA68116843F08D
:1010300001027B6918331B010B441A6000230EE088
:10104000FB685B6A43F40012FB685A62012306E006
:10105000FB685B6A43F48022FB685A6201231846EE
:101060002037BD4680BD00BF0C9E020880B485B00D
:1010700000AF78600023FB607B6893F82030FB7240
:10108000FB7A012B02D0FB7A022B1DD17B681B68F7
:101090009B6803F08063002B02D0FB680133FB6088
:1010A0007B681B689B6803F00063002B02D0FB6821
:1010B0000133FB607B681B689B6803F08053002B47
:1010C00002D0FB680133FB60FB6818461437BD464D
:1010D0005DF8047B7047000080B586B000AFF86013
:1010E000B9607A603B60FB6893F82030FB75BB68A1
:1010F000002B07D0BB68012B04D040F2BD518C48B7
:10110000F7F751F9FB7D012B03D0FB7D022B40F05B
:101110000381BB68002B0ED1FB681B68DB6803F002
:101120000303002B16D1FB685B6A43F40012FB68D3
:101130005A620123F7E0FB681B681B6903F0030395
:10114000002B07D1FB685B6A43F40012FB685A620C
:101150000123E8E0FB681A68BB681B331B011344DA
:101160001B6803F004027B689A607B689B68002B15
:101170000CD1FB681A68BB681B331B0113441B6846
:101180005B0DC3F30A027B681A600BE0FB681A6808
:10119000BB681B331B0113441B68DB0823F0604250
:1011A0007B685A60FB681A68BB681B331B011344D9
:1011B0001B6803F002027B68DA60FB681A68BB6890
:1011C0001B331B01134404331B6803F00803002B7B
:1011D00003D07B6808221A610BE0FB681A68BB68C1
:1011E0001B331B01134404331B6803F00F027B689D
:1011F0001A61FB681A68BB681B331B011344043374
:101200001B681B0ADAB27B689A61FB681A68BB68C4
:101210001B331B01134404331B681B0C9AB27B68FD
:101220005A61FB681A68BB681B01134403F5DC7341
:101230001B68DAB23B681A70FB681A68BB681B014E
:10124000134403F5DC731B681A0A3B680133D2B2FE
:101250001A70FB681A68BB681B01134403F5DC7342
:101260001B681A0C3B680233D2B21A70FB681A680A
:10127000BB681B01134403F5DC731B681A0E3B6843
:101280000333D2B21A70FB681A68BB681B0113449F
:1012900003F5DE731A683B680433D2B21A70FB6838
:1012A0001A68BB681B01134403F5DE731B681A0A36
:1012B0003B680533D2B21A70FB681A68BB681B0121
:1012C000134403F5DE731B681A0C3B680633D2B275
:1012D0001A70FB681A68BB681B01134403F5DE73C0
:1012E0001B681A0E3B680733D2B21A70BB68002B1A
:1012F00008D1FB681B68DA68FB681B6842F02002B3
:10130000DA6007E0FB681B681A69FB681B6842F03B
:1013100020021A61002306E0FB685B6A43F4802226
:10132000FB685A62012318461837BD4680BD00BFCE
:101330000C9E020880B584B000AF786039607B688D
:1013400093F82030FB733B68114A934204D940F272
:1013500056611048F7F727F8FB7B012B02D0FB7B87
:10136000022B09D17B681B6859697B681B683A6846
:101370000A435A61002306E07B685B6A43F48022DB
:101380007B685A62012318461037BD4680BD00BFF6
:101390007F8F03000C9E020880B58AB000AF786092
:1013A00000237B627B681B685B693B627B681B6810
:1013B0005B68FB617B681B689B68BB617B681B6823
:1013C000DB687B617B681B681B693B617B681B6812
:1013D0009B69FB603B6A03F00103002B7CD0BB6977
:1013E00003F00103002B23D07B681B6801229A6065
:1013F000BB6903F00203002B03D0786800F083F987
:1014000016E0BB6903F00403002B04D07B6A43F4AD
:1014100000637B620CE0BB6903F00803002B04D07F
:101420007B6A43F480537B6202E0786800F089F9BC
:10143000BB6903F48073002B24D07B681B684FF4D6
:1014400080729A60BB6903F40073002B03D0786844
:1014500000F063F916E0BB6903F48063002B04D04D
:101460007B6A43F400537B620CE0BB6903F40063C6
:10147000002B04D07B6A43F480437B6202E07868EF
:1014800000F069F9BB6903F48033002B24D07B683A
:101490001B684FF480329A60BB6903F40033002B61
:1014A00003D0786800F043F916E0BB6903F48023A9
:1014B000002B04D07B6A43F400437B620CE0BB69E1
:1014C00003F40023002B04D07B6A43F480337B6257
:1014D00002E0786800F049F93B6A03F00803002B4A
:1014E0000CD07B6903F01003002B07D07B6A43F418
:1014F00000737B627B681B681022DA603B6A03F032
:101500000403002B0BD07B6903F00803002B06D0EB
:101510007B681B680822DA60786800F030F93B6A63
:1015200003F00203002B09D07B681B68DB6803F023
:101530000303002B02D0786808F0F6F83B6A03F04A
:101540004003002B0CD03B6903F01003002B07D0A5
:101550007B6A43F480637B627B681B6810221A619C
:101560003B6A03F02003002B0BD03B6903F0080318
:10157000002B06D07B681B6808221A61786800F08F
:1015800012F93B6A03F01003002B09D07B681B683B
:101590001B6903F00303002B02D0786800F0F9F810
:1015A0003B6A03F40033002B0BD0FB6903F01003FC
:1015B000002B06D07B681B6810225A60786800F008
:1015C000FCF83B6A03F48033002B0BD0FB6903F07B
:1015D0000803002B06D07B681B6808225A607868D5
:1015E00000F0F5F83B6A03F40043002B7BD0FB6965
:1015F00003F00403002B72D03B6A03F48073002BCA
:1016000008D0FB6803F00103002B03D07B6A43F092
:1016100001037B623B6A03F40073002B08D0FB6874
:1016200003F00203002B03D07B6A43F002037B62CA
:101630003B6A03F48063002B08D0FB6803F00403CB
:10164000002B03D07B6A43F004037B623B6A03F404
:101650000063002B43D0FB6803F07003002B3ED0E7
:10166000FB6803F07003602B2BD0602B2ED8502B1F
:1016700022D0502B2AD8402B19D0402B26D8302BE3
:1016800010D0302B22D8102B02D0202B05D01DE0FB
:101690007B6A43F008037B6219E07B6A43F0100326
:1016A0007B6214E07B6A43F020037B620FE07B6A7D
:1016B00043F040037B620AE07B6A43F080037B6275
:1016C00005E07B6A43F480737B6200E000BF7B68C7
:1016D0001B689A697B681B6822F070029A617B68BC
:1016E0001B6804225A607B6A002B08D07B685A6A08
:1016F0007B6A1A437B685A62786800F072F800BF10
:101700002837BD4680BD80B483B000AF786000BF8D
:101710000C37BD465DF8047B704780B483B000AFE2
:10172000786000BF0C37BD465DF8047B704780B41D
:1017300083B000AF786000BF0C37BD465DF8047B16
:10174000704780B483B000AF786000BF0C37BD46EF
:101750005DF8047B704780B483B000AF786000BF51
:101760000C37BD465DF8047B704780B483B000AF92
:10177000786000BF0C37BD465DF8047B704780B4CD
:1017800083B000AF786000BF0C37BD465DF8047BC6
:10179000704780B483B000AF786000BF0C37BD469F
:1017A0005DF8047B704780B483B000AF786000BF01
:1017B0000C37BD465DF8047B704780B483B000AF42
:1017C000786000BF0C37BD465DF8047B704780B47D
:1017D00083B000AF786000BF0C37BD465DF8047B76
:1017E000704780B483B000AF786000BF0C37BD464F
:1017F0005DF8047B7047000080B582B000AF786070
:101800007B68002B01D1012377E07B689B69002B6B
:1018100014D07B681B683B4A93422DD07B681B68C1
:10182000394A934228D07B681B68384A934223D0B8
:101830004FF496713648F6F7B6FD1DE07B681B68DD
:10184000304A934218D07B681B682F4A934213D0CA
:101850007B681B682D4A93420ED07B681B682D4A1B
:10186000934209D07B681B682B4A934204D040F214
:1018700031112748F6F797FD7B68DB6F002B06D107
:101880007B68002283F878207868F7F773FB7B6821
:101890002422DA677B681B681A687B681B6822F061
:1018A00001021A607B685B6A002B02D0786800F046
:1018B00015FF786800F0B2FC0346012B01D101232B
:1018C0001BE07B681B685A687B681B6822F49042A7
:1018D0005A607B681B689A687B681B6822F02A0242
:1018E0009A607B681B681A687B681B6842F001027B
:1018F0001A60786801F042F8034618460837BD467A
:1019000080BD00BF00380140004400400048004056
:10191000449E0208004C00400050004080B58AB050
:1019200000AFF860B9601346FB80FB68DB6F202BCB
:1019300065D1BB68002B02D0FB88002B01D10123AD
:101940005EE0FB68BA68DA64FB68FA88A3F85020A6
:10195000FB68FA88A3F85220FB680022C3F88420B1
:10196000FB682122DA67FB681B6F002B27D0FB681E
:101970001B6F254A9A62FB681B6F244ADA62FB6878
:101980001B6F234A1A63FB681B6F00225A63FB68B4
:10199000186FFB68DB6C1946FB681B6828331A4616
:1019A000FB88FEF7B7F80346002B08D0FB6810222F
:1019B000C3F88420FB682022DA67012320E0FB685B
:1019C0001B6840221A62FB681B6808337B617B69D5
:1019D00053E8003F3B613B6943F080037B62FB6857
:1019E0001B6808337A6A3A62FB61F9693A6A41E82E
:1019F0000023BB61BB69002BE5D1002300E002237B
:101A000018462837BD4680BDFD2D0108912E0108DE
:101A10001130010880B58AB000AFF860B960134694
:101A2000FB80FB68D3F88030202B32D1BB68002BC1
:101A300002D0FB88002B01D101232BE0FB680022A0
:101A40001A66FB681B685B6803F40003002B18D060
:101A5000FB681B687B617B6953E8003F3B613B6926
:101A600043F080637B62FB681B681A467B6A3B62BB
:101A7000FA61F9693A6A41E80023BB61BB69002B4E
:101A8000E6D1FB881A46B968F86801F08DF803467C
:101A900000E0022318462837BD4680BD80B59AB0C5
:101AA00000AF78607B681B68BB64BB6C53E8003F89
:101AB0007B647B6C23F490737B667B681B681A469F
:101AC0007B6E7B653A65396D7A6D41E80023FB6476
:101AD000FB6C002BE6D17B681B6808337B637B6B58
:101AE00053E8003F3B633B6B23F001033B667B689D
:101AF0001B6808333A6E3A64FB63F96B3A6C41E851
:101B00000023BB63BB6B002BE5D17B681B6E012BF5
:101B100018D17B681B683B623B6A53E8003FFB615E
:101B2000FB6923F01003FB657B681B681A46FB6D9D
:101B3000FB62BA62B96AFA6A41E800237B627B6A97
:101B4000002BE6D17B681B689B6803F04003402BA9
:101B500037D17B681B680833FB60FB6853E8003FA4
:101B6000BB60BB6823F04003BB657B681B68083320
:101B7000BA6DBA617B617969BA6941E800233B615A
:101B80003B69002BE5D17B685B6F002B19D07B682C
:101B90005B6F00225A637B685B6F1846FEF728F87C
:101BA0000346002B0DD07B685B6F1846FEF73FF9AC
:101BB0000346202B05D17B681022C3F88420032321
:101BC00017E07B680022A3F85A207B681B680F226D
:101BD0001A627B681B689A697B681B6842F008027E
:101BE0009A617B682022C3F880207B6800221A66F5
:101BF000002318466837BD4680BD000080B5BAB0E6
:101C000000AF78607B681B68DB69C7F8E4307B68ED
:101C10001B681B68C7F8E0307B681B689B68C7F8C7
:101C2000DC30D7F8E42040F60F031340C7F8D83073
:101C3000D7F8D830002B15D1D7F8E43003F02003C3
:101C4000002B0FD0D7F8E03003F02003002B09D091
:101C50007B689B6E002B00F0AB827B689B6E786884
:101C60009847A5E2D7F8D830002B00F01781D7F8B5
:101C7000DC3003F00103002B06D1D7F8E020854BC0
:101C80001340002B00F00A81D7F8E43003F0010381
:101C9000002B11D0D7F8E03003F48073002B0BD069
:101CA0007B681B6801221A627B68D3F8843043F09A
:101CB00001027B68C3F88420D7F8E43003F0020304
:101CC000002B11D0D7F8DC3003F00103002B0BD030
:101CD0007B681B6802221A627B68D3F8843043F069
:101CE00004027B68C3F88420D7F8E43003F00403CF
:101CF000002B11D0D7F8DC3003F00103002B0BD000
:101D00007B681B6804221A627B68D3F8843043F036
:101D100002027B68C3F88420D7F8E43003F008039C
:101D2000002B17D0D7F8E03003F02003002B05D1AB
:101D3000D7F8DC3003F00103002B0BD07B681B6865
:101D400008221A627B68D3F8843043F008027B686B
:101D5000C3F88420D7F8E43003F40063002B12D0DA
:101D6000D7F8E03003F08063002B0CD07B681B6851
:101D70004FF400621A627B68D3F8843043F020028B
:101D80007B68C3F884207B68D3F88430002B00F094
:101D90001182D7F8E43003F02003002B0DD0D7F8E0
:101DA000E03003F02003002B07D07B689B6E002BF4
:101DB00003D07B689B6E786898477B68D3F8843043
:101DC000C7F8D4307B681B689B6803F04003402B46
:101DD00005D0D7F8D43003F02803002B4FD0786813
:101DE00000F0A8FF7B681B689B6803F04003402B52
:101DF00041D17B681B680833C7F89C30D7F89C300A
:101E000053E8003FC7F89830D7F8983023F04003E4
:101E1000C7F8D0307B681B680833D7F8D020C7F8E4
:101E2000A820C7F8A430D7F8A410D7F8A82041E814
:101E30000023C7F8A030D7F8A030002BD9D17B6899
:101E40005B6F002B13D07B685B6F134A5A637B6810
:101E50005B6F1846FDF70AFF0346002B17D07B681F
:101E60005B6F5B6B7A68526F104698470FE078683B
:101E700001F0EEFA0BE0786801F0EAFA07E0786822
:101E800001F0E6FA7B680022C3F8842092E100BFEB
:101E900090E100BF200100048F3001087B681B6EB9
:101EA000012B40F04B81D7F8E43003F01003002BF6
:101EB00000F04481D7F8E03003F01003002B00F06D
:101EC0003D817B681B6810221A627B681B689B68D7
:101ED00003F04003402B40F0B5807B685B6F1B68CC
:101EE0005B68A7F8BE30B7F8BE30002B00F0648105
:101EF0007B68B3F85830B7F8BE209A4280F05C8116
:101F00007B68B7F8BE20A3F85A207B685B6F9B699B
:101F1000202B00F086807B681B68C7F88830D7F8D4
:101F2000883053E8003FC7F88430D7F8843023F472
:101F30008073C7F8B8307B681B681A46D7F8B8308A
:101F4000C7F89430C7F89020D7F89010D7F89420AD
:101F500041E80023C7F88C30D7F88C30002BDAD159
:101F60007B681B6808337B677B6F53E8003F3B67E8
:101F70003B6F23F00103C7F8B4307B681B6808335C
:101F8000D7F8B420C7F88020FB67F96FD7F8802016
:101F900041E80023BB67BB6F002BE1D17B681B6866
:101FA00008333B663B6E53E8003FFB65FB6D23F057
:101FB0004003C7F8B0307B681B680833D7F8B020FF
:101FC000FA66BB66B96EFA6E41E800237B667B6EEB
:101FD000002BE3D17B682022C3F880207B6800229D
:101FE0001A667B681B68FB64FB6C53E8003FBB64AC
:101FF000BB6C23F01003C7F8AC307B681B681A4633
:10200000D7F8AC30BB657A65796DBA6D41E80023CD
:102010003B653B6D002BE4D17B685B6F1846FDF799
:10202000E7FD7B6802225A667B68B3F858207B681C
:10203000B3F85A309BB2D31A9BB21946786800F0B5
:10204000E1F8B9E07B68B3F858207B68B3F85A3000
:102050009BB2D31AA7F8CE307B68B3F85A309BB244
:10206000002B00F0AB80B7F8CE30002B00F0A6803C
:102070007B681B68BB63BB6B53E8003F7B637B6B78
:1020800023F49073C7F8C8307B681B681A46D7F8EA
:10209000C8307B643A64396C7A6C41E80023FB6396
:1020A000FB6B002BE4D17B681B6808337B627B6A87
:1020B00053E8003F3B623B6A23F00103C7F8C4309A
:1020C0007B681B680833D7F8C4203A63FB62F96A5F
:1020D0003A6B41E80023BB62BB6A002BE3D17B680B
:1020E0002022C3F880207B6800221A667B680022C9
:1020F0009A667B681B683B613B6953E8003FFB6065
:10210000FB6823F01003C7F8C0307B681B681A46D1
:10211000D7F8C030FB61BA61B969FA6941E80023B8
:102120007B617B69002BE4D17B6802225A66B7F899
:10213000CE301946786800F065F83FE0D7F8E43013
:1021400003F48013002B0ED0D7F8DC3003F48003A7
:10215000002B08D07B681B684FF480121A627868E5
:1021600000F0D5FF2DE0D7F8E43003F08003002B1A
:102170000ED0D7F8E03003F08003002B08D07B6846
:10218000DB6E002B1CD07B68DB6E7868984717E00D
:10219000D7F8E43003F04003002B12D0D7F8E0303A
:1021A00003F04003002B0CD0786800F086FF08E0B5
:1021B00000BF06E000BF04E000BF02E000BF00E097
:1021C00000BFE837BD4680BD80B483B000AF786003
:1021D00000BF0C37BD465DF8047B704780B483B008
:1021E00000AF786000BF0C37BD465DF8047B7047D8
:1021F00080B483B000AF786000BF0C37BD465DF897
:10220000047B704780B483B000AF78600B467B805E
:1022100000BF0C37BD465DF8047B704780B588B0C1
:1022200000AF78600023BB777B685B68994A934274
:1022300004D940F639319848F6F7B5F87B689B68C1
:10224000002B09D07B689B68B3F5805F04D040F613
:102250003A319148F6F7A7F87B68DB68B3F5805F01
:1022600012D07B68DB68002B0ED07B68DB68B3F58F
:10227000405F09D07B68DB68B3F5005F04D040F6AF
:102280003B318548F6F78FF87B681B6A002B09D035
:102290007B681B6AB3F5006F04D040F63C317E4882
:1022A000F6F781F87B681B69002B0ED07B681B69F1
:1022B000B3F5806F09D07B681B69B3F5C06F04D09C
:1022C00040F63E317448F6F76EF87B685B6923F0A0
:1022D0000C03002B03D17B685B69002B04D140F613
:1022E0003F316D48F6F75FF87B689B69002B13D090
:1022F0007B689B69B3F5807F0ED07B689B69B3F5E3
:10230000007F09D07B689B69B3F5407F04D04FF410
:1023100034616148F6F747F87B68DB69002B09D028
:102320007B68DB69B3F5004F04D040F641315A4871
:10233000F6F739F87B689A687B681B691A437B68F3
:102340005B691A437B68DB6913437B617B681B68AD
:102350001B6823F4164323F00C037A68126879692A
:102360000B4313607B681B685B6823F440517B68F8
:10237000DA687B681B680A435A607B689B697B61EB
:102380007B681B6A7A6913437B617B681B689B6867
:1023900023F430617B681B687A690A439A607B6822
:1023A0001B683E4A934220D13D4B1B6B03F0030355
:1023B000032B17D801A252F823F000BFCD23010848
:1023C000D9230108DF230108D32301080123FB7768
:1023D000C2E00223FB77BFE00423FB77BCE00823C5
:1023E000FB77B9E01023FB77B6E07B681B682D4ACA
:1023F000934224D12A4B1B6B03F44033B3F5403F87
:1024000011D0B3F5403F17D8B3F5003F11D0B3F565
:10241000003F11D8002B03D0B3F5803F06D00BE06E
:102420000023FB7798E00223FB7795E00423FB77FA
:1024300092E00823FB778FE01023FB778CE07B682A
:102440001B68194A934231D1154B1B6B03F440238F
:10245000B3F5402F11D0B3F5402F17D8B3F5002FA7
:1024600011D0B3F5002F11D8002B03D0B3F5802F76
:1024700006D00BE00023FB776EE00223FB776BE0D6
:102480000423FB7768E00823FB7765E01023FB77E4
:1024900062E000BF40548900449E020800380140B9
:1024A0000010024000440040004800407B681B6868
:1024B000864A934224D1864B1B6B03F44013B3F539
:1024C000401F11D0B3F5401F17D8B3F5001F11D02E
:1024D000B3F5001F11D8002B03D0B3F5801F06D031
:1024E0000BE00023FB7737E00223FB7734E0042383
:1024F000FB7731E00823FB772EE01023FB772BE0FE
:102500007B681B68734A934224D1714B1B6B03F4A5
:102510004003B3F5400F11D0B3F5400F17D8B3F512
:10252000000F11D0B3F5000F11D8002B03D0B3F575
:10253000800F06D00BE00023FB770DE00223FB7732
:102540000AE00423FB7707E00823FB7704E010236D
:10255000FB7701E01023FB777B68DB69B3F5004F65
:102560005BD1FB7F082B28D801A252F823F000BFD3
:10257000952501089D250108A5250108BB25010811
:10258000AB250108BB250108BB250108BB250108B7
:10259000B3250108FCF790FBB86113E0FCF7AEFB34
:1025A000B8610FE04C4BBB610CE0FCF725FBB86158
:1025B00008E04FF40043BB6104E00023BB6101234A
:1025C000BB7700BFBB69002B74D0BB695A007B6826
:1025D0005B685B081A447B685B68B2FBF3F33B61A2
:1025E0003B690F2B16D93B69B3F5803F12D23B698B
:1025F0009BB223F00F03FB813B695B089BB203F0A6
:1026000007039AB2FB891343FB817B681B68FA8935
:10261000DA604FE00123BB774CE0FB7F082B28D822
:1026200001A252F823F000BF4D26010855260108EB
:102630005D26010873260108632601087326010838
:1026400073260108732601086B260108FCF734FB8A
:10265000B86113E0FCF752FBB8610FE01E4BBB61A1
:102660000CE0FCF7C9FAB86108E04FF40043BB6125
:1026700004E00023BB610123BB7700BFBB69002BD3
:1026800018D07B685B685A08BB691A447B685B6832
:10269000B2FBF3F33B613B690F2B09D93B69B3F5FF
:1026A000803F05D23B699AB27B681B68DA6001E023
:1026B0000123BB777B6800229A667B680022DA667A
:1026C000BB7F18462037BD4680BD00BF004C004090
:1026D000001002400050004000127A0080B582B025
:1026E00000AF78607B685B6AFF2B04D940F6C2318B
:1026F0009648F5F758FE7B685B6A03F00803002BE9
:1027000018D07B685B6B002B09D07B685B6BB3F5E3
:10271000004F04D040F6C7318C48F5F744FE7B6883
:102720001B685B6823F400417B685A6B7B681B68FD
:102730000A435A607B685B6A03F00103002B18D0E0
:102740007B689B6A002B09D07B689B6AB3F5003FCE
:1027500004D040F6CE317D48F5F725FE7B681B6836
:102760005B6823F400317B689A6A7B681B680A43C4
:102770005A607B685B6A03F00203002B18D07B6809
:10278000DB6A002B09D07B68DB6AB3F5803F04D09D
:1027900040F6D5316D48F5F706FE7B681B685B682F
:1027A00023F480317B68DA6A7B681B680A435A60CD
:1027B0007B685B6A03F00403002B18D07B681B6BFB
:1027C000002B09D07B681B6BB3F5802F04D040F63B
:1027D000DC315E48F5F7E7FD7B681B685B6823F436
:1027E00080217B681A6B7B681B680A435A607B6890
:1027F0005B6A03F01003002B18D07B689B6B002BE7
:1028000009D07B689B6BB3F5805F04D040F6E33161
:102810004E48F5F7C8FD7B681B689B6823F4805120
:102820007B689A6B7B681B680A439A607B685B6A6B
:1028300003F02003002B18D07B68DB6B002B09D042
:102840007B68DB6BB3F5005F04D040F6EA313F48AC
:10285000F5F7A9FD7B681B689B6823F400517B6832
:10286000DA6B7B681B680A439A607B685B6A03F0DB
:102870004003002B54D07B681B68354A93420ED02E
:102880007B681B68334A934209D07B681B68324AD5
:10289000934204D040F6F1312C48F5F784FD7B6873
:1028A0001B6C002B09D07B681B6CB3F5801F04D018
:1028B00040F6F2312548F5F776FD7B681B685B68CA
:1028C00023F480117B681A6C7B681B680A435A608A
:1028D0007B681B6CB3F5801F22D17B685B6C002B7F
:1028E00013D07B685B6CB3F5001F0ED07B685B6C0C
:1028F000B3F5800F09D07B685B6CB3F5C00F04D0D3
:1029000040F6F7311148F5F74EFD7B681B685B68B0
:1029100023F4C0017B685A6C7B681B680A435A60C9
:102920007B685B6A03F08003002B22D07B689B6C82
:10293000002B13D07B689B6CB3F5002F0ED040F6B4
:10294000FF310248F5F72FFD08E000BF449E020862
:102950000038014000440040004800407B681B688C
:102960005B6823F400217B689A6C7B681B680A43D0
:102970005A6000BF0837BD4680BD00BF80B598B023
:1029800002AF78607B680022C3F88420FAF72EFD3E
:1029900078657B681B681B6803F00803082B2ED141
:1029A0006FF07E4300937B6D00224FF40011786836
:1029B00000F08CF80346002B21D07B681B68BB63BA
:1029C000BB6B53E8003F7B637B6B23F080033B656D
:1029D0007B681B681A463B6D7B643A64396C7A6C81
:1029E00041E80023FB63FB6B002BE6D17B682022D0
:1029F000DA677B68002283F87820032362E07B6833
:102A00001B681B6803F00403042B49D16FF07E435D
:102A100000937B6D00224FF48001786800F056F837
:102A20000346002B3CD07B681B687B627B6A53E8C3
:102A3000003F3B623B6A23F49073FB647B681B6836
:102A40001A46FB6C3B63FA62F96A3A6B41E8002371
:102A5000BB62BB6A002BE6D17B681B6808333B6115
:102A60003B6953E8003FFB60FB6823F00103BB6454
:102A70007B681B680833BA6CFA61BB61B969FA6993
:102A800041E800237B617B69002BE5D17B68202234
:102A9000C3F880207B68002283F87820032311E0AC
:102AA0007B682022DA677B682022C3F880207B685D
:102AB00000221A667B6800225A667B68002283F82F
:102AC0007820002318465837BD4680BD80B584B0B5
:102AD00000AFF860B9603B601346FB714FE0BB6923
:102AE000B3F1FF3F4BD0FAF781FC02463B68D31AA3
:102AF000BA699A4202D3BB69002B01D103234EE08D
:102B0000FB681B681B6803F00403002B37D0BB680D
:102B1000802B34D0BB68402B31D0FB681B68DB694D
:102B200003F00803082B10D1FB681B6808221A6207
:102B3000F86800F0FFF8FB680822C3F88420FB68FF
:102B4000002283F87820012329E0FB681B68DB69F9
:102B500003F40063B3F5006F11D1FB681B684FF4F9
:102B600000621A62F86800F0E5F8FB682022C3F8FA
:102B70008420FB68002283F8782003230FE0FB68A1
:102B80001B68DA69BB681340BA689A420CBF01231C
:102B90000023DBB21A46FB799A42A0D000231846E4
:102BA0001037BD4680BD000080B596B000AFF8601C
:102BB000B9601346FB80FB68BA685A65FB68FA88FF
:102BC000A3F85820FB680022C3F88420FB68222267
:102BD000C3F88020FB685B6F002B28D0FB685B6F1D
:102BE0003E4A9A62FB685B6F3D4ADA62FB685B6F44
:102BF0003C4A1A63FB685B6F00225A63FB68586F9C
:102C0000FB681B6824331946FB685B6D1A46FB881A
:102C1000FCF780FF0346002B09D0FB681022C3F8A5
:102C20008420FB682022C3F88020012351E0FB6848
:102C30001B69002B18D0FB681B68FB63FB6B53E818
:102C4000003FBB63BB6B43F480737B65FB681B6811
:102C50001A467B6DBB647A64796CBA6C41E80023D8
:102C60003B643B6C002BE6D1FB681B680833BB62FE
:102C7000BB6A53E8003F7B627B6A43F001033B651C
:102C8000FB681B6808333A6D7A633B63396B7A6B78
:102C900041E80023FB62FB6A002BE5D1FB681B685F
:102CA00008337B617B6953E8003F3B613B6943F03C
:102CB0004003FB64FB681B680833FA6C3A62FB61F3
:102CC000F9693A6A41E80023BB61BB69002BE5D191
:102CD000002318465837BD4680BD00BFAD2E010801
:102CE000D32F01081130010880B489B000AF78609B
:102CF0007B681B68FB60FB6853E8003FBB60BB68F8
:102D000023F0C003FB617B681B681A46FB69BB614B
:102D10007A617969BA6941E800233B613B69002B1C
:102D2000E6D17B682022DA6700BF2437BD465DF814
:102D3000047B704780B495B000AF78607B681B68F7
:102D40007B637B6B53E8003F3B633B6B23F49073E7
:102D5000FB647B681B681A46FB6C3B64FA63F96B87
:102D60003A6C41E80023BB63BB6B002BE6D17B6868
:102D70001B6808333B623B6A53E8003FFB61FB6919
:102D800023F00103BB647B681B680833BA6CFA62EA
:102D9000BB62B96AFA6A41E800237B627B6A002B56
:102DA000E5D17B681B6E012B18D17B681B68FB602B
:102DB000FB6853E8003FBB60BB6823F010037B64F3
:102DC0007B681B681A467B6CBB617A617969BA695A
:102DD00041E800233B613B69002BE6D17B68202260
:102DE000C3F880207B6800221A667B6800229A66FE
:102DF00000BF5437BD465DF8047B704780B590B086
:102E000000AF78607B685B6AFB637B689B69202B03
:102E100037D0FB6B0022A3F85220FB6B1B680833F2
:102E20007B627B6A53E8003F3B623B6A23F080038E
:102E3000BB63FB6B1B680833BA6B3A63FB62F96ACE
:102E40003A6B41E80023BB62BB6A002BE5D1FB6B08
:102E50001B683B613B6953E8003FFB60FB6843F044
:102E600040037B63FB6B1B681A467B6BFB61BA619B
:102E7000B969FA6941E800237B617B69002BE6D1DF
:102E800002E0F86B00F022FB00BF4037BD4680BD7A
:102E900080B584B000AF78607B685B6AFB60F868DF
:102EA000FFF792F900BF1037BD4680BD80B59CB0DA
:102EB00000AF78607B685B6AFB667B689B69202B50
:102EC00071D0FB6E0022A3F85A20FB6E1B68FB64D6
:102ED000FB6C53E8003FBB64BB6C23F48073BB66A0
:102EE000FB6E1B681A46BB6EBB657A65796DBA6D61
:102EF00041E800233B653B6D002BE6D1FB6E1B6870
:102F00000833BB63BB6B53E8003F7B637B6B23F0F1
:102F100001037B66FB6E1B6808337A6E7A643B6440
:102F2000396C7A6C41E80023FB63FB6B002BE5D125
:102F3000FB6E1B6808337B627B6A53E8003F3B6291
:102F40003B6A23F040033B66FB6E1B6808333A6E16
:102F50003A63FB62F96A3A6B41E80023BB62BB6AE1
:102F6000002BE5D1FB6E2022C3F88020FB6E1B6E88
:102F7000012B18D1FB6E1B683B613B6953E8003F96
:102F8000FB60FB6823F01003FB65FB6E1B681A46B1
:102F9000FB6DFB61BA61B969FA6941E800237B61A5
:102FA0007B69002BE6D1FB6E00225A66FB6E1B6E1E
:102FB000012B07D1FB6EB3F858301946F86EFFF7B6
:102FC00021F902E0F86EFFF709F900BF7037BD463E
:102FD00080BD80B584B000AF78607B685B6AFB60C1
:102FE000FB6801225A66FB681B6E012B09D1FB6846
:102FF000B3F858305B089BB21946F868FFF702F93E
:1030000002E0F868FFF7F4F800BF1037BD4680BD56
:1030100080B586B000AF78607B685B6A7B617B6956
:10302000DB6F3B617B69D3F88030FB607B691B6899
:103030009B6803F08003802B09D13B69212B06D1CB
:103040007B690022A3F852207869FFF74DFE7B6967
:103050001B689B6803F04003402B09D1FB68222BBF
:1030600006D17B690022A3F85A207869FFF762FE37
:103070007B69D3F8843043F010027B69C3F8842065
:10308000786900F0E5F900BF1837BD4680BD80B50E
:1030900084B000AF78607B685B6AFB60FB680022ED
:1030A000A3F85A20FB680022A3F85220F86800F029
:1030B000CFF900BF1037BD4680BD80B588B000AFE6
:1030C00078607B681B68FB60FB6853E8003FBB606F
:1030D000BB6823F04003FB617B681B681A46FB69F1
:1030E000BB617A617969BA6941E800233B613B6958
:1030F000002BE6D17B682022DA677B680022DA6643
:10310000786800F0E3F900BF2037BD4680BD80B489
:1031100083B000AF786000BF0C37BD465DF8047B1C
:103120007047000080B400AF064BD3F88830054AE2
:1031300043F47003C2F8883000BFBD465DF8047BDD
:10314000704700BF00ED00E080B582B000AF0346DD
:10315000FB71FB79022B1DD1214BDB6F202B0DD195
:103160001F4B1B68DB6903F04003402B06D11C4B4F
:103170001B68DB6903F08003802B01D000232BE068
:10318000FAF734F90246174B1B68D31A012B22D8E1
:10319000002321E0FB79032B1DD1134BDB6F202B88
:1031A0000DD1114B1B68DB6903F04003402B06D1A6
:1031B0000D4B1B68DB6903F08003802B01D00023DB
:1031C0000AE0FAF713F90246084B1B68D31A012BE1
:1031D00001D8002300E0012318460837BD4680BD12
:1031E00098070020E40A002020080020E80A0020B8
:1031F00080B582B000AF78600B46FB70FB781A4652
:103200007968034808F075FB00BF0837BD4680BDEC
:10321000C80A002080B582B000AF0023FB800220E6
:10322000FFF792FF0346002B15D04FF480720C4934
:103230000C4808F0ECFB0346FB80FB88002B0AD00F
:10324000FB881A4606490848FEF768FBFAF7CEF8ED
:103250000346064A136000BF0837BD4680BD00BF65
:10326000EC0A0020C80A002098070020E40A002089
:1032700080B582B000AF78600B46FB70FAF7B6F805
:1032800003460D4A136000BFFAF7B0F802460A4B36
:103290001B68D31A012BF7D9FB789BB21A467968C1
:1032A0000648FEF73BFBFAF7A1F80346044A136011
:1032B00000BF0837BD4680BD140D00202008002047
:1032C000E80A002080B500AF164B1B681A68154B42
:1032D0001B6842F010021A604FF4807212491148C4
:1032E000FEF798FB0F4B1B689A680E4B1B6842F069
:1032F00001029A600D4B1B681A680C4B1B6842F068
:1033000010021A604FF4807209490848FEF782FBE8
:10331000064B1B689A68054B1B6842F001029A60D5
:1033200000BF80BD980700200E000020200800206C
:10333000A400002080B582B000AF78607B683C4A72
:10334000934225D13A4B1B68DB6903F01003102B25
:103350001ED1374B1B6810221A623548FEF79EFBC0
:103360007B685B6F1B685B68DBB25B42DAB2314B38
:1033700083F818212F4B93F818311A462E492F48FD
:1033800008F0B7FA4FF480722B492948FEF742FB48
:103390007B682B4A934246D1294B1B68DB6903F0BB
:1033A0001003102B3FD1264B1B6810221A622448B1
:1033B000FEF774FB7B685B6F1B685B68DBB25B428C
:1033C000DAB21C4B83F818211E4B1B7A002B08D055
:1033D000184B93F818319BB219461B4801F08AFE2E
:1033E0001CE01A4B1B7A002B08D0124B93F81831B3
:1033F0009BB21946144801F0C1FE0FE00D4B93F843
:1034000018319BB21946104801F0B8FE094B93F8E9
:1034100018319BB219460C4801F06CFE80220A4913
:103420000748FEF7F7FA00BF0837BD4680BD00BF6A
:10343000980700200C0000200E000020EC0B00205C
:103440002008002000100020A40000200C10002004
:1034500080B582B000AF78607B681B68DB6903F0E1
:103460000803082B03D17B681B6808221A627B685B
:103470001B68DB6903F02003202B03D17B681B68EA
:1034800020221A627B681B6801221A627B680B4A41
:10349000934206D14FF4807209490848FEF7BAFA00
:1034A00008E07B68074A934204D180220649054818
:1034B000FEF7B0FA00BF0837BD4680BD9807002070
:1034C0000E00002020080020A400002080B483B05B
:1034D00000AF786000BF0C37BD465DF8047B7047D5
:1034E00080B584B000AF78600023FB73C9E1844BE2
:1034F0001B78002B0AD0F9F779FF0246814B1B6835
:10350000D31AC82B02D97E4B00221A707C4B1B7831
:10351000082B00F2AB8101A252F823F041350108DB
:103520005F3501086D3501087B35010895350108C7
:10353000CF350108E33501082B360108553601085F
:10354000714B1A78FB7B9A4240F09481F9F74EFF59
:1035500003466C4A13606A4B01221A708AE1FA7BB7
:10356000694B5A70664B02221A7086E1FA7B664BF1
:103570009A70634B03221A707FE1634BDA78FB7B0E
:103580009A4203D15E4B04221A7076E15C4B002212
:103590001A7072E1FB7B002B0ED0FB7BCC2B0BD087
:1035A000FB7B332B08D0FB7B342B05D0FB7B382BEC
:1035B00002D0FB7BDE2B06D1FA7B534B1A71504BAA
:1035C00005221A7059E14E4B00221A7055E1FA7B20
:1035D0004D4B5A714A4B06221A704C4B00221A70FE
:1035E0004BE1494B9B791A46484B1B781344F97BB6
:1035F000454A13440A469A72444B1B780133DAB2A7
:10360000424B1A70404B5A78404B1B789A4203D178
:103610003B4B07221A702FE13B4B5B78002B40F0AD
:103620002B81374B08221A7026E1374B9B791A46BB
:10363000364B1B781344F97B334A13440A469A727B
:10364000324B1B780133DAB2304B1A702C4B082204
:103650001A7012E12C4B9B791A462C4B1B781344A1
:10366000F97B294A13440A469A72274B1A78264B4B
:103670009A72254B5A78244BDA72234B9A78224B54
:103680001A73214BDA78204B5A731F4B1A791E4B51
:103690009A731D4B5A791C4BDA731B4B5B789AB2A9
:1036A000194B9B799BB213449AB2174BDB799BB2AF
:1036B00013449BB21946164801F06AFC0346002BDE
:1036C00040F0D080104B1B79002B03D00E4B1B79A0
:1036D000CC2B25D10C4B5A790E4B5A710A4B5B7887
:1036E0001A46094B9B791344074AD27913441A4668
:1036F0000749094813F038FD084B01221A70B1E060
:10370000040C0020180D0020340100201C0D0020A6
:103710003E010020080C0020120C00200C000020AC
:10372000604B1B79332B03D15F4B1B7A002B0FD1DE
:103730005C4B1B79342B03D15C4B1B7A002B07D1DC
:10374000584B1B79382B3BD1594B1B7A002B37D068
:10375000584B5B7883F00103DBB2002B21D0F9F7E3
:1037600045FE0346534AC2F819314E4B5B781A4660
:103770004C4B9B7913444B4AD27913441A464E4919
:103780004E4813F0F1FC4B4B01225A70454B5B79CC
:10379000C82B66D14A4B01221A704A4B00221A608C
:1037A0005FE0F9F723FE0246424BD3F81931D31AF2
:1037B00040F6B832934254D93E4B00225A7050E042
:1037C000384B1B79DE2B0BD0364B1B79332B07D0B4
:1037D000344B1B79342B03D0324B1B79382B41D11E
:1037E000304B5B79C82B12D140F2271200213148AF
:1037F00013F0C8FC2B4B1B692E4AC2F820312D4B0D
:103800000122A3F81E212B4B012283F81D21254BF9
:103810005B781A46234B9B791344224AD27913448E
:103820001A462549254813F09FFC224BB3F81E3158
:103830001A46224B9B791946204BDB791B020B441D
:103840009A420ADD174B5B79C92B06D11B4B1B79BA
:103850001D4AC921184608F0F1F8164B01225A708A
:1038600000E000BF194B00221A7006E0174B00223F
:103870001A7002E000BF00E000BF0E4B1B78002B67
:103880000BD107F10F0301221946786808F0BFF841
:103890000346002B7FF42BAE00E000BF00BF1037C3
:1038A000BD4680BD34010020BC040020040500207A
:1038B000600300200C0000203E010020300A0020A0
:1038C000E00A0020A4260020360A0020040C002074
:1038D00080B58AB008AF7A23AB4A41F28831AB4851
:1038E0000DF0E4FC7A23AA4A41F28831A9480DF090
:1038F000DDFC4623A84A41F28831A8480DF0D6FCE9
:103900004623A74A41F28831A6480DF0CFFC3E235A
:10391000A54A41F28831A5480DF0C8FC40F24D138C
:10392000A34A41F28831A2480DF0C0FC40F24D1389
:10393000A04A41F288319F480DF0B8FC9E4B93F8A5
:10394000D730012B05D09D4B93F8D730012B40F099
:1039500039839B4B012283F8E021974B93F8D730B2
:10396000012B40F09081944BB3F840319AB2954BC3
:10397000A3F85920904BB3F8F8309BB2112B07D91C
:103980008D4BB3F8EC309AB28E4BA3F85B200BE072
:10399000894BB3F8EC309BB28B4AA2FB0323DB08C4
:1039A0009AB2884BA3F85B20834BB3F8F0309BB2FC
:1039B0001AB2844BA3F85F207F4BB3F8F2309BB26E
:1039C000DAB2804B83F861207B4BB3F8F6309BB2C0
:1039D0001B0A9BB2052B06D0774BB3F8F6309BB28F
:1039E0001B0A9BB200E00023764AA2F86230724BB9
:1039F000B3F8F8309BB2DAB2724B1A716E4BB3F86F
:103A0000FA309AB26F4BA3F805206B4BB3F8FC3039
:103A10009AB26C4BA3F80720674BB3F8FE309AB20A
:103A2000684BA3F80920644BB3F800319AB2654B98
:103A3000A3F80B20604BB3F802319AB2614BA3F8A4
:103A40000D205D4BB3F804319AB25E4BA3F80F2002
:103A5000594BB3F806319AB25A4BA3F81120564B82
:103A6000B3F808319AB2574BA3F81320524BB3F86E
:103A70000A319AB2534BA3F815204F4BB3F80C31CF
:103A80009AB2504BA3F817204B4BB3F80E319AB2B1
:103A90004C4BA3F81920484BB3F810319AB2494B5C
:103AA000A3F81B20444BB3F812319AB2454BA3F84C
:103AB0001D20414BB3F814319AB2424BA3F81F209A
:103AC0003D4BB3F816319AB23E4BA3F821203A4B46
:103AD000B3F818319AB23B4BA3F82320364BB3F816
:103AE0001A319AB2374BA3F82520334BB3F81C3167
:103AF0009AB2344BA3F827202F4BB3F81E319AB259
:103B0000304BA3F829202C4BB3F820319AB22D4B1F
:103B1000A3F82B20284BB3F822319AB2294BA3F8F3
:103B20002D20254BB3F824319AB2264BA3F82F2031
:103B3000214BB3F826319AB2224BA3F831201E4B09
:103B4000B3F828319AB21F4BA3F833201A4BB3F8BD
:103B50002A319AB21B4BA3F83520174BB3F82C31FE
:103B60009AB2184BA3F83720134B93F85621154BF4
:103B700083F83920104B93F85721124B83F83A20E1
:103B800001237B6049E000BF342400201B24002077
:103B9000982500207F250020641200205412002068
:103BA0008813002078130020B43A0020F43A002053
:103BB000200D0020700E00204C230020B024002097
:103BC000903B002040020020CDCCCCCC7B68013360
:103BD000524A134493F856311B09DAB27B685B00F2
:103BE0003032D1B24E4A13440A4683F839207B68FA
:103BF00001334A4A134493F8563103F00F03DAB203
:103C00007B685B0001333032D1B2454A13440A4627
:103C100083F839207B6801337B607B680A2BD5DD14
:103C20003E4BB3F8EE309BB21AB23D4BA3F85D2089
:103C30003B4B0F22A3F8642020213A480DF0A2FB51
:103C4000034683F00103DBB2002B21D0364B93F8FF
:103C5000543083F00103DBB2002B19D00823069304
:103C6000324B059300230493002303930023029314
:103C700000230193202300932A4B00220E212A487F
:103C80000EF028F804E066220021254813F07AFAA5
:103C9000274B93F8D730012B40F08081244BB3F8A9
:103CA00040319AB2234BA3F85920214BB3F8F83096
:103CB0009BB2112B07D91E4BB3F8EC309AB21D4BB7
:103CC000A3F85B200BE01A4BB3F8EC309BB21A4A16
:103CD000A2FB0323DB089AB2164BA3F85B20144B1C
:103CE000B3F8F0309BB21AB2124BA3F85F20104B1E
:103CF000B3F8F2309BB2DAB20E4B83F861200C4B72
:103D0000B3F8F6309BB21B0A9BB2052B16D0084BBA
:103D1000B3F8F6309BB21B0A9BB210E04C23002094
:103D20004002002079020020B83F00207C9E02085B
:103D3000B0240020A8020020CDCCCCCC00239B4A8C
:103D4000A2F862309A4BB3F8F8309BB2DAB2974BD4
:103D50001A71974BB3F8FA309AB2944BA3F8052036
:103D6000934BB3F8FC309AB2904BA3F80720904BDA
:103D7000B3F8FE309AB28D4BA3F809208C4BB3F800
:103D800000319AB2894BA3F80B20894BB3F802316A
:103D90009AB2864BA3F80D20854BB3F804319AB242
:103DA000824BA3F80F20824BB3F806319AB27F4BB7
:103DB000A3F811207E4BB3F808319AB27B4BA3F8DD
:103DC00013207B4BB3F80A319AB2784BA3F8152035
:103DD000774BB3F80C319AB2744BA3F81720744B9D
:103DE000B3F80E319AB2714BA3F81920704BB3F8A7
:103DF00010319AB26D4BA3F81B206D4BB3F8123102
:103E00009AB26A4BA3F81D20694BB3F814319AB2E9
:103E1000664BA3F81F20664BB3F816319AB2634B7A
:103E2000A3F82120624BB3F818319AB25F4BA3F884
:103E300023205F4BB3F81A319AB25C4BA3F82520CC
:103E40005B4BB3F81C319AB2584BA3F82720584B60
:103E5000B3F81E319AB2554BA3F82920544BB3F84E
:103E600020319AB2514BA3F82B20514BB3F8223199
:103E70009AB24E4BA3F82D204D4BB3F824319AB291
:103E80004A4BA3F82F204A4BB3F826319AB2474B3E
:103E9000A3F83120464BB3F828319AB2434BA3F82C
:103EA0003320434BB3F82A319AB2404BA3F8352064
:103EB0003F4BB3F82C319AB23C4BA3F837203D4B23
:103EC00093F85621394B83F839203A4B93F8572110
:103ED000364B83F83A2001233B6026E03B680133F0
:103EE000334A134493F856311B09DAB23B685B003E
:103EF0003032D1B22D4A13440A4683F839203B6848
:103F000001332B4A134493F8563103F00F03DAB20E
:103F10003B685B0001333032D1B2244A13440A4675
:103F200083F839203B6801333B603B680A2BD5DDC1
:103F30001F4BB3F8EE309BB21AB21C4BA3F85D20B6
:103F40001A4B0F22A3F8642020211B480DF01AFA07
:103F5000034683F00103DBB2002B00F06A84174BA9
:103F600093F8543083F00103DBB2002B00F061843E
:103F700008230693124B0593002304930023039315
:103F80000023029300230193202300930A4B002275
:103F90000F210A480DF09EFE00F04BBC6622002166
:103FA000024813F0EFF800F044BC00BFA802002064
:103FB000B02400204C230020E10200201440002007
:103FC000849E0208714B93F8D430012B05D0704BBE
:103FD00093F8D430012B40F0E1816E4B012283F83D
:103FE000E0216A4B93F8D430012B40F0E3806A4B18
:103FF00001221A70654BB3F8E8309AB2674BA3F808
:104000005920624BB3F8E0309BB2654AA2FB032310
:10401000DB089AB2614BA3F85B205C4BB3F8E43049
:104020009BB21A46920013445B009BB21AB25B4BE0
:10403000A3F85F20554BB3F8E6309BB2DAB2574B8A
:1040400083F86120554B0022A3F862204F4BB3F850
:1040500020319BB2DAB2514B1A714C4BB3F8EC30B1
:104060009AB24E4BA3F80520484BB3F8EE309AB203
:104070004A4BA3F80720454BB3F8F0309AB2474BB0
:10408000A3F80920414BB3F8F2309AB2434BA3F89E
:104090000B203E4BB3F8F4309AB2404BA3F80D20FE
:1040A0003A4BB3F8F6309AB23C4BA3F80F20374B9B
:1040B000B3F8F8309AB2394BA3F81120334BB3F868
:1040C000FA309AB2354BA3F81320304BB3F8FC30DA
:1040D0009AB2324BA3F815202C4BB3F8FE309AB2AB
:1040E0002E4BA3F81720294BB3F800319AB22B4B73
:1040F000A3F81920254BB3F802319AB2274BA3F845
:104100001B20224BB3F804319AB2244BA3F81D2094
:104110001E4BB3F806319AB2204BA3F81F20102291
:104120002049214813F020F8184BB3F9E2301AB2B5
:104130001A4BA3F85D20194B0B22A3F86420202111
:1041400019480DF01FF9034683F00103DBB2002B81
:1041500035D0164B93F8543083F00103DBB2002BBB
:104160002DD007230693124B0593002304930023BD
:1041700003930023029300230193102300930A4B1F
:1041800000220E2109480DF0A5FD18E0881100203D
:10419000AC120020903B002035230020400200207C
:1041A000CDCCCCCC9812002079020020B83F002062
:1041B0008C9E0208662200216F4812F0E3FF6F4BCD
:1041C00093F8D430012B40F0D1806D4B02221A704D
:1041D0006A4BB3F8E8309AB26A4BA3F85920674BA0
:1041E000B3F8E0309BB2684AA2FB0323DB089AB223
:1041F000644BA3F85B20614BB3F8E4309BB21A46E2
:10420000920013445B009BB21AB25E4BA3F85F208E
:104210005A4BB3F8E6309BB2DAB25A4B83F86120BE
:10422000584B0022A3F86220544BB3F820319BB2C4
:10423000DAB2544B1A71514BB3F8EC309AB2514B7D
:10424000A3F805204D4BB3F8EE309AB24D4BA3F8CE
:1042500007204A4BB3F8F0309AB24A4BA3F8092032
:10426000464BB3F8F2309AB2464BA3F80B20434BBF
:10427000B3F8F4309AB2434BA3F80D203F4BB3F898
:10428000F6309AB23F4BA3F80F203C4BB3F8F8300E
:104290009AB23C4BA3F81120384BB3F8FA309AB2DB
:1042A000384BA3F81320354BB3F8FC309AB2354B9A
:1042B000A3F81520314BB3F8FE309AB2314BA3F876
:1042C00017202E4BB3F800319AB22E4BA3F81920C9
:1042D0002A4BB3F802319AB22A4BA3F81B20274B82
:1042E000B3F804319AB2274BA3F81D20234BB3F83F
:1042F00006319AB2234BA3F81F20102223492448E9
:1043000012F032FF1D4BB3F9E2301AB21D4BA3F885
:104310005D201C4B0B22A3F8642020211C480DF0CB
:1043200031F8034683F00103DBB2002B00F08382F7
:10433000184B93F8543083F00103DBB2002B00F0EC
:104340007A8207230693144B0593002304930023DA
:1043500003930023029300230193102300930C4B3B
:1043600000220F210B480DF0B5FC64E2662200210B
:10437000044812F007FF5EE240020020AC12002069
:1043800035230020A8020020CDCCCCCCBC130020CB
:10439000E102002014400020949E02086D4B1B7A1D
:1043A000012B40F0E9806C4B012283F8E0216B4B3C
:1043B00001221A706A4BB3F833309AB2694BA3F8F2
:1043C0005920674BB3F823309AB2664BA3F85B20B1
:1043D000634B93F83D30002B18D0614B1B781A4685
:1043E0005F4B5B7813445E4A927813445E4A82FBCB
:1043F0000312DB17D31A283B9BB21A4692001344D0
:104400005B009BB21AB2574BA3F85F20544B93F852
:104410002720544B83F86120514BB3F821309AB2D6
:10442000504BA3F862204E4B93F832204D4B1A713B
:104430004B4BB3F803309AB24A4BA3F80520484BD4
:10444000B3F805309AB2474BA3F80720444BB3F8B2
:1044500007309AB2434BA3F80920414BB3F8093017
:104460009AB2404BA3F80B203D4BB3F80B309AB2F5
:104470003C4BA3F80D203A4BB3F80D309AB2394BB0
:10448000A3F80F20364BB3F80F309AB2354BA3F890
:104490001120334BB3F811309AB2324BA3F81320EA
:1044A0002F4BB3F813309AB22E4BA3F815202C4B98
:1044B000B3F815309AB22B4BA3F81720284BB3F85A
:1044C00017309AB2274BA3F81920254BB3F81930AF
:1044D0009AB2244BA3F81B20214BB3F81B309AB29D
:1044E000204BA3F81D201E4BB3F81D309AB21D4B74
:1044F000A3F81F2007221D491D4812F035FE184B56
:10450000B3F825309BB21AB2164BA3F85D20154BB9
:104510000E22A3F86420174B93F8533083F0010365
:10452000DBB2002B00F08A81082306930F4B059322
:104530000023049300230393002302930023019399
:1045400000230093002300220E210A480DF0C2FB35
:1045500074E100BFF43A0020903B00203523002096
:10456000B43A002040020020565555559C9E020842
:1045700079020020B83F0020B24B1B7A012B04D0F7
:10458000B14B1B7A012B40F04681B04B012283F8DE
:10459000E021AC4B1B7A012B40F09680AC4B012202
:1045A0001A70A84BB3F83621AA4BA3F85920A54B93
:1045B000B3F89620A74BA3F85B20A24BB3F99C203D
:1045C000A44BA3F85F209F4BB3F8A030A24AA2FBF4
:1045D0000323DB089BB2DAB29E4B83F86120994B30
:1045E000D3F8A2309AB29B4BA3F86220954BB3F854
:1045F000A630DAB2974B1A7134229849984812F0D3
:10460000B3FD14229749984812F0AEFD8D4BD3F8B4
:104610009830964A82FB03129210DB17D31A1AB213
:104620008C4BA3F85D208B4B0A22A3F86420202139
:104630008D480CF0A7FE034683F00103DBB2002B8C
:104640001BD08B4B93F8543083F00103DBB2002B6B
:1046500013D0002306930023059300230493002323
:1046600003930023029300230193202300937E4BA6
:1046700000220E217E480DF02DFB14217D480CF008
:1046800081FE034683F00103DBB2002B22D0784B7E
:1046900093F8573083F00103DBB2002B1AD01023BC
:1046A0000693744B05930023049300230393002384
:1046B00002930023019300230093002300220E2184
:1046C0006B480DF007FB05E040F24D1200215D48FC
:1046D00012F058FD5C4B1B7A012B40F096805C4B2E
:1046E00002221A70584BB3F83621634BA3F85920B5
:1046F000554BB3F89620604BA3F85B20524BB3F9AF
:104700009C205D4BA3F85F204F4BB3F8A030524A7A
:10471000A2FB0323DB089BB2DAB2574B83F861207C
:10472000494BD3F8A2309AB2534BA3F86220464BC0
:10473000B3F8A630DAB2504B1A7134224F495048C0
:1047400012F012FD14224F494F4812F00DFD3E4B5E
:10475000D3F89830454A82FB03129210DB17D31A24
:104760001AB2454BA3F85D20434B0A22A3F86420FC
:10477000202145480CF006FE034683F00103DBB21E
:10478000002B1BD0414B93F8543083F00103DBB274
:10479000002B13D0002306930023059300230493DA
:1047A000002303930023029300230193202300930B
:1047B000354B00220F2135480DF08CFA1421344876
:1047C0000CF0E0FD034683F00103DBB2002B34D094
:1047D0002E4B93F8573083F00103DBB2002B2CD023
:1047E000102306932A4B059300230493002303937D
:1047F000002302930023019300230093002300224F
:104800000F2122480DF066FA17E0662200211A48AF
:1048100012F0B8FC11E00D4B93F8E031012B0DD1F3
:104820000A4B022283F8E0210A4B0022A3F86220FF
:1048300004E000BF02E000BF00E000BF00BF083797
:10484000BD4680BD200D0020700E0020903B002052
:104850003523002040020020CDCCCCCCC80D002058
:1048600045020020240E002079020020676666665B
:10487000B83F0020FC0D0020A8020020180F0020E7
:10488000AD020020740F0020E1020020144000203F
:104890004C0F002080B586B000AF00237B61002361
:1048A0003B610023FB730023BB7300237B73002356
:1048B0007B600023BB6000237B80A74B1B78012B10
:1048C00005D1A54B02221A70A44B7B6108E0A24BD4
:1048D0001B78022B04D1A04B01221A70A04B7B61E4
:1048E0007B691B7A012B40F032817B691B7C002B9A
:1048F0001BD00123BB73BB7B1B0543F460227B6988
:104900005B7CDB02134343F039033B610223FB73FF
:1049100056233B7131237B71F97B3B1D3A69184665
:1049200005F0D0FA7B6900221A747B6993F84A314A
:1049300083F00103DBB2002B15D00023FB730323AC
:10494000BB73BB7B1B0543F460227B695B7CDB0292
:10495000134343F039033B61F97B3B1D3A69184629
:1049600005F0B0FA3AE07B6993F84B3183F001032C
:10497000DBB2002B15D00023FB730423BB73BB7B7E
:104980001B0543F460227B695B7CDB02134343F02D
:1049900039033B61F97B3B1D3A69184605F092FAF1
:1049A0001CE07B6993F84C3183F00103DBB2002BF0
:1049B00014D00023FB730523BB73BB7B1B0543F49F
:1049C00060227B695B7CDB02134343F039033B616C
:1049D000F97B3B1D3A69184605F074FA614B9B78E8
:1049E000002B53D00723BB7314215F4800F0D0FA8B
:1049F00003467B807B88BB807B7B5A4A1344D91D4E
:104A00003B1D02330622184612F0AEFBBB7B1B0592
:104A100043F460227B695B7CDB02134343F0310388
:104A20003B613B1D3A690821184605F04BFA7B7B38
:104A300006337B73BB7B1B0543F460227B695B7C85
:104A4000DB02134343F022033B617B7B454A134463
:104A500007333A690821184605F034FA7B7B08339E
:104A60007B73BB7B1B0543F460227B695B7CDB02B1
:104A7000134343F02B033B617B7B3A4A13440733D8
:104A80003A690621184605F01DFA61E0354BDB78DE
:104A9000012B15D10823BB73BB7B1B0543F460229C
:104AA0007B695B7CDB02134343F039033B610123E9
:104AB0003B713B1D3A690121184605F003FA47E0B6
:104AC0002A4B1B68002B20D0294B1B78002B1CD0B5
:104AD0000923BB73BB7B1B0543F460227B695B7CB2
:104AE000DB02134343F039033B61204B1B687B60BF
:104AF0003B1D3A690421184605F0E4F91C4B1B786C
:104B0000013BDAB21A4B1A7022E0F8F76FFC02464A
:104B1000184B1B68D31AB3F5FA7F19D90223BB735C
:104B2000BB7B1B0543F460227B695B7CDB02134388
:104B300043F039033B613B1D3A690021184605F0FB
:104B4000C1F9F8F753FC03460A4A136000E000BFBE
:104B50001837BD4680BD00BF0F030020200D002088
:104B6000700E0020C8030020CF030020883A0020E8
:104B70000E030020C00F002080B500AF64210B4859
:104B80000CF0C5FB0346002B03D0FEF7A1FEFFF798
:104B900081FEC82106480CF0BAFB0346002B03D067
:104BA00004F03CFA0AF03AF900BF80BDC40F0020BF
:104BB000C80F002080B588B000AFF860B960134618
:104BC000FB710023BB6100237B610023FB74002386
:104BD000BB7400237B740023FB61FB681B0D03F097
:104BE0003F037B61FB685B0903F03F03BB61FB682C
:104BF0001B09DBB203F00103FB74FB68DB08DBB2CB
:104C000003F00103BB74FB68DBB203F007037B74A2
:104C10009C4B1B68BA699A4203D09A4B1B68002BC5
:104C200009D1984ABB691360974BFB61BB69DAB243
:104C3000FB695A7405E0954BFB61BB69DAB2FB690D
:104C40005A74FB6901221A72F8F7D0FB0246FB691D
:104C50001A60FB7C012B0AD1BB7C012B07D1FB69BD
:104C60001633FA79B968184612F07EFAA6E0FB7C92
:104C7000012B24D1BB7C002B21D1FB6900221A75AA
:104C8000FB6902225A75FB6901229A74FB690022B2
:104C9000DA74FB691B7D1033FA6913440633FA7921
:104CA000B968184612F060FAFB691A7DFB79134463
:104CB000DAB2FB691A75764A7B6913607EE0FB699C
:104CC0009B7C002B3AD0FB7C002B37D1BB7C002B8C
:104CD00034D16F4B1B687A699A422FD1FB695B7D97
:104CE0007A7C9A4226D1FB691B7D1033FA69134402
:104CF0000633FA79B968184612F036FAFB691A7D5C
:104D0000FB791344DAB2FB691A75FB695B7D0133E9
:104D1000DAB2FB695A75FB695B7D082B02D1FB692E
:104D200001225A75FB695B7D072B46D9FB6900227E
:104D30005A7542E0FB6900229A743EE0FB7C002B2E
:104D40003CD1BB7C012B39D1FB699B7C002B35D03E
:104D50004F4B1B687A699A4230D1FB691B7D103337
:104D6000FA6913440633FA79B968184612F0FCF967
:104D7000FB691A7DFB791344DAB2FB691A75FB698A
:104D800000229A74FB6903F11802FB691B7D9BB238
:104D9000023B9BB21946104600F0FAF803461A4649
:104DA000FB699B7D1946FB69DB7D1B020B449A4224
:104DB00004D1FB690122DA7400E000BF7B69013B8A
:104DC000082B00F2AA8001A252F823F0F14D01084D
:104DD000154E0108394E0108634E0108954E010831
:104DE0001B4F0108BF4E0108EF4E01080B4F010891
:104DF000FB699B7D562B40F09280FB69DB7D312B5C
:104E000040F08D80FB6901221A74BB69DAB2FB693C
:104E10005A7484E0FB69DB7C002B00F08280FB6924
:104E200003F19600FB6918334622194612F09CF9EB
:104E3000FB690022DA7474E0FB69DB7C002B72D022
:104E4000FB6903F1DC00FB6918335022194612F0AC
:104E50008BF9FB690022DA74FB69012283F84A218D
:104E600061E0FB6903F59670FB6916330822194669
:104E700012F07AF9FB690022DA74FB69012283F8E7
:104E80004B2155E0CC0F0020200D0020700E00209B
:104E9000D00F0020FB69DB7C002B46D0FB6903F5BB
:104EA0009A70FB6918331622194612F05DF9FB69F6
:104EB0000022DA74FB69012283F84C2135E01E4B95
:104EC00000229A70FB699B7D002B06D11A4B0122B0
:104ED000DA70194B01229A7102E0174B02229A7183
:104EE000154B03225A71144B01225A7020E0124BC9
:104EF00004225A71FB699A7D0F4B9A710E4B012265
:104F00005A700D4B0022DA7012E0FB699B7D002B7A
:104F10000DD10A4B00221A7009E000BF08E000BF63
:104F200006E000BF04E000BF02E000BF00E000BFF9
:104F300000BF2037BD4680BDC80300200E030020FF
:104F400080B485B000AF786039600023FB600FE06B
:104F5000FB681A0A7B68591C79601B785340DBB2E6
:104F60000A4A32F813301A46FB681B025340FB60B2
:104F70003B685A1E3A60002BEADCFB68DB431846AC
:104F80001437BD465DF8047B704700BFAC9F020834
:104F900080B485B000AF78600B467B80FF23FB7345
:104FA000FF23BB7313E07B685A1C7A601A78BB7BC3
:104FB0005340DBB2BB600F4ABB6813441A78FB7BDB
:104FC0005340BB730C4ABB6813441B78FB737B884C
:104FD0005A1E7A80002BE6D1FB7B1B021AB2BB7BE8
:104FE0001BB213431BB29BB218461437BD465DF883
:104FF000047B7047ACA10208ACA2020880B485B063
:1050000000AF03460A46FB8013467B717B799BB257
:105010001B029AB2FB885340FB800023FB6012E026
:10502000B7F90630002B08DAFB885B009BB283F4EB
:10503000815383F00103FB8002E0FB885B00FB806F
:10504000FB680133FB60FB68072BE9DDFB88184632
:105050001437BD465DF8047B7047F0B587B000AFEC
:105060000146C7E900230B46FB8100237B611BE05F
:10507000D7E900237969C1F12006A1F1200022FAC5
:1050800001F403FA06F6344323FA00F0044323FA4A
:1050900001F5E2B2FB8911461846FFF7AFFF034660
:1050A000FB817B6908337B617B693F2BE0DDFB89FA
:1050B00018461C37BD46F0BD80B584B000AF03462E
:1050C000B9607A60FB810AE0BB685A1CBA601A7842
:1050D000FB8911461846FFF791FF0346FB817B6869
:1050E0005A1E7A60002BEFD1FB8918461037BD4657
:1050F00080BD000080B584B000AF78600B467B8037
:105100000023FB817B681B785A2B2DD17B680133F0
:105110001B78A52B28D17B6802331B781A2B23D14F
:105120007B6803331B78022B1ED17B689B787B73D3
:105130007B7B9BB205339BB219467868FFF728FF4B
:105140000346002B10D10123FB810A4B01221A7266
:105150007B6803337A7B1946074812F005F8F8F7A5
:1051600045F90346034A1360B7F90E301846103765
:10517000BD4680BD001000201003002080B586B021
:1051800000AF78600B467B800023FB820023BB606E
:1051900000233B617B681B785A2B4AD17B68013323
:1051A0001B78A52B45D17B6802331B78272B40D178
:1051B0007B6804331B78032B3BD17B689B78FB73A4
:1051C0007B68DB78BB73FB7B9BB206339BB21946D3
:1051D0007868FFF7DDFE0346002B2AD17B680C338D
:1051E0001B68BB600123FB82164B1B68002B04D09D
:1051F000BA68144B1B689A4210D1134B3B61134B96
:1052000001221A72F8F7F2F80346104A13600D4BA8
:105210001B68002B02D1BB680A4A1360BB7B012BC1
:1052200009D138697B680433FA7B194611F09CFF79
:1052300002E000BF00E000BFB7F91630184618378B
:10524000BD4680BDE81000202C0300200C1000207B
:1052500080B586B000AFF860B9601346FB71FB689B
:10526000B3F5807F08D1A74B01221A72F8F7BEF878
:105270000346A44A136091E1FB68B3F5E07F06D1D1
:10528000FB791A46B968A04811F06EFF86E1FB6809
:1052900040F2C112934209D19A4B01221A72FB7952
:1052A0001A46B968994811F05FFF77E1FB68B3F5DA
:1052B000E17F06D1FB791A46B968954811F054FF91
:1052C0006CE1FB6840F2C312934240F083800023FC
:1052D000FB750023BB7509E0BB7DBA6813441A78DF
:1052E000FB7D1344FB75BB7D0133BB75BB7D072B79
:1052F000F2D9884B9B680133864A9360FB7D002B73
:1053000062D1FB791A46B968834811F02DFF814BB1
:105310001B78C3F30303DBB201337B4A927FC2F3F2
:105320000312D2B2934204D07A4B1B690133794AFB
:105330001361754B9B7FC3F30313D9B2754A13787E
:1053400061F303031370704B5B7E112B0CD1734B15
:105350001B78002B08D0714B00221A70704B002272
:105360001A80704B01221A70674B5B7E122B09D199
:105370006C4B1B78002B05D06A4B00221A70684BCF
:1053800000221A80604B5B7E142B0CD1664B1B787D
:10539000002B08D0644B00221A70614B00221A8047
:1053A000624B01221A70584B5B7E152B40F0F68041
:1053B0005E4B1B78002B00F0F1805C4B00221A70D2
:1053C000574B00221A80E9E0524BDB680133514A07
:1053D000D360E3E0FB68B3F5E27F06D1FB791A46C0
:1053E000B968534811F0C0FED8E0FB68B3F5F07F10
:1053F00019D9FB68B3F5F87F15D2424B01221A7216
:105400004C4B1B6801334B4A13604B4B1B7883F0AA
:105410000103DBB2002B06D0464B1B680A2B02DDD2
:10542000454B01221A70FB68312B33D0FB68312BBE
:10543000C0F0B380FB68B3F5F77F00F2AE80FB6885
:10544000B3F5F07F40F2A980FB68A3F2E1130D2BC6
:1054500000F2A38001A252F823F000BF9B5501087F
:105460009D540108B5540108C75401089B55010813
:105470009B5501089B550108D7540108F7540108B2
:105480005D550108695501087555010883550108E6
:105490008F550108294B01221A707FE0284B012209
:1054A0001A70284B0A221A700822B968264811F08F
:1054B0005BFE73E0254B01221A700822B96824486C
:1054C00011F052FE6AE01C4BBA6811331168196082
:1054D00092889A8062E00822B9681E4811F044FE62
:1054E000BB6804331B789B09DBB203F00303124A49
:1054F000C2F8173052E00822B968174811F034FE9C
:105500004CE000BFAC10002070100020781000208C
:105510008010002098100020881000201810002013
:10552000BC100020191000201A1000201B100020B1
:1055300090100020B8100020201000201D10002026
:105540001E10002053030020211000201F100020F7
:1055500029100020371000203F1000200822B968D1
:10556000134811F001FE19E00822B968114811F042
:10557000FBFD13E0BB681B889BB20F4AA2F83930D1
:105580000CE00822B9680D4811F0EEFD06E0072294
:10559000B9680B4811F0E8FD00E000BFF7F726FFFF
:1055A0000346084A136000BF1837BD4680BD00BFE0
:1055B0004710002051100020201000206110002012
:1055C00069100020AC10002080B582B000AF00232D
:1055D0003B6000237B60284B1B7883F00103DBB228
:1055E000002B45D0254B1B78012B41D9244B12228F
:1055F0009A71234B0022DA71214B9A79204BDB7987
:105600001344DAB21E4B1B7BC3F30313DBB21B0143
:10561000DBB21344DBB25AB2194B5A73184B93F9ED
:105620000D30DBB25B42DBB25AB2154B5A733B46CC
:1056300008221449184611F097FD114B1B7BC3F348
:105640000313DBB2013303F00F03D9B20C4A137B0F
:1056500061F3071313733B464FF4F07208211846A9
:1056600004F0D0FC054B1B78013BDAB2034B1A70F7
:1056700000BF0837BD4680BD201000205C0300201D
:10568000C0100020C610002080B582B000AF0023FB
:105690003B6000237B60614B1B7883F00103DBB22E
:1056A000002B06D15E4B1B7883F00103DBB2002B8D
:1056B00070D05A4B1B7883F00103DBB2002B03D070
:1056C000584B16229A7109E0554B1B7883F0010361
:1056D000DBB2002B02D0534B17229A71514B0022A0
:1056E000DA71504B9A794F4BDB791344DAB24D4B58
:1056F0001B7BC3F30313DBB21B01DBB21344DBB22E
:105700005AB2484B5A73474B93F90D30DBB25B42A8
:10571000DBB25AB2434B5A733B4608224249184601
:1057200011F022FD3F4B1B7BC3F30313DBB20133AC
:1057300003F00F03D9B23B4A137B61F307131373D2
:105740003B464FF4F0720821184604F05BFC374BDF
:105750001B78013BDAB2354B1A70344B1B78002BA7
:1057600056D1324B0A221A702C4B1B7883F001035E
:10577000DBB2002B03D0294B01221A7048E0284BE2
:105780001B7883F00103DBB2002B41D0244B0122B4
:105790001A703DE0234B12229A71254B1A78214B47
:1057A000DA71204B9A791F4BDB791344DAB21D4B27
:1057B0001B7BC3F30313DBB21B01DBB21344DBB26D
:1057C0005AB2184B5A73174B93F90D30DBB25B4248
:1057D000DBB25AB2134B5A733B46082212491846A1
:1057E00011F0C2FC0F4B1B7BC3F30313DBB201337D
:1057F00003F00F03D9B20B4A137B61F30713137342
:105800003B464FF4F0720821184604F0FBFB00E021
:1058100000BF00BF0837BD4680BD00BF1E1000207E
:105820001F100020C0100020C610002053030020CD
:10583000CE10002080B582B000AF3C4B1B7A012B0C
:1058400070D10320FDF780FC0346002B6AD00023B3
:10585000BB800023FB71FB795A1CFA711A46344B4A
:105860005A219954FB795A1CFA711A46304BA521DA
:105870009954FB795A1CFA711A462D4B04219954FC
:10588000FB795A1CFA711A46294B0A219954294B63
:105890001B78802B07D1FB795A1CFA711A46244BCE
:1058A0000121995406E0FB795A1CFA711A46204BE3
:1058B00000219954204BB3F90E3019B2FB795A1CD0
:1058C000FA711A46C9B21A4B99541B4BB3F91230EC
:1058D00019B2FB795A1CFA711A46C9B2144B995481
:1058E000154BB3F912301BB21B1219B2FB795A1CBB
:1058F000FA711A46C9B20E4B9954FB799BB21946FC
:105900000B48FFF745FB0346BB80FB79084A13446D
:10591000BA881A80FB790233FB71FB791946044877
:10592000FDF7A6FC00BF0837BD4680BD0C10002067
:10593000D0100020CE100020183A002080B586B08C
:1059400000AFA14B1B7A012B63D1A04B1B78052B19
:105950005FD1F7F74BFD02469D4B1B68D31ADE2B38
:1059600057D90023FB6000233B6100237B81F7F7BD
:105970003DFD0346964A1360964BDB889BB2BB8184
:10598000944BB3F908301BB21A46924BB3F9083066
:105990001BB203FB02F28F4BB3F90A301BB219465C
:1059A0008C4BB3F90A301BB201FB03F3134407EE2F
:1059B000903AF8EEE77AB0EE670A12F063F9F0EE8B
:1059C000407AFDEEE77A17EE903A1BB27B817B8935
:1059D000FB81804B1B889BB23B827E4BDB899BB259
:1059E0007B8207F10C034FF4F8720821184604F08B
:1059F00009FB784BD3F81630FB60764BD3F81A309E
:105A00003B6107F10C0340F2F1120821184604F043
:105A1000F9FA6D4B1B7A012B40F02781F7F7E6FC72
:105A200002466D4B1B68D31A642B40F21E81002383
:105A30003B6000237B60F7F7D9FC0346664A13609E
:105A4000FFF7C2FD654B1B78002B02D0FFF71CFE51
:105A50000BE1604BB3F912301BB29AB2604B9A80E3
:105A60005C4BB3F90E301BB2042B0CBF0123002397
:105A7000DBB203F00F03D9B2594A937961F3030300
:105A80009371574B9B79C3F30313DBB2013303F0DC
:105A90000F03D9B2524A937961F307139371514BB3
:105AA0001B78002B17D0504BB3F900309BB2013359
:105AB0009BB21AB24C4B1A804B4BB3F90030052BFA
:105AC00005DD484B00221A70474B00221A80444BD8
:105AD00011225A709BE0454B1B78002B1AD0424B89
:105AE000B3F900309BB201339BB21AB23E4B1A801D
:105AF0003D4BB3F90030052B05DD3C4B00221A70FD
:105B0000394B00221A80364B12225A70344B002235
:105B10005A807CE0364B1B78002B17D0324BB3F900
:105B200000309BB201339BB21AB22F4B1A802E4B1E
:105B3000B3F90030052B05DD2D4B00221A702A4BDE
:105B400000221A80264B14225A7060E0294B1B78E1
:105B5000002B1AD0244BB3F900309BB201339BB217
:105B60001AB2214B1A80204BB3F90030052B05DD0A
:105B7000204B00221A701C4B00221A80184B152251
:105B80005A70174B00225A8041E01B4B1B78002BA8
:105B900034D0154BB3F900309BB201339BB21AB22B
:105BA000114B1A80104BB3F90030052B05DD124B59
:105BB00000221A700C4B00221A80094B17225A70CF
:105BC000074B00225A8022E0AC100020D40F0020A6
:105BD000EC100020183A0020F010002020100020C7
:105BE0005403002018100020BC10002019100020C1
:105BF0001A1000201B1000201C1000201D4B10222A
:105C00005A701C4B00225A801B4B00221A803B46C4
:105C100007221849184611F0A7FA164B0022DA712C
:105C20000023FB750DE0134BDA79FB7D18333B4401
:105C300013F8183C1344DAB20E4BDA71FB7D0133D2
:105C4000FB75FB7D062BEED90A4BDB795B42DAB2A2
:105C5000084BDA714FF4D0720821064804F0D2F9EB
:105C6000064B5B680133054A536000BF1837BD46D9
:105C700080BD00BF54030020BC10002098100020FD
:105C800080B582B000AF1A23704A41F28831704863
:105C90000BF00CFB27236F4A41F288316E480BF062
:105CA00005FB28236D4A41F288316D480BF0FEFA5E
:105CB000674B1B7A012B5CD16A4B01221A706A4B2D
:105CC00002221A70614BB3F801309AB2664BA3F806
:105CD00001205E4BB3F803309AB2634BA3F8032064
:105CE0005A4BB3F805309AB25F4BA3F80520574BD7
:105CF000B3F807309BB21AB25B4BA3F80720534BA3
:105D0000D3F80930584AC2F80930504BB3F80D3077
:105D10009AB2554BA3F80D204C4BB3F80F309AB202
:105D2000514BA3F80F20494B5A7C4F4B5A74474BA9
:105D30005A8A4D4B5A82454B1A7D4B4B1A75434B31
:105D4000B3F815309AB2484BA3F815203F4BB3F87F
:105D500017309AB2444BA3F817203C4B5B7E9AB2A3
:105D6000414BA3F8192004224049414811F0FCF9A5
:105D70003CE2394B1B7A012B7CD13A4B01221A7041
:105D8000394B03221A70334BB3F80D309AB2364BAD
:105D9000A3F801202F4BB3F80F309AB2324BA3F87F
:105DA00003202C4BB3F811309AB22F4BA3F80520E7
:105DB000284BB3F813309BB21AB22B4BA3F8072031
:105DC000244BD3F81530284AC2F80930214BB3F8D8
:105DD00019309AB2244BA3F80D201E4BB3F81B3098
:105DE0009AB2214BA3F80F201A4B5A7F1E4B5A74BC
:105DF000184BDA8B1C4B5A82164B93F820201A4B07
:105E00001A75144BB3F821309AB2174BA3F815202A
:105E1000104BB3F823309AB2134BA3F817200D4B55
:105E2000B3F825309AB2104BA3F81920094BD3F8D8
:105E300009300D4AC2F823300B4B064A1B3301329E
:105E40001168526819605A60D0E100BF1003002049
:105E5000001000202C0300200C10002070100020E7
:105E6000AC100020E4100020D40F0020A49E0208F3
:105E7000EF0F00205A4B1B7A012B40F0A881594BA1
:105E800001221A70584B04221A70584B1B7883F069
:105E90000103DBB2002B00F0B780554B1A89524B3F
:105EA000A3F80120524B5B8907EE903AF8EEE77AAF
:105EB0009FED507A67EE877AFCEEE77A17EE903A1C
:105EC0009AB2494BA3F80320494B1B8A5B009AB254
:105ED000454BA3F80520464B5B8AA3F57A739BB22A
:105EE0005B009BB21AB2404BA3F80720404B1B6AE1
:105EF0003D4AC2F809303E4B9A8C3B4BA3F80D202B
:105F00003B4BDA8C384BA3F80F20394BDA7B364BFE
:105F10005A74374B9B8A23F010039AB2324B5A8241
:105F2000334B1B7B07EE903AF8EEE77AB6EE007A39
:105F300067EE877AFCEEE77AC7ED017A3B79DAB251
:105F4000294B1A752A4B5B7B9BB2283B9AB2264B96
:105F5000A3F81520244B0022DA7500221A76244B70
:105F60009B7B9BB2283B9AB21F4BA3F819201E4B78
:105F70001F4A1B3301321188927819809A701A4B8C
:105F80002D229A771A4B1B781B4A04211B4811F0CB
:105F900001F9174B1B791A46194B03FB02F2144BFC
:105FA0005B791946174B01FB03F31A44104B9B799D
:105FB00019464FF47A7301FB03F313440C4AD27968
:105FC00013441A46084BC3F82320094B1A7E064B8C
:105FD00083F82720064BDA7D034B83F8282005E160
:105FE000AC100020E4100020D40F0020201000206E
:105FF00070100020CDCCCC3DAC9E0208F30F0020E9
:1060000080969800A08601007A4B9B78422B0AD19B
:10601000784BDB78522B06D1764B1B794F2B02D174
:10602000754B05221A70734BB3F81F309AB2724B3E
:10603000A3F801206F4B1B8DC3F30B139BB207EE2C
:10604000903AF8EEE77A9FED6D7A67EE877AFCEE8C
:10605000E77A17EE903A9AB2674BA3F80320654BA4
:10606000B3F821309BB207EE903AF8EEE77A9FED55
:10607000647A67EE877AFCEEE77A17EE903A9AB286
:106080005D4BA3F805205B4BB3F923301BB207EE41
:10609000903AF8EEE77A9FED597A67EE877A9FEDAE
:1060A000597A77EEC77AFDEEE77A17EE903A1BB28F
:1060B0009BB21A46920013445B009BB21AB24E4B3D
:1060C000A3F807204B4BD3F809304B4AC2F80930EC
:1060D000484BB3F80D309AB2474BA3F80D20454B0F
:1060E000B3F80F309AB2444BA3F80F20414BDB7E3C
:1060F000C3F38113DBB21A463F4B5A743D4BB3F8DE
:1061000039309AB23C4B5A823A4B93F8333007EE0F
:10611000903AF8EEE77AB6EE007A67EE877AFCEE10
:10612000E77AC7ED017A3B79DAB2334B1A75314B16
:106130001B7F9BB2283B9AB22F4BA3F815202D4B07
:106140005B7F9BB2283B9AB22B4BA3F81720294BBD
:106150009B7F9BB2283B9AB2274BA3F81920264B72
:10616000244A1B3302321188927819809A70224B8C
:106170002D229A771F4B5B78234A0421234811F084
:1061800009F81C4B5B791A46214B03FB02F2194BB1
:106190009B7919461F4B01FB03F31A44154BDB791E
:1061A00019464FF47A7301FB03F31344114A127A30
:1061B00013441A46104BC3F823200E4BDB7EC3F367
:1061C0000113DBB21A460C4B83F827200EE0124B6A
:1061D0001B78012B0AD1104B02221A7029220021B0
:1061E000054810F0CFFF044BFF221A7000BF08379C
:1061F000BD4680BD20100020D40F0020CDCC4C3DEA
:10620000CDCCCC3D0000C843AC9E0208F30F00206B
:1062100080969800A0860100E410002080B500AFB1
:10622000642107480BF073F80346002B03D0FFF7F7
:1062300027FDFFF7FFFAFFF781FB00BF80BD00BF1E
:10624000F410002080B500AFF7F7D0F80346114AEC
:106250001361F7F7CBF803460F4A1361F7F7C6F857
:1062600003460E4A1361F7F7C1F803460C4A13615F
:10627000F7F7BCF803460B4A1361F7F7B7F8034684
:10628000094A1361F7F7B2F80346084A136100BFE1
:1062900080BD00BFF81000200C110020201100204C
:1062A00034110020481100205C11002070110020E2
:1062B00090B583B000AF0446084611461A462346FF
:1062C000FB710346BB710B467B7113463B71FB7937
:1062D000002B1ED1BB79642202FB03F31A46744BD8
:1062E0005A607B79642202FB03F31A46704B9A6072
:1062F000002201216F48F9F78BFA3B796C4AD36091
:10630000F7F774F803466A4A1361694B00221A7062
:10631000CAE0FB79012B1ED1BB79642202FB03F397
:106320001A46654B5A607B79642202FB03F31A46D6
:10633000614B9A60002202215E48F9F769FA3B79C5
:106340005D4AD360F7F752F803465B4A13615A4B34
:1063500000221A70A8E0FB79022B1ED1BB796422BF
:1063600002FB03F31A46554B5A607B79642202FB09
:1063700003F31A46514B9A60002204214D48F9F765
:1063800047FA3B794D4AD360F7F730F803464B4A5A
:1063900013614A4B00221A7086E0FB79032B1ED151
:1063A000BB79642202FB03F31A46454B5A607B79A2
:1063B000642202FB03F31A46414B9A600022052136
:1063C0003C48F9F725FA3B793D4AD360F7F70EF8D8
:1063D00003463B4A13613A4B00221A7064E0FB7992
:1063E000042B1ED1BB79642202FB03F31A46354B02
:1063F0005A607B79642202FB03F31A46314B9A60A0
:10640000002203212B48F9F703FA3B792D4AD36088
:10641000F6F7ECFF03462B4A13612A4B00221A7051
:1064200042E0FB79052B1ED1BB79642202FB03F30A
:106430001A46254B5A607B79642202FB03F31A4605
:10644000214B9A60002206211A48F9F7E1F93B79BD
:106450001D4AD360F6F7CAFF03461B4A13611A4B65
:1064600000221A7020E0FB79062B1DD1BB79642233
:1064700002FB03F31A46154B5A607B79642202FB38
:1064800003F31A46114B9A60002207210948F9F7D5
:10649000BFF93B790D4AD360F6F7A8FF03460B4AD4
:1064A00013610A4B00221A7000BF0C37BD4690BD25
:1064B000F810002000040048201100200C110020DA
:1064C000341100205C1100204811002070110020C0
:1064D00080B500AF9F4BB3F90230122B00F044831C
:1064E0009D4B1B7883F00103DBB2002B1ED0F6F727
:1064F0007DFF034643F69722934205D801220121EE
:106500009648F9F785F911E0F6F770FF0246944BCB
:106510001B68D31AB3F5FA6F08D901218F48F9F730
:10652000A7F9F6F763FF03468D4A13608D4BDB68CE
:10653000002B18D18C4BDB68002B14D18B4BDB6804
:10654000002B10D18A4BDB68002B0CD1894BDB6808
:10655000002B08D1884BDB68002B04D1874BDB680C
:10656000002B00F003837C4B1B78002B00F00D8385
:106570007C4BDB68002B64D07A4B9B6846F29C32E4
:10658000934205D0774B5B6846F29C3293421BD115
:10659000744B0022DA60734B9B6846F29C32934244
:1065A00005D1002201216D48F9F732F9E0E26D4B87
:1065B0005B6846F29C32934240F0DA82012201216C
:1065C0006648F9F725F9D3E2664B1B78FF2B1AD101
:1065D000F6F70CFF0246634B1B69D21A614B5B68EE
:1065E0009A4240F2D2825F4BDB68013B5D4AD36046
:1065F000002201215948F9F70BF9FFF723FE594B07
:1066000000221A70C1E2F6F7F1FE0246554B1B69F3
:10661000D21A544B9B689A4240F2B782514BDB68C6
:10662000002B00F0B282012201214C48F9F7F0F86A
:10663000F6F7DCFE03464B4A13614A4BFF221A7001
:10664000A3E24A4BDB68002B64D0484B9B6846F2C0
:106650009C32934205D0454B5B6846F29C32934294
:106660001BD1424B0022DA60404B9B6846F29C32C1
:10667000934205D1002202213848F9F7C9F879E29E
:106680003A4B5B6846F29C32934240F0738201229F
:1066900002213248F9F7BCF86CE2344B1B78FF2B2F
:1066A0001AD1F6F7A3FE0246304B1B69D21A2F4BC4
:1066B0005B689A4240F269822C4BDB68013B2B4AB3
:1066C000D360002202212548F9F7A2F8FFF7BAFDAE
:1066D000264B00221A7058E2F6F788FE0246234B3A
:1066E0001B69D21A214B9B689A4240F24E821F4B83
:1066F000DB68002B00F04982012202211748F9F7DC
:1067000087F8F6F773FE0346184A1361174BFF220A
:106710001A703AE2144BDB68002B7BD0124B9B685B
:1067200046F29C32934205D00F4B5B6846F29C3296
:10673000934232D10C4B0022DA600B4B9B6846F23D
:106740009C3293421CD1002204210448F9F760F8DE
:1067500012E200BFEC4F0020A03A002000040048E5
:1067600084110020F81000200C11002020110020BE
:1067700048110020341100205C110020701100200D
:10678000A34B5B6846F29C32934240F0F5810122B4
:106790000421A048F9F73CF8EEE19D4B1B78FF2B54
:1067A0001AD1F6F723FE0246994B1B69D21A984B71
:1067B0005B689A4240F2E981954BDB68013B944A61
:1067C000D360002204219348F9F722F8FFF73AFD3D
:1067D0008F4B00221A70D8E1F6F708FE02468C4B68
:1067E0001B69D21A8A4B9B689A4240F2CE81884B31
:1067F000DB68002B00F0C981012204218548F9F7EC
:1068000007F8F6F7F3FD0346814A1361804BFF2238
:106810001A70BAE1804BDB68002B64D07E4B9B681A
:1068200046F29C32934205D07B4B5B6846F29C3229
:1068300093421BD1784B0022DA60774B9B6846F27B
:106840009C32934205D1002205217248F8F7E0FFFF
:1068500094E1714B5B6846F29C32934240F08E812A
:10686000012205216B48F8F7D3FF87E16A4B1B78BB
:10687000FF2B1AD1F6F7BAFD0246674B1B69D21AF5
:10688000654B5B689A4240F28081634BDB68013B59
:10689000614AD360002205215E48F8F7B9FFFFF78F
:1068A000D1FC5D4B00221A706FE1F6F79FFD0246A6
:1068B000594B1B69D21A584B9B689A4240F265812A
:1068C000554BDB68002B00F0608101220521514807
:1068D000F8F79EFFF6F78AFD03464F4A13614E4BC9
:1068E000FF221A7051E14D4BDB68002B64D04B4BFB
:1068F0009B6846F29C32934205D0484B5B6846F257
:106900009C3293421BD1454B0022DA60434B9B687B
:1069100046F29C32934205D1002203213D48F8F70C
:1069200077FF2DE13D4B5B6846F29C32934240F08D
:106930002781012203213748F8F76AFF20E1374B0E
:106940001B78FF2B1AD1F6F751FD0246334B1B691A
:10695000D21A324B5B689A4240F217812F4BDB68A8
:10696000013B2E4AD360002203212A48F8F750FF4A
:10697000FFF768FC294B00221A7006E1F6F736FD96
:106980000246264B1B69D21A244B9B689A4240F25E
:10699000FC80224BDB68002B00F0F78001220321F2
:1069A0001C48F8F735FFF6F721FD03461B4A136133
:1069B0001A4BFF221A70E8E0194BDB68002B6ED0EF
:1069C000174B9B6846F29C32934205D0144B5B6890
:1069D00046F29C32934225D1114B0022DA60104BD3
:1069E0009B6846F29C32934205D100220621094859
:1069F000F8F70EFFC6E00A4B5B6846F29C32934202
:106A000040F0C080012206210248F8F701FFB9E0FA
:106A10000C11002000040048341100205C110020FB
:106A200048110020594B1B78FF2B1AD1F6F7DEFCDA
:106A30000246564B1B69D21A544B5B689A4240F28D
:106A4000A480524BDB68013B504AD36000220621F0
:106A50004F48F8F7DDFEFFF7F5FB4C4B00221A70AC
:106A600093E0F6F7C3FC0246484B1B69D21A474B2A
:106A70009B689A4240F28980444BDB68002B00F00F
:106A80008480012206214248F8F7C2FEF6F7AEFCE8
:106A900003463E4A13613D4BFF221A7075E03D4BA1
:106AA000DB68002B71D03B4B9B6846F29C329342D3
:106AB00005D0384B5B6846F29C3293421AD1354B75
:106AC0000022DA60334B9B6846F29C32934205D138
:106AD000002207212E48F8F79BFE55E02D4B5B68FE
:106AE00046F29C3293424FD1012207212848F8F701
:106AF0008FFE49E0274B1B78FF2B19D1F6F776FC68
:106B00000246244B1B69D21A224B5B689A423CD93D
:106B1000204BDB68013B1F4AD360002207211C4841
:106B2000F8F776FEFFF78EFB1A4B00221A702CE066
:106B3000F6F75CFC0246174B1B69D21A154B9B6893
:106B40009A4222D9134BDB68002B1ED00122072169
:106B50000F48F8F75DFEF6F749FC03460D4A13614E
:106B60000C4BFF221A7010E000BF0EE000BF0CE0DB
:106B700000BF0AE000BF08E000BF06E000BF04E07D
:106B800000BF02E000BF00E000BF80BD4811002050
:106B9000000400487011002080B586B000AFF86096
:106BA000B9601346FB7100237B610023FB74FB6813
:106BB000DBB203F07F03FB74FB7C162B02D1984BF6
:106BC0007B6101E0974B7B617B69DB33FA79013AAA
:106BD000B9680A4412781A707B6993F8DB3023F0A5
:106BE0007F03DBB2002B0AD07B69002283F8D82018
:106BF000002283F8D9207B69012283F8DA207B699F
:106C0000B3F9D8301BB21A46FB791344C82B14DDF4
:106C10007B69181D7B69B3F9D8301BB21A46002175
:106C200010F0B0FA7B69002283F8D820002283F8A4
:106C3000D9207B69002283F8DA207B6993F8DA3067
:106C4000002B1CD07B69B3F9D8301BB21A467B6984
:106C50001344181DFB79013B1A46B96810F084FAF9
:106C60007B69B3F9D8301BB29AB2FB799BB213445B
:106C70009BB2013B9BB21AB27B69A3F8D8207B6917
:106C800093F8DA30002B00F0C6807B6993F8DB3094
:106C900003F04003DBB2002B00F0BD807B690022D3
:106CA00083F8DA207B69012283F8D420F6F79EFB73
:106CB00002467B69C3F8CC207B6993F8DB3023F074
:106CC0007F03DBB2002B40F095807B69B3F9D830AD
:106CD0001BB2072B40F38E807B699A1D7B69B3F949
:106CE000D8301BB29BB2023B9BB21946104600F053
:106CF0009DF84D4B1B881A467B691B7919467B69A9
:106D00005B791B020B449A4274D17B69B3F9D8308A
:106D10001BB2023B442B66D87B69B3F9D8301BB257
:106D2000322B1BD17B69002242F00C0283F8202118
:106D3000002283F821217B6903F1DC007B690633A3
:106D40002822194610F010FA7B6903F584707B69DC
:106D50002E330822194610F007FA4BE07B69B3F98D
:106D6000D8301BB2422B1BD17B69002242F00C02AF
:106D700083F82021002283F821217B6903F1DC00C4
:106D80007B6906332822194610F0EEF97B6903F57A
:106D900084707B692E331822194610F0E5F929E03A
:106DA0007B69B3F9D8301BB2362B05D07B69B3F9B8
:106DB000D8301BB2462B1DD17B69002242F00E0257
:106DC00083F82021002283F821217B6903F1DC0074
:106DD0007B69991D7B69B3F9D8301BB2023B1A4617
:106DE00010F0C2F906E07B69DC3346220021184628
:106DF00010F0C8F97B69181D7B69B3F9D8301BB254
:106E00001A46002110F0BEF97B69002283F8D820D1
:106E1000002283F8D92000BF1837BD4680BD00BFCF
:106E200088110020AC120020CE13002080B582B063
:106E300000AF78600B467B80064B4FF6FF721A80DE
:106E40007B881946786800F03FF800BF0837BD46D8
:106E500080BD00BFCE13002080B485B000AF0346D4
:106E6000FB71FB791B021AB2164B1B881BB25340F5
:106E70001BB29AB2134B1A800023FB6017E0114B30
:106E80001B881BB2002B09DA0E4B1B885B009BB2E0
:106E900083F4815383F001039BB203E0094B1B8809
:106EA0005B009BB2074A1380FB680133FB60FB6801
:106EB000072BE4D900BF00BF1437BD465DF8047B43
:106EC000704700BFCE13002080B582B000AF78605D
:106ED0000B467B8006E07B685A1C7A601B7818465C
:106EE000FFF7BAFF7B885A1E7A80002BF3D100BFD0
:106EF00000BF0837BD4680BD80B584B000AF02201A
:106F0000FCF722F90346002B31D0A34B93F8243130
:106F1000002B0BD0A14B1B79A14AC821184604F0C5
:106F20008DFD9D4B002283F8242120E09A4B93F89D
:106F30002531002B0BD0994B1B79994AC921184652
:106F400004F07CFD944B002283F825210FE0924B46
:106F500093F82631002B0AD0904B1B79904ACA2116
:106F6000184604F06BFD8C4B002283F826218A4BD7
:106F700093F81D3183F00103DBB2002B40F0B081A8
:106F8000F6F734FA0246874B1B68D31A312B40F2CE
:106F9000A981F6F72BFA0346824A13600023BB81CE
:106FA00000237B600023BB600023FB730023BB73C3
:106FB0007A4B1B79382B02D15623BB7310E0774BE9
:106FC0001B79332B02D11123BB7309E0734B1B795F
:106FD000342B02D11223BB7302E0704B1B79BB73BD
:106FE0006E4B5B79CA2B00F04781CA2B00F37C8182
:106FF000C82B03D0C92B00F02A8175E1BB7B3B7104
:10700000664BD3F80630C7F805303B79DE2B00F32A
:10701000B180DA2B0FDA782B00F0AE80782B00F3FA
:10702000A980562B73D0562B00F3A480112B13D0BC
:10703000122B45D09EE0DA3B042B00F29B8001A28C
:1070400052F823F075710108757101087571010816
:10705000757101085D710108534B93F8CD30152B04
:1070600007D13B1D053303225049184610F07CF828
:1070700084E04D4B93F8CD301B2B07D13B1D0533DE
:1070800003224B49184610F06FF877E0464B93F80F
:10709000CD30182B07D13B1D053303224549184637
:1070A00010F062F86AE0404B93F84032252B65D12E
:1070B0003B1D053303224049184610F055F85DE0AA
:1070C000394B93F8D830162B07D13B1D05330322DB
:1070D0003649184610F048F852E0334B93F8D83050
:1070E000192B07D13B1D053303223249184610F0F6
:1070F0003BF845E02C4B93F87432262B40D13B1DD6
:10710000053303222D49184610F02EF838E0264B9F
:1071100093F8C830142B07D13B1D053303222349B4
:10712000184610F021F82DE01F4B93F8C8301A2BA9
:1071300028D11D4B93F83C32012B07D13B1D053361
:1071400003221F49184610F00FF81BE03B1D0533C2
:1071500003221C49184610F007F813E0124B1B7D60
:10716000002B11D13B1D05330322174918460FF0A0
:10717000FBFF09E000BF08E000BF06E000BF04E03D
:1071800000BF02E000BF00E000BF3B1D0F4A082126
:10719000184602F097FEACE00C000020300A0020F8
:1071A000360A0020DC130020903B0020B09E02082D
:1071B000B49E0208B89E0208BC9E0208C09E020847
:1071C000C49E0208C89E0208CC9E02080014380023
:1071D000FB7B002B24D1484B5B789BB2023B9BB2DC
:1071E00019464648FDF7D4FE0346BB81FE233B719A
:1071F000FE237B71BB7BBB713F4B5B78023BDBB2F9
:10720000FB713D4B9B793B723B4BDB797B72BB89BE
:10721000DBB2BB72BB891B0A9BB2DBB2FB7207E01D
:10722000FB7B354A99183B1D082218460FF09CFF3E
:10723000FB7B0833FB733B1D314A0821184602F0E3
:1072400041FE3B1D0822002118460FF09BFF2A4BF0
:107250005B785A1DFB7B9A4248DB2A4BB3F81E3100
:107260009BB21A46244B9B791946234BDB791B02B0
:107270000B449A42ACD039E0BB7B3B713B1D224AA8
:107280000821184602F01EFE1E4B002283F81D2125
:10729000BB7B112B13D11D4B93F8CD301B2B04D08E
:1072A0001A4B93F84032252B03D1194B002283F857
:1072B0002C205922002117480FF064FF18E0BB7BF7
:1072C000562B15D1114B93F8CD301A2B02D1124BFE
:1072D00000225A765922002110480FF053FF07E090
:1072E00000BF06E000BF04E000BF02E000BF00E016
:1072F00000BF1037BD4680BD300A0020380A00208C
:10730000001440000C00002000144800903B0020B6
:1073100080490020003F0020B8150020A43E002036
:1073200080B58CB008AF78607B6804331B78012B84
:1073300040F0F981AD4B04221A707B681B78DE2B7C
:1073400000F3F381DA2B11DA782B00F0F081782B3F
:1073500000F3EB81562B00F00781562B00F3E581FB
:10736000112B15D0122B00F0CB80DEE1DA3B042B81
:1073700000F2DB8101A252F823F000BF2B77010855
:107380002B7701082B7701082B7701081777010865
:107390007B6801330322964918460FF0D5FE034659
:1073A000002B0CD1F6F722F80346924A1360914B5A
:1073B00001225A72904B152283F8CD20BAE17B68E6
:1073C000013303228D4918460FF0BEFE0346002B01
:1073D0003ED18B4B01221A72F6F708F80346884A11
:1073E0001360874B01225A72834B1B2283F8CD20F6
:1073F000834B44225A77824B57229A77804B312213
:10740000DA777F4B4E2283F820200423FB7307E0BA
:10741000FB7B7B4A134430225A77FB7B0133FB739F
:10742000FB7B092BF4D906230693764B05930023A7
:107430000493002303930A230293734B01930023C5
:107440000093002300220C2170480AF043FC71E1F4
:107450007B68013303226E4918460FF075FE034620
:10746000002B0ED1F5F7C2FF0346634AC2F854322F
:10747000614B012283F85C225F4B252283F8402276
:1074800058E15F4B01221A72F5F7B0FF03465C4AE0
:1074900013605B4B01225A72574B1B2283F8CD209D
:1074A000574B44225A77564B57229A77544B3122E6
:1074B000DA77534B4F2283F820200423BB7307E075
:1074C000BB7B4F4A134430225A77BB7B0133BB73DB
:1074D000BB7B092BF4D9062306934A4B0593002363
:1074E0000493002303930A230293474B0193002341
:1074F0000093002300220C2144480AF0EBFB19E121
:107500007B68013303223A4918460FF01DFE0346FB
:10751000002B0FD13F4B01221A72F5F767FF03468C
:107520003C4A13603B4B01225A72334B162283F8BC
:10753000D820FEE07B6801330322374918460FF05C
:1075400003FE0346002B40F0F480F5F74FFF03469F
:10755000294AC2F88832284B012283F89022264B10
:10756000262283F87422E4E07B6801330322204959
:1075700018460FF0E9FD0346002B0FD1274B0122DF
:107580001A72F5F733FF0346244A1360234B012296
:107590005A72194B142283F8C820CBE07B68013360
:1075A00003221F4918460FF0CFFD0346002B5BD185
:1075B0001C4B01221A72F5F719FF0346194A136092
:1075C000184B01225A720C4B1A2283F8C820154B13
:1075D0004422DA76134B53221A77124B31225A7710
:1075E000104B4E229A7704237B7325E0C4030020BE
:1075F000B09E0208F0480020903B0020B49E020894
:1076000080490020D09E02089D490020003F0020B4
:10761000BC9E020838490020C09E0208E8130020E2
:10762000C89E0208B81500207B7B444A13443022D0
:10763000DA767B7B01337B737B7B092BF4D90623C2
:1076400006933F4B059300230493002303930A23DF
:1076500002933C4B019300230093002300220B2153
:1076600039480AF037FB65E07B680133032237496C
:1076700018460FF069FD0346002B0ED1F5F7B6FE54
:107680000346334AC2F83432314B012283F83C229C
:107690002F4B252283F82C224CE0284B01221A7212
:1076A000F5F7A4FE0346254A1360244B01225A72C3
:1076B000274B1A2283F8C820204B4422DA761F4B2E
:1076C00053221A771D4B31225A771C4B4F229A773F
:1076D00004233B7307E03B7B184A13443022DA76DD
:1076E0003B7B01333B733B7B092BF4D90623069389
:1076F000134B059300230493002303930A2302935F
:10770000104B019300230093002300220B210E480D
:107710000AF0E0FA0EE07B68013303220D491846B7
:107720000FF012FD06E000BF04E000BF02E000BF62
:1077300000E000BF1037BD4680BD00BFB815002077
:10774000D49E0208D3150020A43E0020C49E020847
:10775000903B0020CC9E020880B485B000AFF8605A
:10776000B9601346FB71BB6801331B78062B11D13E
:10777000BB6802331B78F22B0CD1BB6803331B7838
:10778000AA2B07D1BB681A786C4B9A706B4B0222FC
:107790005A70CCE0BB6801331B78062B11D1BB6853
:1077A00002331B78F22B0CD1BB6803331B78552BAB
:1077B00007D1BB681A78614B9A70604B03225A70EC
:1077C000B5E0BB681A785D4B9B789A424CD1BB6898
:1077D00001331B78062B47D1BB6802331B78F42B8F
:1077E00042D1BB6803331B78002B3DD1BB68043307
:1077F0001B78FF2B38D1BB6805331B78FF2B33D1A7
:10780000BB6806331B78FF2B2ED1BB6807331B7870
:10781000FF2B29D1494B5B78032B07D1474B04221F
:107820005A70474B012283F824217FE0434B5B7859
:10783000052B03D0414B5B78072B77D13F4B5B681F
:1078400080333E4A53603E4BB3F81E319BB2013346
:107850009AB23B4BA3F81E21384B04225A70384B86
:10786000012283F8252161E0BB681A78334B9B78AD
:107870009A422ED1BB6801331B78062B29D1BB68F5
:1078800002331B78F42B24D1BB6803331B78002B05
:107890001FD1BB6804331B78042B04D0BB680433AE
:1078A0001B78082B15D1BB6805331B78002B10D132
:1078B000BB6806331B78FF2B0BD1BB6807331B78E3
:1078C000FF2B06D11D4B05225A701C4B0A229A72BF
:1078D0002DE0BB681A78194B9B789A4227D1BB6878
:1078E00001331B78062B22D1BB6802331B78F42BA3
:1078F0001DD1BB6803331B78072B18D1BB68043339
:107900001B78FF2B13D1BB6805331B78FF2B0ED1DF
:10791000BB6806331B78FF2B09D1BB6807331B7884
:10792000FF2B04D1054B04225A7000E000BF00BFBA
:107930001437BD465DF8047B704700BFD0130020AC
:107940000C00002080B582B000AF78607B681B78A7
:107950009BB21B029AB27B6801331B789BB2134423
:107960009BB21AB2184B1A807B6802331B789BB209
:107970001B029AB27B6803331B789BB213449BB201
:107980001AB2114B5A807B6804331B789BB21B02DE
:107990009AB27B6805331B789BB213449BB21AB230
:1079A000094B9A80084BB3F90020084B9A81F5F7F0
:1079B0001DFD0346054A1360044B01221A7200BFE5
:1079C0000837BD4680BD00BFE013002060030020E3
:1079D00080B584B000AFF860B9601346FB71FB68F6
:1079E000A3F54073132B00F2888001A252F823F014
:1079F000417A0108FB7A0108FB7A0108FB7A010849
:107A0000FB7A0108FB7A0108FB7A0108FB7A01087E
:107A1000FB7A0108FB7A0108FB7A0108FB7A01086E
:107A2000FB7A0108FB7A0108FB7A0108FB7A01085E
:107A3000FB7A0108AF7A0108DF7A0108ED7A0108C4
:107A4000BB6803331A78BB6804331B781344DAB27B
:107A5000BB6805331B781344DAB2BB6806331B7866
:107A60001344DAB2274B9A73BB6807331A78254B55
:107A70009B7B9A420ED1BB6804331B789BB21B02DE
:107A80009AB2BB6803331B789BB213449BB21AB201
:107A90001C4B9A81F5F7AAFC03461A4A1360194B4E
:107AA00001221A72184B142283F8C82026E0174BC3
:107AB000BA681068516803C3F5F798FC0346124A88
:107AC000C2F83432104B012283F83C220E4B1422B0
:107AD00083F82C220C4B142283F8C8200EE00B4BA9
:107AE000BA6808331068516803C307E0074BBA68E7
:107AF00010331068516803C300E000BF00BF1037A7
:107B0000BD4680BDE8130020903B002044140020B7
:107B100090B58FB008AFF860B9601346FB71FB6891
:107B2000984A934240F09080BB68DA79964BDA71BC
:107B3000964B01221A72F5F759FC0346934A1360DB
:107B4000914BDB7903F00203DBB2002B1AD0072242
:107B5000B9688D480FF008FB8B4B1B781E2B02D9A0
:107B6000894B1E221A708A4B00221A70864B1B7892
:107B7000002B61D1874B1B78002B5DD1864B0022F7
:107B80001A7059E0804BDB7903F00103DBB2002B64
:107B900042D07D4B1B78012B18D07D4B1B780833CE
:107BA000794A9818784B1B789A007C4B83FB021318
:107BB00013449910D317C91A0B46DB005B1AD11A6C
:107BC0000B461A46B9680FF0CFFA07E0704B1B78E6
:107BD00008336D4A1344BA6812681A606A4BB3F8E6
:107BE00003309CB2684B1B789BB29B009BB219463A
:107BF0006B48FDF7CDF903469C421DD1654B1B78C0
:107C0000002B19D1604B1B7802339B001A465E494A
:107C100061480FF0A9FA0FE05D4B1B7808335A4A10
:107C200013440722B96818460FF09EFA584B1B7888
:107C30000733DAB2564B1A70554B1B78F72B22D903
:107C4000534B00221A701EE0FB68564A93421AD129
:107C5000554B01221A72F5F7C9FB0346524A1360CD
:107C6000524B1A2283F8C820BB6803331B789AB2A0
:107C7000BB6804331B789BB21B029BB213449BB2BC
:107C80001AB2494B9A81FB68494A934240F0A4805A
:107C9000BB681B78012B40F09F8000237B61BB6891
:107CA000DA79394BDA71384BDB7903F00203DBB256
:107CB000002B31D0BB6801331B687B617B690922D3
:107CC0003C49184609F054FA7A693B4BA3FB02136E
:107CD0009B0D3A4901FB03F3D31A394A934203D867
:107CE000314B4F229A7702E02F4B4E229A77062390
:107CF0000693344B0593002304930023039300233E
:107D0000029300230193092300932A4B00220B21A5
:107D10002D4809F0DFFFEFE01B4BDB7903F0010397
:107D2000DBB2002B00F0E880BB6801331B687B618D
:107D30007B6906222549184609F01AFA1A4B442293
:107D4000DA76194B53221A77174B31225A770623CA
:107D500006931C4B059300230493002303930A23EB
:107D600002931B4B019300230093002300220B215D
:107D7000154809F0AFFF0C4B01225A76154B04222F
:107D80001A70B9E0001390005C140020A0150020C8
:107D90009A1500209B150020FC1400209324499282
:107DA0006414002001139000B8150020903B0020BF
:107DB00001139800E91500206BCA5F6B809698004C
:107DC00056312600DC9E0208A43E0020D715002074
:107DD000D3150020C4030020FB684A4A934222D1F5
:107DE000BB681B78082B03D0BB681B78052B1AD106
:107DF000BB681B78082B03D1434B012283F82E204C
:107E0000BB6801331B789AB2BB6802331B789BB204
:107E10001B029BB213449BB21BB2562207211620B1
:107E200003F076FE69E0FB68364A934222D1BB68D4
:107E30001B78092B03D0BB681B78072B1AD1BB68B2
:107E40001B78092B03D1304B012283F82F20BB680C
:107E500001331B789AB2BB6802331B789BB21B02BA
:107E60009BB213449BB21BB256220821162003F08A
:107E70004FFE42E0FB68234A934222D1BB681B7845
:107E80000A2B03D0BB681B780B2B1AD1BB681B785D
:107E90000B2B03D11C4B012283F83020BB6801332C
:107EA0001B789AB2BB6802331B789BB21B029BB251
:107EB00013449BB21BB256220F21162003F028FE5A
:107EC0001BE0FB680F4A934217D1BB681B78042B59
:107ED00013D1BB6801331B789AB2BB6802331B789D
:107EE0009BB21B029BB213449BB21BB2002209211E
:107EF000162003F00DFE00E000BF00BF1C37BD469A
:107F000090BD00BF01139800B815002090B58FB048
:107F100008AFF860B9601346FB71FB689F4A934253
:107F200040F09080BB68DA799D4BDA719D4B01225D
:107F30001A72F5F75BFA03469A4A1360984BDB799D
:107F400003F00203DBB2002B1AD00722B968944871
:107F50000FF00AF9924B1B781E2B02D9904B1E2270
:107F60001A70914B00221A708D4B1B78002B61D137
:107F70008E4B1B78002B5DD18D4B00221A7059E07F
:107F8000874BDB7903F00103DBB2002B42D0844B3B
:107F90001B78012B18D0844B1B780833804A981823
:107FA0007F4B1B789A00834B83FB02131344991079
:107FB000D317C91A0B46DB005B1AD11A0B461A46B7
:107FC000B9680FF0D1F807E0774B1B780833744A93
:107FD0001344BA6812681A60714BB3F803309CB24C
:107FE0006F4B1B789BB29B009BB219467248FCF703
:107FF000CFFF03469C421DD16C4B1B78002B19D13F
:10800000674B1B7802339B001A46654968480FF09E
:10801000ABF80FE0644B1B780833614A1344072226
:10802000B96818460FF0A0F85F4B1B780733DAB237
:108030005D4B1A705C4B1B78F72B22D95A4B0022F0
:108040001A701EE0FB685D4A93421AD15C4B012214
:108050001A72F5F7CBF90346594A1360594B1B22A4
:1080600083F8CD20BB6803331B789AB2BB68043316
:108070001B789BB21B029BB213449BB21AB2504BAB
:10808000DA81FB68504A934240F0F6804F4B012260
:108090001A72F5F7ABF903464C4A1360494B252297
:1080A00083F84022BB68DA79494BDA71484BDB79B7
:1080B00003F00203DBB2002B0FD00722B96844485B
:1080C0000FF052F8424B1B78822B02D9404B822290
:1080D0001A70404B00221A60C5E03D4BDB7903F07B
:1080E0000103DBB2002B00F0AF80394B1B78012B72
:1080F00072D0374B1B781A4613469B001A442D4BFF
:1081000083FB021313449910D317C91A0B46DB00E3
:108110005B1AD11A002931D02E4B1B6808332C4A28
:1081200098182B4B1B781A4613469B001A44214B78
:1081300083FB021313449910D317C91A0B46DB00B3
:108140005B1AD11A0B461A46B9680FF00DF8204B8E
:108150001B781A4613469B001A44164B83FB0213E6
:1081600013449910D317C91A0B46DB005B1AD11AB6
:10817000184B1B680B44174A13603CE0154B1B68F7
:108180000833134A13440722B96818460EF0ECFF6F
:10819000104B1B6807330F4A13602CE00013A0003C
:1081A0005C140020A01500209A1500209B150020CB
:1081B000FC14002093244992641400200113A000B1
:1081C00080490020903B00201013A000AC15002037
:1081D000141600201C1B0020924B1B680833924A87
:1081E00013440522B96818460EF0BEFF8D4B1B687C
:1081F00005338C4A13608C4BB3F803309CB28A4B26
:108200001B789BB21A46920013449BB219468748CA
:10821000FCF7BEFE03469C4225D1854B1B78002B04
:1082200021D1814B1A78834B5A707F4B1B781A46A9
:1082300013469B0013441A467C497F480EF094FF76
:108240007E4B01221A700EE0764B1B680833764A8B
:1082500013440722B96818460EF086FF714B1B685D
:108260000733704A13606F4B1B6840F2F54293422C
:1082700002DD6C4B00221A60FB68714A93423BD1CD
:10828000BB6801331B789AB2BB6802331B789BB280
:108290001B029BB213449BB21AB26A4B1A80BB6892
:1082A00003331B789AB2BB6804331B789BB21B0262
:1082B0009BB213449BB21AB2624B5A80BB6805331F
:1082C0001B789AB2BB6806331B789BB21B029BB229
:1082D00013449BB21AB25B4B9A80F5F787F80346BA
:1082E000594AC2F85432584B012283F85C22564B4B
:1082F000252283F8402262E0FB68544A93422DD144
:10830000BB6801331B789AB2BB6802331B789BB2FF
:108310001B029BB213449BB21AB24A4BDA80BB6871
:1083200003331B789AB2BB6804331B789BB21B02E1
:108330009BB213449BB21AB2424B1A81BB680533FD
:108340001B789AB2BB6806331B789BB21B029BB2A8
:1083500013449BB21AB23B4B5A8130E0FB683C4A53
:1083600093422CD1BB6801331B789AB2BB680233AD
:108370001B789BB21B029BB213449BB21AB2314BC7
:108380009A81BB6803331B789AB2BB6804331B78AD
:108390009BB21B029BB213449BB21AB2294BDA81E7
:1083A000BB6805331B789AB2BB6806331B789BB257
:1083B0001B029BB213449BB21AB2224B1A82FB6877
:1083C000244A934240F0A480BB681B78012B40F004
:1083D0009F8000237B61BB68DA791F4BDA711E4BEB
:1083E000DB7903F00203DBB2002B5AD0BB68013308
:1083F0001B687B617B6909221849184608F0B8FEA2
:108400007A69174BA3FB02139B0D164901FB03F37B
:10841000D31A154A93422BD8144B4F2283F82020AD
:108420002AE000BF1C1B0020141600201C16002090
:108430009C150020201B0020221B0020101E002065
:108440000213A00000160020903B00200313A000A0
:108450000413A0000113A8005C140020B1490020FF
:108460006BCA5F6B809698005631260080490020C9
:10847000954B4E2283F8202006230693934B0593B9
:10848000002304930023039300230293002301930A
:10849000092300938E4B00220C218E4809F01AFC10
:1084A00050E18D4BDB7903F00103DBB2002B00F0D0
:1084B0004981BB6801331B687B617B690622874960
:1084C000184608F055FE804B44225A777E4B5722BF
:1084D0009A777D4B3122DA77062306937B4B0593FF
:1084E00000230493002303930A2302937C4B0193FC
:1084F00000230093002300220C21764809F0EAFBB8
:10850000714B012283F82C20764B04221A7019E15A
:10851000FB68754A934222D1BB681B78082B03D0B5
:10852000BB681B78052B1AD1BB681B78082B03D1BD
:10853000654B012283F82E20BB6801331B789AB269
:10854000BB6802331B789BB21B029BB213449BB2E5
:108550001BB211220721162003F0DAFAF3E0FB68C0
:10856000614A934222D1BB681B78092B03D0BB68B8
:108570001B78072B1AD1BB681B78092B03D1524BF0
:10858000012283F82F20BB6801331B789AB2BB68A5
:1085900002331B789BB21B029BB213449BB21BB2EB
:1085A00011220821162003F0B3FACCE0FB684E4AF2
:1085B000934222D1BB681B780A2B03D0BB681B787F
:1085C0000B2B1AD1BB681B780B2B03D13E4B01221E
:1085D00083F83020BB6801331B789AB2BB68023342
:1085E0001B789BB21B029BB213449BB21BB211229D
:1085F0000F21162003F08CFAA5E0FB683A4A93425B
:1086000016D1BB681B78042B12D1BB6801331B78D1
:108610009AB2BB6802331B789BB21B029BB2134415
:108620009BB21BB200220921162003F071FA8AE0E6
:10863000FB682E4A934221D1BB681B780D2B03D0D7
:10864000BB681B780C2B19D1BB681B780D2B02D192
:10865000274B01221A73BB6801331B789AB2BB689F
:1086600002331B789BB21B029BB213449BB21AB21B
:108670001F4B1A801F4B01221A7064E0FB681B4AD3
:10868000934239D1BB681B780F2B03D0BB681B7892
:108690000E2B31D1BB681B780F2B02D1144B01225A
:1086A0005A73BB6801331B789AB2BB6802331B78DC
:1086B0009BB21B029BB213449BB21AB20C4B5A8062
:1086C0000C4B01221A703EE080490020DC9E02081B
:1086D000B1490020003F00205C140020A149002087
:1086E0009D490020C40300200113A8000213A80024
:1086F00030140020111E0020FB68154A934222D13D
:10870000BB681B780A2B03D0BB681B780B2B1AD1D4
:10871000BB681B780B2B02D10E4B01221A74BB686D
:1087200001331B789AB2BB6802331B789BB21B02E1
:108730009BB213449BB21AB2064B9A80064B01229D
:108740001A7000E000BF00BF1C37BD4690BD00BFDF
:108750000213A80030140020111E002090B585B02F
:1087600000AFF860B9601346FB71FB68A14A934201
:1087700040F0CD80A04B262283F87422BB68DA79C2
:108780009E4BDA719D4BDB7903F00203DBB2002BC9
:1087900008D00722B96899480EF0E6FC984B0022F1
:1087A0001A60ABE0954BDB7903F00103DBB2002BE1
:1087B00000F09580914B1B78012B54D08F4B1B7888
:1087C0001A4613469B001A448E4B83FB0213134434
:1087D0009910D317C91A0B46DB005B1AD11A00296E
:1087E00031D0874B1B680833844A9818834B1B7819
:1087F0001A4613469B001A44824B83FB0213134410
:108800009910D317C91A0B46DB005B1AD11A0B4615
:108810001A46B9680EF0A8FC784B1B781A46134626
:108820009B001A44774B83FB021313449910D31710
:10883000C91A0B46DB005B1AD11A714B1B680B443B
:108840006F4A13601EE06E4B1B6808336B4A13447B
:108850000722B96818460EF087FC694B1B6807337E
:10886000674A13600EE0664B1B680833634A134483
:108870000522B96818460EF077FC614B1B6805337A
:108880005F4A1360604B1B7A012B37D05B4BB3F808
:1088900003309CB2594B1B789BB21A46920013448A
:1088A0009BB219465948FCF773FB03469C4225D1FD
:1088B000574B1B78002B21D1504B1A78554B5A70CF
:1088C0004E4B1B781A4613469B0013441A464F49D9
:1088D00051480EF049FC514B01221A700EE0484BF2
:1088E0001B680833454A13440722B96818460EF03E
:1088F0003BFC434B1B680733414A1360404B1B68EA
:1089000040F2F542934202DD3D4B00221A60FB68C3
:10891000434A93423BD1BB6801331B789AB2BB6890
:1089200002331B789BB21B029BB213449BB21AB258
:108930003C4B1A80BB6803331B789AB2BB68043384
:108940001B789BB21B029BB213449BB21AB2354BED
:108950005A80BB6805331B789AB2BB6806331B7814
:108960009BB21B029BB213449BB21AB22D4B9A804E
:10897000F4F73CFD0346204AC2F888321E4B012220
:1089800083F890221C4B262283F87422F2E0FB68C5
:10899000254A93424AD1BB6801331B789AB2BB681F
:1089A00002331B789BB21B029BB213449BB21AB2D8
:1089B0001C4BDA80BB6803331B789AB2BB68043364
:1089C0001B789BB21B029BB213449BB21AB2154B8D
:1089D0001A81BB6805331B789AB2BB6806331B78D3
:1089E0009BB21B029BB213449BB21AB20D4B5A812D
:1089F000C0E000BF1013B000903B0020281E0020F4
:108A00003023002093244992AC150020301E002012
:108A100034230020201B0020221B0020101E0020D9
:108A20000213B000141E00200313B000FB68534A69
:108A300093422DD1BB6801331B789AB2BB680233D5
:108A40001B789BB21B029BB213449BB21AB24C4BD5
:108A50009A81BB6803331B789AB2BB6804331B78D6
:108A60009BB21B029BB213449BB21AB2444BDA81F5
:108A7000BB6805331B789AB2BB6806331B789BB280
:108A80001B029BB213449BB21AB23D4B1A8271E097
:108A9000FB683C4A934221D1BB681B780A2B03D068
:108AA000BB681B780B2B19D1BB681B780B2B02D131
:108AB000354B01225A74BB6801331B789AB2BB68EC
:108AC00002331B789BB21B029BB213449BB21AB2B7
:108AD0002D4B5A812D4B01221A704BE0FB68294A1D
:108AE000934221D1BB681B780D2B03D0BB681B7848
:108AF0000C2B19D1BB681B780D2B02D1224B012204
:108B00009A73BB6801331B789AB2BB6802331B7837
:108B10009BB21B029BB213449BB21AB21A4BDA806F
:108B20001A4B01221A7025E0FB68164A934221D1A4
:108B3000BB681B780F2B03D0BB681B780E2B19D199
:108B4000BB681B780F2B02D10F4B0122DA73BB6875
:108B500001331B789AB2BB6802331B789BB21B02AD
:108B60009BB213449BB21AB2074B1A81074B0122E6
:108B70001A70FFE700BF1437BD4690BD0413B00064
:108B8000141E00200213B80030140020111E002013
:108B900080B58AB000AFF860B9601346FB7100235E
:108BA0007B628F4B1B68FA689A4239D08D4B1B68E9
:108BB000FA689A4234D08C4B1B78002B0BD18A4B2D
:108BC00003221A70864B7B627B6AFA681A60874BB5
:108BD00001221A7040E0864B1B78002B0BD1844B8E
:108BE00003221A707F4B7B627B6AFA681A607F4BA4
:108BF00002221A7030E07C4B1B78002B05D07A4B98
:108C00001B78013BDAB2784B1A70794B1B78002B3A
:108C100022D0774B1B78013BDAB2754B1A701BE000
:108C20006F4B1B68FA689A4208D16F4B03221A7087
:108C30006B4B7B627B6AFA681A600EE0694B1B68BB
:108C4000FA689A4209D16A4B03221A70654B7B621B
:108C50007B6AFA681A6000E000BF7B6A002B00F0B4
:108C6000D58104226349B8680EF06EFA0346002BE2
:108C70000AD17B6A002283F8CC20002283F8CD2021
:108C80007B6A012283F8CE207B6AB3F9CC301BB219
:108C90001A46FB791344C82B14DD7B6A181D7B6AC6
:108CA000B3F9CC301BB21A4600210EF06BFA7B6A86
:108CB000002283F8CC20002283F8CD207B6A00229A
:108CC00083F8CE207B6A93F8CE30002B19D07B6AD4
:108CD000B3F9CC301BB21A467B6A13440433FA79D9
:108CE000B96818460EF040FA7B6AB3F9CC301BB273
:108CF0009AB2FB799BB213449BB21AB27B6AA3F877
:108D0000CC207B6A93F8CE30002B00F07F817B6A09
:108D1000181D7B6AB3F9CC301BB2374A194608F0EC
:108D2000CFF80346002B00F071817B6A002283F8A4
:108D3000CE207B6ADB7AFB77FB7FBB2B40F04A813E
:108D40007B6A9B7ABB77BB7FBE2B00F24381BB7FE4
:108D500008337A6A13441B791B02BA7F0932796A95
:108D60000A4412791344BB617B6A0C33BA7F114603
:108D70001846FCF7E5F803469BB2BA699A4240F000
:108D800029817B6A1B7A9BB21B029AB27B6A5B7A4F
:108D90009BB21344FB827B6A012283F8D7207B6A53
:108DA00093F8E13083F00103DBB2002B43D07B6A00
:108DB000B3F9E2301BB29BB201339BB21AB27B6AA9
:108DC000A3F8E2207B6AB3F9E2301BB2012B15D184
:108DD000F4F70CFB02467B6AC3F8E4202BE000BFEB
:108DE0004C230020B02400205326002035230020EF
:108DF00054260020E49E0208EC9E02087B6AB3F928
:108E0000E2301BB2092B16DD7B6A002283F8E220D8
:108E1000002283F8E320F4F7E9FA02467B6AD3F8EC
:108E2000E430D31A3B613B697A4A934203D87B6AA8
:108E3000012283F8E120F4F7D9FA02467B6AC3F8ED
:108E4000CF20FB8AB3F5034F00F0A080B3F5034FAA
:108E500000F3C280B3F5024F69D0B3F5024F00F3BF
:108E6000BB80002B03D0B3F5407F31D0B4E0BB7F93
:108E7000422B00F2B380002387F8233020E097F8DC
:108E8000233004335B007A6A13441B799BB21B02C4
:108E900099B297F823305B0009337A6A13441B793F
:108EA0009AB297F823300A4491B27A6A74335B001D
:108EB00013440A469A8097F82330013387F8233009
:108EC000BB7F5B08DBB297F823209A42D7D385E0BB
:108ED000BB7F122B00F28480002387F822301EE033
:108EE00097F8223004335B007A6A13441B799BB2F3
:108EF0001B0299B297F822305B0009337A6A134457
:108F00001B799BB297F822200B4499B27B6A9C3262
:108F100023F8121097F82230013387F82230BB7FF4
:108F20005B08DBB297F822209A42D9D358E0BB7F86
:108F3000042B1BD8002387F8213012E097F821304A
:108F400003F1080297F82130796A0A4411797A6AA4
:108F500013440A4683F8522197F82130013387F8E9
:108F6000213097F82120BB7F9A42E7D37B6A03F533
:108F7000A9730422284918460EF0E6F80346002B90
:108F800030D17B6A012283F8DC202BE07B6A01224E
:108F900083F8DB20BB7F0C2B26D8002387F82030FA
:108FA00012E097F8203003F1080297F82030796A30
:108FB0000A4411797A6A13440A4683F8562197F8CD
:108FC0002030013387F8203097F82020BB7F9A4269
:108FD000E7D309E000BF08E000BF06E000BF04E0FF
:108FE00000BF02E000BF00E000BF7B6A181D7B6A83
:108FF000B3F9CC301BB21A4600210EF0C3F87B6ADD
:10900000002283F8CC20002283F8CD2000BF28372F
:10901000BD4680BD3F4B4C003823002080B582B058
:1090200000AF6D4B1B7883F00103DBB2002B55D0F2
:109030006A4B93F8E13083F00103DBB2002B4DD093
:10904000F4F7D4F9034647F22F52934246D8F4F787
:10905000CDF90246624B1B68D31AFA2B3ED9F4F7BE
:10906000C5F903465E4A13605E4B5A221A705D4B87
:1090700046225A705B4B4B229A705A4B4A22DA7046
:10908000584B80221A71574B00225A71554B0122BE
:109090009A71544BBB22DA71524B79221A72514B9E
:1090A0009B7919465048FBF74BFF0346FB80B7F905
:1090B00006301B121BB2DAB24A4B5A72FB88DAB284
:1090C000484B9A72474B4522DA72464B4E221A732E
:1090D000444B44225A73404B01221A703E4B1B787A
:1090E000002B07D03C4B00221A70404A0E213D480D
:1090F00000F0E8FE3E4B1B78002B09D03C4B0022D1
:109100001A70364B1B681A4611213A4800F0DAFEF5
:10911000324B93F8D730012B4BD1304B93F8E130E1
:10912000002B46D02D4B93F8DB3083F00103DBB2EC
:10913000002B3ED0304B1B7883F00103DBB2002BB9
:1091400037D0F4F753F902462C4B1B68D31AB3F50A
:109150007A7F2ED9F4F74AF90346284A1360284B40
:109160005A221A70264B46225A70254B4B229A706F
:10917000234B4A22DA70224B83221A71204B0022A1
:109180005A711F4B00229A711D4BBB22DA711C4B86
:10919000FF221A721A4BFF225A72194B45229A72F9
:1091A000174B4E22DA72164B44221A73124B0122CD
:1091B0001A70114B1B78002B09D00F4B00221A702C
:1091C000064B1B681A460D210D4800F07BFE00BFC0
:1091D0000837BD4680BD00BF502600204C2300202C
:1091E00048260020142600201C26002000003515EB
:1091F0005126002024260020522600204C26002044
:109200003826002084B080B500AF07F1080C8CE848
:109210000F003B69002B40F0C580BB6840F2134251
:10922000934200F23D81B3F5826F61D840F2034270
:10923000934200F23581B3F5806F4FD8B3F5457F87
:1092400080F02E81B3F5447F66D840F2023293421B
:1092500000F22681B3F5407F54D8B3F5407F29D082
:10926000B3F5407F00F21C81B3F5047F2CD0B3F539
:10927000047F00F21581B3F5F87F80F01181B3F51A
:10928000F07F7BD2B3F5E27F00F20A81B3F5E07F95
:1092900056D2B3F5807F5DD0B3F5807F00F20081B8
:1092A000FB2B43D0FB2B00F2FB80312B5CD03D2B02
:1092B0006ED0F5E07F4B1B687E4A1269D2B27E49C0
:1092C0001846FEF785FBEEE07A4B1B68794A126977
:1092D000D2B27949184601F027FAE4E0754B1B68D1
:1092E000744A1269D2B27449184608F049FFDAE0AC
:1092F000704B1B686F4A1269D2B26F49184608F06A
:109300003FFFD0E06B4B1B686A4A1269D2B26A49D0
:10931000184609F09BF9C6E0664B1B68654A12695E
:10932000D2B265491846FEF753FBBCE0614B1B689F
:10933000604A1269D2B26049184609F0F5F9B2E004
:109340005C4B1B685B4A1269D2B25B491846FBF75B
:109350007FFFA8E0574B1B68564A1269D2B25649A4
:109360001846FBF775FF9EE0524B1B68514A126985
:10937000D2B251491846FBF76BFF94E04D4B1B6886
:109380004C4A1269D2B24C491846FBF761FF8AE099
:10939000484B1B68474A1269D2B247491846FEF744
:1093A000DBF980E03B69042B7CD1FB68434A9342A4
:1093B00064D0424A93426AD8414A934267D2414AB2
:1093C000934224D244F26E62934260D844F26C62BB
:1093D00093424AD243F26E62934258D843F26C628F
:1093E000934239D242F26E62934250D842F26C629A
:1093F000934228D2B3F5866F03D8B3F5826F10D2AB
:1094000045E0A3F5B3530C3B022B40D812E0294BA7
